:100000000C9446160C9477160C9477160C9477166D
:100010000C9477160C9477160C9477160C9477162C
:100020000C9477160C9477160C9477160C9477161C
:100030000C9477160C9448590C9477160C947716F8
:100040000C9477160C9440C40C9477160C94771685
:100050000C9477160C9477160C9473760C94FE58C7
:100060000C9477160C94B14B0C9477160C9477166D
:100070000C9477160C9477160C9477160C947716CC
:100080000C9477160C9477160C9477160C947716BC
:100090000C9477160C9477160C9477160C947716AC
:1000A0000C9477160C9477160C9477160C9477169C
:1000B0000C9477160C9477160C9477160C9477168C
:1000C0000C9477160C9477160C9477160C9477167C
:1000D0000C9477160C9477160C9463580C9424584F
:1000E0000C9477168731A431D531F2310732303292
:1000F0009D320333AC33F4370238FB3722382638CD
:1001000040389B3C5538A138C838EF3818396E391B
:100110007F399039A139B239C3399B3CA63B9B3C0E
:10012000B13B213C273C473CF3B0F6B0E5B0E9B029
:10013000EFB02DB1FAB0FEB004B108B10CB112B1FC
:1001400016B11AB12DB120B124B128B18DB692B635
:1001500097B6A1B6ABB624B7B5B6BDB6C5B6CFB6E1
:10016000D9B6E3B6F2B6FCB624B706B710B71AB7DD
:10017000084AD73B3BCE016E84BCBFFDC12F3D6C0E
:1001800074319ABD56833DDA3D00C77F11BED9E474
:10019000BB4C3E916BAAAABE000000803F05A84C54
:1001A000CDB2D44EB93836A9020C50B99186880820
:1001B0003CA6AAAA2ABE000000803F004E414E493C
:1001C0004E495459494E46CDCCCC3D0AD7233C1715
:1001D000B7D13877CC2B329595E6241FB14F0A0062
:1001E0000020410000C84200401C4620BCBE4CCA52
:1001F0001B0E5AAEC59D74434F4D4D554E4943415C
:1002000054494F4E0044525952554E004552524F98
:10021000525300494E464F004543484F0047322F46
:1002200047332062616420706172616D657465722C
:10023000730A00206F6620004D424C20473239205F
:10024000706F696E74200059206F7574206F66207E
:1002500072616E67652028312D35292E0A005820DD
:100260006F7574206F662072616E67652028312D6E
:1002700035292E0A004D6573682070726F62696EB1
:100280006720646F6E652E0A005374617274206D6E
:100290006573682070726F62696E67207769746831
:1002A0002022473239205331222066697273742E1E
:1002B0000A004732380A47323920533200537461FA
:1002C00074653A20004D65736820626564206C6532
:1002D00076656C696E6720686173206E6F2064615B
:1002E00074612E0A0053206F7574206F662072614E
:1002F0006E67652028302D35292E0A004D657368FC
:1003000020706F696E742063616E6E6F7420626519
:10031000207265736F6C7665640A00456E642066B2
:10032000696C65206C6973740A00426567696E20A8
:1003300066696C65206C6973740A00286E6F2066AC
:10034000696C6529005344207072696E74696E6728
:10035000206279746520004E6F74205344207072BF
:10036000696E74696E670A0043757272656E7420F7
:1003700066696C653A20002569730025696D202542
:100380006973002569682025696D2025697300253A
:100390006964202569682025696D20256973002519
:1003A000697920256964202569682025696D2025E3
:1003B0006973005072696E742074696D653A20002B
:1003C0006F6E2E0A006F66662E0A00473236204492
:1003D000656275672000180213020C020502F7011E
:1003E0006F66660044454255473A004B494C4C45C0
:1003F000442E20004D3131332053006F6B002C20F0
:10040000002C2000544845524D414C5F50524F54EF
:10041000454354494F4E004155544F5245504F5259
:10042000545F53445F53544154555300454D455216
:1004300047454E43595F5041525345520043415343
:10044000455F4C494748545F4252494748544E45DE
:10045000535300544F47474C455F4C49474854530A
:1004600000534F4654574152455F504F5745520035
:100470004255494C445F50455243454E54004C450B
:1004800056454C494E475F44415441005A5F5052D3
:100490004F4245004155544F4C4556454C00505233
:1004A000494E545F4A4F420050524F4752455353B2
:1004B000004155544F5245504F52545F54454D5092
:1004C00000564F4C554D45545249430045455052F6
:1004D0004F4D0053455249414C5F584F4E5F584F66
:1004E0004646004649524D574152455F4E414D45A3
:1004F0003A4D61726C696E20312E312E39202847B9
:1005000069746875622920534F555243455F434FC4
:1005100044455F55524C3A68747470733A2F2F6794
:1005200069746875622E636F6D2F4D61726C696EB0
:100530004669726D776172652F4D61726C696E20CC
:1005400050524F544F434F4C5F56455253494F4EB4
:100550003A312E30204D414348494E455F54595061
:10056000453A3344205072696E7465722045585480
:1005700052554445525F434F554E543A31205555DC
:1005800049443A63656465326132662D34316132C3
:100590002D343734382D396231322D633535633699
:1005A000326633363766660A002F2F20002054004B
:1005B000205200416363656C65726174696F6E3AC5
:1005C0002050005741524E494E4721204C6F772012
:1005D0005A204A65726B206D6179206C65616420D8
:1005E000746F20756E77616E7465642070617573C9
:1005F00065732E0A00546F6F206661722066726FF9
:100600006D207265666572656E636520706F696ED8
:10061000740A0020466C6F773A20000001363726B6
:10062000032BFFFFFF3C3D382AFFFFFFFF2E303E2C
:1006300012FFFFFFFFFFFFFF0809FF2C071A1C181E
:10064000FFFFFF08440A2C4324221E20643A0020A6
:10065000693A0020703A00496E76616C69642065E1
:10066000787472756465720A0043290A0061626CCD
:10067000656420286D696E2074656D702000436F7D
:100680006C6420657874727564657320617265208E
:100690000020643A0020693A0020703A004E6F2032
:1006A00063617365206C696768740A004545505240
:1006B0004F4D204F4B0A00205A004475616C204575
:1006C0006E6473746F702041646A7573746D656EC7
:1006D0007420286D6D293A20003F4B2076616C759F
:1006E00065206F7574206F662072616E67652028C3
:1006F000302D3130292E0A00416476616E63652009
:100700004B3D004163746976652045787472756469
:1007100065723A2000496E76616C69642065787470
:1007200072756465720A0043616E6E6F7420656E47
:10073000746572207375626469723A2000473931BA
:100740000A4731205A2D302E30320A4739300053B3
:1007500070656369616C204D656E753A205A20445E
:100760006F776E20302E310A004739310A47312029
:100770005A2D302E30320A47393000537065636984
:10078000616C204D656E753A205A20446F776E205B
:10079000302E30320A004739310A4731205A2B3087
:1007A0002E30320A473930005370656369616C201E
:1007B0004D656E753A205A20557020302E30320A21
:1007C000004739310A4731205A2B302E310A473938
:1007D00030005370656369616C204D656E753A2019
:1007E0005A20557020302E310A00473239205332BA
:1007F000005370656369616C204D656E753A204EDB
:10080000657874204D65736820506F696E740A00B6
:10081000473239205331005370656369616C204D54
:10082000656E753A205374617274204D657368204B
:100830004C6576656C696E670A004D313430205323
:100840003630005370656369616C204D656E753A92
:100850002050726568656174204265640A004D35F8
:100860003031005370656369616C204D656E753A77
:10087000205265616420454550524F4D0A004D3568
:100880003030005370656369616C204D656E753A58
:10089000205361766520454550524F4D0A004D3337
:1008A000303320452D312053363020433130205510
:1008B00031005370656369616C204D656E753A2037
:1008C0004175746F2054756E6520486F746265645D
:1008D000205069640A004D31303620533137380AD0
:1008E0004D333033204530205332313020433130C6
:1008F000205531005370656369616C204D656E75DC
:100900003A204175746F2054756E6520486F746588
:100910006E64205049440A003C5370656369616C01
:100920005F4D656E753E003C5370656369616C5F39
:100930004D656E753E002F002F002F002F2E2E0AC2
:10094000002F2E2E002F2E2E003C53706563696100
:100950006C5F4D656E753E0A003C5370656369615E
:100960006C204D656E753E003C5370656369616C2B
:10097000204D656E753E003C5265616420454550D2
:10098000524F4D3E003C5265616420454550524FE8
:100990004D3E003C4175746F2054756E6520486F64
:1009A00074626564205049443E003C4175746F2078
:1009B00054756E6520486F74626564205049443EEA
:1009C000003C4175746F2054756E6520486F7465E6
:1009D0006E64205049443E003C4175746F2054754C
:1009E0006E6520486F74656E64205049443E003C3B
:1009F000457869743E003C457869743E003C53611B
:100A0000766520454550524F4D3E003C536176651A
:100A100020454550524F4D3E003C4E657874204D68
:100A200065736820506F696E743E003C4E65787443
:100A3000204D65736820506F696E743E003C53749E
:100A4000617274204D657368204C6576656C696EC3
:100A5000673E003C5374617274204D657368204C8E
:100A60006576656C696E673E003C507265686561CD
:100A700074206265643E003C507265686561742054
:100A80006265643E003C5A20446F776E20302E3100
:100A90003E003C5A20446F776E20302E313E003CA1
:100AA0005A20446F776E20302E30323E003C5A2060
:100AB000446F776E20302E30323E003C5A20557005
:100AC00020302E30323E003C5A20557020302E30DF
:100AD000323E003C5A20557020302E313E003C5AA8
:100AE00020557020302E313E0056313136004A33C9
:100AF0003320004D3530300A4D3432302053310A26
:100B00004731205A313020463234300A473120589C
:100B100030205930204636303030004A3232004AD8
:100B20003232004731205A3520463234300A4731BC
:100B30002058313930205932302046363030300A92
:100B40004731205A302046323430004731205A3560
:100B500020463234300A473120583139302059315B
:100B600039302046363030300A4731205A3020465E
:100B7000323430004731205A3520463234300A476B
:100B8000312058313930205932302046363030301B
:100B90000A4731205A302046323430004739310A72
:100BA0004731205A313020463234300A4739300A32
:100BB0004732380A4732390A4731205832302059F3
:100BC00032302046363030300A4731205A30204605
:100BD000323430004A3032004A3132004731205A34
:100BE0003130004F4B004731205A31300047393007
:100BF00000473120452569463530300047312045D2
:100C00002D302E314625690047312045302E3146A2
:100C10002569004731205A2569462569004731205A
:100C20005A2D302E31462569004731205A302E3159
:100C30004625690047312059256946256900473115
:100C400020592D302E314625690047312059302E4C
:100C500031462569004731205825694625690047F6
:100C60003120582D302E314625690047312058302B
:100C70002E31462569004739310047323800473266
:100C800038205A004732382059004732382058005F
:100C90004132305620004731205A3130004A30343A
:100CA000004A3231004A3230004B494C4C45442E08
:100CB00020004A303400454E4400464E20004A3061
:100CC00032003939393A393939004D004800413755
:100CD000562000413656202D2D2D004A303200413D
:100CE000365620005A3A2000593A2000583A20003F
:100CF00041355600413456200041335620004132E0
:100D0000562000413156200041305620004D3834E5
:100D1000004A3136004A3138004739310A4731201C
:100D20005A313020463234300A473930004A3134A3
:100D3000004A3030004A3031004A31300024F4D4C7
:100D40003050C38E20C2A24017828B7011127A914C
:100D50000D816CD90AA861E108C758660761514343
:100D6000061E4B5D05C145A7041A411104093D98B3
:100D700003713931034036DB0265339102D43054BC
:100D800002802E1D02632CEE01752AC501B028A039
:100D900001102781018F2564012B244B01E02234AF
:100DA00001AC211F018D200D01801FFC00841EED70
:100DB00000971DDF00B81CD200E61BC600201BBC3C
:100DC00000641AB200B219A8000A19A0006A1899A2
:100DD00000D117910040178B00B516840031167EA4
:100DE00000B31579003A157300C7146F0058146AE0
:100DF00000EE1366008813630025135E00C7125BC4
:100E0000006C12570015125400C111510070114F9F
:100E10000021114B00D61049008D104700461044A8
:100E20000002104200C00F4000800F3E00420F3C05
:100E300000060F3B00CB0E3800930E37005C0E35DA
:100E400000270E3400F30D3200C10D3100900D303B
:100E500000600D2E00320D2D00050D2C00D90C2B3D
:100E600000AE0C2900850C29005C0C2700350C27EE
:100E7000000E0C2600E80B2400C40B2400A00B235A
:100E8000007D0B23005A0B2100390B2100180B2089
:100E900000F80A1F00D90A1E00BB0A1E009D0A1D89
:100EA00000800A1D00630A1C00470A1B002C0A1B55
:100EB00000110A1A00F7091A00DD091900C40919FE
:100EC00000AB091900920917007B09180063091784
:100ED000004C09160036091600200916000A0915EB
:100EE00000F5081500E0081400CC081400B8081438
:100EF00000A4081400900813007D0812006B08136A
:100F00000058081200460812003408110023081186
:100F1000001208110001081100F0071000E007108E
:100F200000D0071000C0071000B0070F00A1071085
:100F30000091070E0083070F0074070F0065070E6E
:100F40000057070E0049070E003B070D002E070E45
:100F50000020070D0013070D0006070D00F9060C11
:100F600000ED060D00E0060C00D4060C00C8060CCF
:100F700000BC060C00B0060C00A4060B0099060C81
:100F8000008D060B0082060B0077060B006C060B2B
:100F90000061060A0057060B004C060A0042060ACA
:100FA0000038060A002E060A0024060A001A060A5D
:100FB000001006090007060A00FD050900F40509EE
:100FC00000EB050900E2050900D9050900D0050973
:100FD00000C7050900BE050900B5050800AD0508F4
:100FE00000A50509009C050800940508008C05086B
:100FF00000840508007C050800740508006C0507DE
:1010000000650508005D050700560508004E050748
:1010100000470507004005080038050700310507AF
:10102000002A050700230507001C05060016050712
:10103000000F0507000805060002050700FB04066F
:1010400000F5040700EE040600E8040600E20407C9
:1010500000DB040600D5040600CF040600C9040620
:1010600000C3040600BD040600B7040600B1040571
:1010700000AC040600A6040600A00405009B0406BC
:101080000095040500900406008A04050085040507
:1010900000800406007A040500750405007004054C
:1010A000006B04050066040500610405005C04058E
:1010B0000057040500520405004D040500480405CE
:1010C00000430405003E0404003A0405003504050D
:1010D00000300404002C0405002704040023040548
:1010E000001E0404001A0404001604050011040480
:1010F000000D0404000904050004040400000404B5
:1011000000FC030400F8030400F4030400F00304EB
:1011100000EC030400E8030400E4030400E003041B
:1011200000DC030400D8030400D4030400D003044B
:1011300000CC030400C8030300C503030024F40427
:10114000D9201BC40C5C0E9804C4095F02650771AA
:1011500001F405F900FB04B30048048700C10369EA
:10116000005803550003034500BE023A00840231D3
:101170000053022A002902250004022000E4011C79
:1011800000C8011900AF0117009801140084011371
:1011900000710110006101100051010E0043010DAA
:1011A0000036010B002B010B0020010B001501097B
:1011B000000C01090003010800FB000800F300080F
:1011C00000EB000700E4000600DE000600D8000681
:1011D00000D2000600CC000500C7000500C20005D3
:1011E00000BD000400B9000400B5000400B1000413
:1011F00000AD000400A9000400A5000300A2000344
:10120000009F0004009B000300980003009500026B
:101210000093000300900003008D0002008B000388
:1012200000880002008600020084000300810002A2
:10123000007F0002007D0002007B000200790002B6
:1012400000770001007600020074000200720001C5
:1012500000710002006F0002006D0001006C0002CE
:10126000006A0001006900020067000100660001D9
:1012700000650001006400020062000100610001DD
:1012800000600001005F0002005D0001005C0001E1
:10129000005B0001005A00010059000100580001E4
:1012A00000570001005600010055000100540001E4
:1012B00000530000005300010052000100510001E2
:1012C00000500001004F0001004E0000004E0001E0
:1012D000004D0001004C0001004B0000004B0001DC
:1012E000004A0001004900010048000000480001D8
:1012F00000470001004600000046000100450000D4
:1013000000450001004400010043000000430001CB
:1013100000420000004200010041000000410001C5
:1013200000400001003F0000003F0001003E0000BF
:10133000003E0001003D0000003D0001003C0000B7
:10134000003C0000003C0001003B0000003B0001AD
:10135000003A0000003A00010039000000390001A5
:10136000003800000038000000380001003700009D
:101370000037000100360000003600000036000192
:101380000035000000350000003500010034000089
:10139000003400000034000100330000003300007E
:1013A0000033000100320000003200000032000172
:1013B0000031000000310000003100010030000069
:1013C0000030000000300001002F0000002F00005E
:1013D000002F0000002F0001002E0000002E000052
:1013E000002E0001002D0000002D0000002D000047
:1013F000002D0001002C0000002C0000002C00003B
:10140000002C0001002B0000002B0000002B00002E
:10141000002B0001002A0000002A0000002A000022
:10142000002A000100290000002900000029000016
:101430000029000000290001002800000028000009
:1014400000280000002800000028000100270000FC
:1014500000270000002700000027000000270001EF
:1014600000260000002600000026000000260000E4
:1014700000260001002500000025000000250000D6
:1014800000250000002500000025000100240000C8
:1014900000240000002400000024000000240001BB
:1014A00000230000002300000023000000230000B0
:1014B00000230000002300000023000100220000A0
:1014C0000022000000220000002200000022000094
:1014D0000022000100210000002100000021000086
:1014E0000021000000210000002100000021000177
:1014F000002000000020000000200000002000006C
:10150000002000000020000000200000002000015A
:10151000001F0000001F0000001F0000001F00004F
:10152000001F0000001F0000001F0001001E00003F
:10153000001E0000001E0000001E000000232C0002
:1015400000B8220000561800003A0F0000B808004A
:1015500000B1040000710200003E010000696E202D
:101560006D6F76655F746F282920666565645F76A8
:10157000616C756520666F722058593A002C2065A1
:10158000793D0029202D3E202865783D002C2073D0
:10159000793D0020436F6E6E656374696E672077D6
:1015A00069746820766572746963616C206C696E19
:1015B00065202873783D002C2065793D0029202D79
:1015C0003E202865783D002C2073793D0020436F34
:1015D0006E6E656374696E67207769746820686FE2
:1015E00072697A6F6E74616C206C696E6520287305
:1015F000783D003F53706563696669656420582CC7
:101600005920636F6F7264696E617465206F7574C1
:10161000206F6620626F756E64732E0A003F285239
:101620002965706561742076616C7565206E6F74D4
:1016300020706C61757369626C653B206D757374A5
:10164000206265206174206C6561737420312E0AFC
:10165000003F2852296570656174206D7573742090
:101660006265207370656369666965642077686583
:101670006E206E6F74207573696E6720616E204CEA
:1016800043442E0A003F53706563696669656420B0
:101690006E6F7A7A6C652074656D706572617475B1
:1016A0007265206E6F7420706C61757369626C6511
:1016B0002E0A003F53706563696669656420666938
:1016C0006C616D656E742073697A65206E6F74202D
:1016D000706C61757369626C652E0A003F537065AA
:1016E000636966696564207072696D65206C656EFA
:1016F000677468206E6F7420706C61757369626CBA
:10170000652E0A003F5072696D65206C656E6774C6
:1017100068206D75737420626520737065636966F7
:10172000696564207768656E206E6F7420757369D3
:101730006E6720616E204C43442E0A003F53706553
:10174000636966696564206E6F7A7A6C6520736977
:101750007A65206E6F7420706C61757369626C6558
:101760002E0A003F5370656369666965642052659F
:101770007472616374696F6E204D756C7469706CFE
:10178000696572206E6F7420706C61757369626C2C
:10179000652E0A003F52657472616374696F6E2032
:1017A0004D756C7469706C696572206D7573742009
:1017B0006265207370656369666965642E0A003F1F
:1017C000537065636966696564206C617965722030
:1017D000686569676874206E6F7420706C617573DA
:1017E00069626C652E0A003F5370656369666965BE
:1017F00064206265642074656D70657261747572D1
:1018000065206E6F7420706C61757369626C652001
:101810002834302D31343043292E0A004732362007
:10182000636F6D6D616E6420737461727465642E94
:101830002057616974696E6720666F722068656100
:101840007465722873292E0A00024A3135004A3124
:1018500032004A3137002020506C616E6E65724252
:10186000756666657242797465733A200020467227
:101870006565204D656D6F72793A2000436F6D701C
:10188000696C65643A204465632031372032303119
:10189000380A00207C20417574686F723A202864F1
:1018A0006176696472616D69726F2C20666F722057
:1018B000416E796375626963206933204D656761A4
:1018C000290A00323031382D31322D313300204C8D
:1018D00061737420557064617465643A2000312E20
:1018E000312E390A004D61726C696E0020536F66AB
:1018F00074776172652052657365740A00205761C0
:10190000746368646F672052657365740A002042CF
:10191000726F776E206F75742052657365740A005C
:101920002045787465726E616C2052657365740A27
:1019300000506F77657255700A0073746172740A93
:10194000004D3234004D3233202573006175746FC1
:1019500025692E67006572726F72207772697469EB
:101960006E6720746F2066696C650A00205A3A0021
:1019700020593A0020583A00656E6473746F707392
:10198000206869743A2000446F6E6520736176693F
:101990006E672066696C652E0A004D32390020742E
:1019A0006F6F206C6F6E6720657874727573696FE6
:1019B0006E2070726576656E7465640A0020636FD0
:1019C0006C6420657874727573696F6E20707265CF
:1019D00076656E7465640A00454550524F4D20642B
:1019E00061746173697A65206572726F722E0A0084
:1019F000290A002062797465733B206372632000BA
:101A000053657474696E67732053746F72656420D4
:101A10002800290A002062797465733B2063726391
:101A200020002073746F7265642073657474696E2E
:101A3000677320726574726965766564202800207A
:101A40002863616C63756C6174656429210A0020E8
:101A5000213D2000454550524F4D20435243206DBB
:101A600069736D61746368202D202873746F7265CB
:101A7000642920002053697A653A2000496E646524
:101A8000783A2000204D61726C696E3D56353529DB
:101A90000A0028454550524F4D3D00454550524F94
:101AA0004D2076657273696F6E206D69736D617418
:101AB000636820001000C90210012C0140012201BE
:101AC00070011801B0010E01F00104015002FA008A
:101AD000B002F0003003E600D003DC009004D20036
:101AE0007005C800A006BE000008B400B009AA0036
:101AF000D00BA000600E960060118C0000158200D3
:101B000020197800C01D6E00A0226400B0275A0082
:101B1000902C500000314600E0343C001038320078
:101B2000903A2800603C1E00A03D1400803E0A0050
:101B3000203F00002CFFFFFFFFFF0001010101011A
:101B40006265640A002C2073797374656D20737468
:101B50006F7070656421204865617465725F4944E7
:101B60003A20004265642068656174696E6720668A
:101B700061696C65640048656174696E67206661BF
:101B8000696C65640045312048656174696E672041
:101B90006661696C65640048656174696E6720669A
:101BA00061696C65640070012C0190012701B0012E
:101BB0002201C0011D01F0011801100213013002C1
:101BC0000E016002090190020401C002FF0000033F
:101BD000FA004003F5008003F000D003EB0020047E
:101BE000E6007004E100E004DC004005D700C00519
:101BF000D2004006CD00D006C8008007C3003008E0
:101C0000BE00F008B900C009B400B00AAF00B00BC4
:101C1000AA00D00CA500000EA000500F9B00C01021
:101C200096005012910000148C00C0158700B01768
:101C30008200B0197D00D01B7800001E7300402088
:101C40006E0090226900F024640040275F00902914
:101C50005A00E02B5500102E500020304B0010325F
:101C60004600E033410090353C00103737007038B3
:101C70003200A0392D00B03A2800A03B2300603C80
:101C80001E00103D1900903D1400103E0F00703EE4
:101C90000A00C03E0500003F0000403FFBFF803FC0
:101CA000F6FFC03FF1FF453120544845524D414CAD
:101CB0002052554E41574159004245442054484511
:101CC000524D414C2052554E415741590054686580
:101CD000726D616C2052756E6177617900453120BB
:101CE0004572723A204D415854454D50004572722C
:101CF0003A204D415854454D5020424544004D41F5
:101D00005854454D50207472696767657265640068
:101D10004531204572723A204D494E54454D500090
:101D20004572723A204D494E54454D50204245442B
:101D3000004D494E54454D50207472696767657275
:101D40006564004D383420582059205A2045002021
:101D50002F002042403A0020403A006F70656E200C
:101D60006661696C65642C2046696C653A200043A5
:101D7000616E6E6F74206F70656E2073756264693A
:101D80007220004A3035004A3233004739310A4761
:101D900031205A2D313020463234300A4739300054
:101DA00053442063617264206F6B0A006F70656E2C
:101DB000526F6F74206661696C65640A00766F6C9F
:101DC000756D652E696E6974206661696C65640A5B
:101DD000004572726F723A00534420696E69742034
:101DE0006661696C0A006563686F3A00205A3A00C0
:101DF00020593A0020436F756E7420583A002045F0
:101E00003A00205A3A0020593A00583A003A004322
:101E100061703A00205A00205900580020204D617E
:101E2000783A2000205A00205900580020204D699F
:101E30006E3A20004F6E20004F666600536F667446
:101E400020656E6473746F70733A20004B642000D9
:101E500023646566696E652044454641554C545F70
:101E6000004B69200023646566696E652044454621
:101E700041554C545F004B70200023646566696EC9
:101E8000652044454641554C545F0050494420412B
:101E900075746F74756E652066696E6973686564C4
:101EA000212050757420746865206C617374204B18
:101EB000702C204B6920616E64204B6420636F6E30
:101EC0007374616E74732066726F6D2062656C6FDF
:101ED0007720696E746F20436F6E666967757261F3
:101EE00074696F6E2E680A00504944204175746F02
:101EF00074756E65206661696C6564212074696D16
:101F0000656F75740A00453120544845524D414C67
:101F10002052554E415741590042454420544845AE
:101F2000524D414C2052554E41574159005468651D
:101F3000726D616C2052756E617761790045312058
:101F400048656174696E67206661696C656400420A
:101F500065642068656174696E67206661696C6597
:101F6000640048656174696E67206661696C6564C8
:101F700000504944204175746F74756E6520666128
:101F8000696C6564212054656D7065726174757249
:101F90006520746F6F20686967680A00204B643A97
:101FA0002000204B693A2000204B703A20000A2084
:101FB000436C617373696320504944200A002054C4
:101FC000753A2000204B753A2000206D61783A2048
:101FD00000206D696E3A200020643A20002062697A
:101FE00061733A2000504944204175746F74756ED6
:101FF00065206661696C65642120426164206578B2
:10200000747275646572206E756D6265720A005037
:102010004944204175746F74756E652073746172E4
:10202000740A004F66660A00466164652048656967
:102030006768742000426564204C6576656C696E43
:102040006720004661696C656420746F20656E616D
:10205000626C6520426564204C6576656C696E67CC
:102060000A004D65736820426564204C6576656C96
:1020700020646174613A0A004D65736820706F696D
:102080006E742063616E6E6F74206265207265737A
:102090006F6C7665640A004D34323120696E636F6F
:1020A000727265637420706172616D65746572200F
:1020B00075736167650A00656E7175657565696E32
:1020C000672022004B494C4C45442E200050726939
:1020D0006E7465722073746F7070656420647565CA
:1020E00020746F206572726F72732E20466978209B
:1020F000746865206572726F7220616E64207573FA
:1021000065204D39393920746F207265737461729E
:10211000742E202854656D70657261747572652027
:1021200069732072657365742E2053657420697419
:102130002061667465722072657374617274696E71
:1021400067290A004E6F20436865636B73756D20C5
:1021500077697468206C696E65206E756D62657252
:102160002C204C617374204C696E653A20004E6FD0
:1021700020436865636B73756D2077697468206CA4
:10218000696E65206E756D6265722C204C6173748A
:10219000204C696E653A2000636865636B73756DEA
:1021A000206D69736D617463682C204C61737420B9
:1021B0004C696E653A20004C696E65204E756D6203
:1021C0006572206973206E6F74204C617374204CAB
:1021D000696E65204E756D6265722B312C204C61E5
:1021E0007374204C696E653A20004D313130004DDA
:1021F00033310053442072656164206572726F72DE
:102200000A00446F6E65207072696E74696E672093
:1022100066696C650A007C3C3E5E2B3D3F2F5B5D32
:102220003B2C2A225C00627573793A2070617573C9
:10223000656420666F7220696E7075740A0062753D
:1022400073793A2070617573656420666F722075CA
:102250007365720A00627573793A2070726F6365F4
:102260007373696E670A004A3135004B494C4C451F
:10227000442E20004B494C4C2063617573656420EB
:102280006279204B494C4C20627574746F6E2F70CC
:10229000696E0A004B494C4C45442E20004B494C7A
:1022A0004C2063617573656420627920746F6F20C0
:1022B0006D75636820696E61637469766520746901
:1022C0006D65202D2063757272656E7420636F6D6D
:1022D0006D616E643A20004A3131005072696E744B
:1022E00065722068616C7465642E206B696C6C2863
:1022F000292063616C6C6564210A000000A0C000A5
:10230000000000000000005761726E696E673A209D
:10231000486F6D696E672042756D702044697669FB
:10232000736F72203C20310A000202040000A040BA
:102330000000A040000000400000614300005C433A
:1023400000004D43FFFFFF20496E76616C696420F9
:10235000657874727564657220000000A0C000008A
:1023600000000000000000005C4300005C4300002F
:102370004D43486F6D696E67206661696C656400E6
:10238000206E6F7420656E74657265642E0A004657
:10239000696C652064656C657465643A0044656CBD
:1023A0006574696F6E206661696C65642C2046698E
:1023B0006C653A200050726F7465637465642050D8
:1023C000696E0A004A3036004A3034004A3037001D
:1023D00020573A004A3038004A30390020573A0036
:1023E00000002100240027002A002D0030003300C7
:1023F00001010000040107010A010000220025007C
:1024000028002B002E0031003400020100000501DD
:1024100008010B01000020002300260029002C00E9
:102420002F0032000001000003010601090105052B
:102430000505070508080808020202020A0A08083A
:102440000404040401010101010101010303030368
:1024500003030303040707070C0C0C0C0C0C0C0CF7
:102460000202020206060606060606060B0B0B0B08
:102470000B0B0B0B0102102020080810204010202D
:102480004080020102010804020101020408102038
:102490004080804020100804020180040201804036
:1024A000201008040201080402010102040810209F
:1024B0004080010204081020408000000A0B02093D
:1024C0000C0D0E08070304010000000000000000CE
:1024D00000000000000000000000000000000000FC
:1024E00000000000000012111000000000000000B9
:1024F00000000000000000000000000000000000DC
:10250000556E6B6E6F776E20636F6D6D616E643AA2
:102510002022002066697273740A005A005900581C
:1025200000486F6D652000000048420000484200EE
:10253000008040000000005452494747455245443E
:10254000006F70656E003A20007A325F6D696E0030
:102550007A5F6D696E00795F6D696E00785F6D6995
:102560006E005265706F7274696E6720656E647379
:10257000746F70207374617475730A000A4D65611D
:10258000737572656420706F696E74733A0A005ACD
:10259000206F66667365743A20004E756D20582C66
:1025A000593A20352C350A000000000100000001D6
:1025B00000008000555555000000400033333300C3
:1025C000AAAA2A004992240000002000C7711C001A
:1025D00099991900D1451700555515003BB11300C5
:1025E0002449120011111100000010000F0F0F00FC
:1025F000E3380E0043790D00CCCC0C00C3300C0046
:10260000E8A20B0064210B00AAAA0A00703D0A0090
:102610009DD80900427B090092240900DCD3080000
:10262000888808001042080000000800F0C1070078
:102630008787070075500700711C07003EEB0600F6
:10264000A1BC06006990060066660600703E0600A2
:102650006118060017F4050074D105005BB0050091
:10266000B2900500627205005555050078390500E5
:10267000B81E0500050505004EEC040087D40400D3
:10268000A1BD040090A7040049920400C17D04008C
:10269000EE690400C7560400444404005C320400A0
:1026A0000821040041100400000004003FF0030072
:1026B000F8E0030026D20300C3C30300CCB5030037
:1026C0003AA803000A9B0300388E0300C081030070
:1026D0009F750300D0690300505E03001D53030083
:1026E00034480300913D03003333030016290300EF
:1026F000381F030097150300300C03000303030089
:102700000BFA020049F10200BAE802005CE00200A4
:102710002DD802002DD0020059C80200B0C002001E
:1027200031B90200DAB10200AAAA0200A0A3020095
:10273000BC9C0200FA9502005C8F0200DF88020058
:1027400082820200457C0200277602002770020088
:10275000436A02007C640200D05E02003F5902001E
:10276000C853020048617264636F64656420446505
:102770006661756C742053657474696E6773204C60
:102780006F616465640A00B80B0000B80B00003C80
:10279000000000102700000000FA430000FA430088
:1027A00000C040000070420000A0420000A04200B3
:1027B00000C8433333B94220286D6D290020204DD5
:1027C000393030204B004C696E656172204164766F
:1027D000616E63653A0A0020440020490020204DC4
:1027E00033303420500020440020490020204D3355
:1027F00030312050005049442073657474696E670D
:10280000733A0A00205A0020204D36363600456EB5
:102810006473746F702061646A7573746D656E742F
:102820003A0A00205A00205900202047323920530C
:1028300033205800205A0020204D343230205300DD
:102840004D65736820426564204C6576656C696EE1
:10285000673A0A00205A0020590020204D323036B5
:10286000205800486F6D65206F66667365743A0A7C
:1028700000204500205A0020590020580020540014
:1028800020530020204D32303520510020453C6D32
:1028900061785F655F6A65726B3E0020583C6D61D0
:1028A000785F785F6A65726B3E20593C6D61785F36
:1028B000795F6A65726B3E205A3C6D61785F7A5F22
:1028C0006A65726B3E00416476616E6365643A20AE
:1028D000513C6D696E5F7365676D656E745F746999
:1028E0006D655F75733E20533C6D696E5F6665650F
:1028F00064726174653E20543C6D696E5F747261F0
:1029000076656C5F66656564726174653E0020542F
:102910000020520020204D323034205000416363AB
:10292000656C65726174696F6E2028756E69747369
:102930002F7332293A20503C7072696E745F616364
:1029400063656C3E20523C726574726163745F61B2
:102950006363656C3E20543C74726176656C5F61A4
:102960006363656C3E0A00204500205A0020590030
:1029700020204D3230312058004D6178696D756DE1
:1029800020416363656C65726174696F6E202875A0
:102990006E6974732F7332293A0A00204500205A59
:1029A0000020590020204D3230332058004D6178EE
:1029B000696D756D20666565647261746573202844
:1029C000756E6974732F73293A0A00204500205AE6
:1029D0000020590020204D39322058005374657072
:1029E000732070657220756E69743A0A0020204D5C
:1029F0003230302044300A0020204D323030204424
:102A0000002044697361626C65640A0046696C6108
:102A10006D656E742073657474696E67733A002017
:102A200020473231202020203B00FFFDFCFAF8F641
:102A3000F4F2F0EEECEAE9E7E5E3E1E0DEDCDAD936
:102A4000D7D5D4D2D0CFCDCBCAC8C7C5C3C2C0BFDB
:102A5000BDBCBAB9B7B6B4B3B2B0AFADACAAA9A851
:102A6000A6A5A4A2A1A09E9D9C9A9998979594939F
:102A700092908F8E8D8B8A898887868483828180CD
:102A80007F7E7D7B7A797877767574737271706FDB
:102A90006E6D6C6B6A696867666564636261605FCE
:102AA0005E5D5C5B5A5958585756555453525150B5
:102AB000504F4E4D4C4B4A4A494847464645444381
:102AC000424241403F3E3E3D3C3B3B3A393838373D
:102AD000363535343332323130302F2E2E2D2C2BEB
:102AE0002B2A29292827272625252423232221218B
:102AF00020201F1E1E1D1C1C1B1B1A19191818171D
:102B00001616151514131312121111100F0F0E0EA5
:102B10000D0D0C0C0B0A0A09090808070706060523
:102B200005040403030202010000526573656E642C
:102B30003A20006F6B0020746F6F206C6F6E6720FF
:102B4000657874727573696F6E2070726576656EE4
:102B50007465640A0020636F6C6420657874727514
:102B600073696F6E2070726576656E7465640A00B5
:102B70004572726F722077726974696E6720746F24
:102B800020454550524F4D210A0057726974696EB5
:102B90006720746F2066696C653A20006F70656EFF
:102BA000206661696C65642C2046696C653A20007A
:102BB0006F70656E206661696C65642C2046696C77
:102BC000653A200046696C652073656C65637465C1
:102BD000640A002053697A653A200046696C6520D2
:102BE0006F70656E65643A20002066696C653A20F6
:102BF00000646F696E67006672657368004E6F7778
:102C00002000454E4420535542524F5554494E459D
:102C10000A002220706F73002220706172656E744A
:102C20003A2200535542524F5554494E4520434194
:102C30004C4C207461726765743A22004B494C4CCD
:102C400045442E2000747279696E6720746F20638A
:102C5000616C6C207375622D67636F6465206669B3
:102C60006C6573207769746820746F6F206D616E76
:102C700079206C6576656C732E204D4158206C650B
:102C800076656C2069733A00B4DF6AE111241FBED7
:102C9000CFEFD1E2DEBFCDBF00E00CBF14E0A0E07B
:102CA000B2E0EEE8FCED01E00BBF02C007900D9230
:102CB000A431B107D9F728E1A4E1B4E001C01D9225
:102CC000A83CB207E1F716E1C5E4D6E100E006C092
:102CD00021970109802FFE010E949FEDC434D10786
:102CE00080E00807A9F70E9414DA0C9436EE0C94E1
:102CF00000002F923F924F925F926F927F928F923D
:102D00009F92AF92BF92CF92DF92EF92FF920F937A
:102D10001F93CF93DF93CDB7DEB7CA58D1090FB653
:102D2000F894DEBF0FBECDBF21E020933F1080910D
:102D300015188D3411F40C947721843511F40C940A
:102D40009F2E873411F00C94EB2E809113189091E4
:102D500014188A31910509F4BEC79CF4843091059A
:102D60003CF482309105B4F597FF2DC00C9473218B
:102D70008430910509F4D2C1059709F40EC20C9470
:102D800073218A32910511F40C946A204CF48C3131
:102D9000910509F4A4C74D9709F4A6C70C947321B3
:102DA0008B35910511F40C94F5208C35910511F4B7
:102DB0000C94F9208A35910511F00C94732110922E
:102DC00027040C94ED2E8091270281110C94F22E91
:102DD0000C94ED2E20912702222311F40C94ED2E59
:102DE00011E0029709F010E00E94C9AA19821A8224
:102DF0001B821C821D821E821F82188682E50E9411
:102E00008B4C882309F43AC10E940B4C4B015C01A6
:102E100020E030E0A9010E9457E6882309F444C16C
:102E2000C0903204D0903304E0903404F090350424
:102E3000CCAADDAAEEAAFFAAC0903604D09037042F
:102E4000E0903804F0903904C8AED9AEEAAEFBAEDB
:102E5000C090AE10D090AF10E090B010F090B110D4
:102E6000CCAEDDAEEEAEFFAEC090B210D090B310DF
:102E7000E090B410F090B5102496CCAEDDAEEEAE7E
:102E8000FFAE24972CAD3DAD4EAD5FAD6CA97DA9D5
:102E90008EA99FA90E9457E681110BC0A701960138
:102EA00068AD79AD8AAD9BAD0E9457E6882309F4E1
:102EB000FBC020E030E0A901C501B4010E9457E643
:102EC000881F8827881F181739F0C12CD12C80E85B
:102ED000E82E8FEBF82E06C0C12CD12C00E8E02E96
:102EE0000FE3F02E2C96CCAEDDAEEEAEFFAE2C97FF
:102EF0002CA93DA94EA95FA96CAD7DAD8EAD9FAD4E
:102F00000E94A2EA28966CAF7DAF8EAF9FAF289744
:102F100028AD39AD4AAD5BAD24966CAD7DAD8EADBF
:102F20009FAD24970E94A2EA6B017C0128962CADEC
:102F30003DAD4EAD5FAD2897CA01B9010E94BCE618
:102F40002B013C01A7019601C701B6010E94BCE616
:102F50009B01AC01C301B2010E94A3EA0E940EEDE5
:102F60002B013C0120E030E040E05FE30E94BCE642
:102F700060966CAF7DAF8EAF9FAF6097A501940157
:102F8000C501B4010E94BCE64B015C0160962CAD0A
:102F90003DAD4EAD5FAD6097CA01B9010E94BCE680
:102FA0009B01AC01C501B4010E94A2EA0E940EED92
:102FB0002C962CAD3DAD4EAD5FAD2C970E94BCE67E
:102FC0004B015C01C701B6019058A30192010E9418
:102FD0007FEBA50194010E94BCE66B017C012CAD46
:102FE0003DAD4EAD5FAD6CA97DA98EA99FA90E9494
:102FF000A3EA20E030E040E05FE30E94BCE69B01F2
:10300000AC01C701B6010E94A3EA2CA93DA94EA9B3
:103010005FA90E94A2EA69837A838B839C832496AA
:103020002CAD3DAD4EAD5FAD249768AD79AD8AADA9
:103030009BAD0E94A3EA20E030E040E05FE30E9405
:10304000BCE66B017C01A301920128966CAD7DADBD
:103050008EAD9FAD28970E947FEBA50194010E9441
:10306000BCE69B01AC01C701B6010E94A3EA28ADF2
:1030700039AD4AAD5BAD0E94A2EA12C089E40E945C
:103080008B4C882331F00E940B4C69837A838B83AD
:103090009C838AE40E948B4C882331F00E940B4C65
:1030A0006D837E838F83988720E030E0A90169815A
:1030B0007A818B819C810E9457E681110EC020E0AD
:1030C00030E0A9016D817E818F8198850E9457E64D
:1030D000811103C0E1EDFDE10DC0412FBE016F5F25
:1030E0007F4F8EEA90E10E94EBA40C94ED2E0E949B
:1030F000E193F80184918F010F5F1F4F8111F7CF8A
:10310000EDE1F2E084918F010F5F1F4F882311F4EE
:103110000C94ED2E0E94E193F801F4CF80E50E941B
:103120008B4C882379F080912104909122040097A0
:1031300049F04AE050E060E070E00E94D6E46B01A4
:103140007C0103C0C12CD12C760183E50E948B4CFD
:10315000882361F00E940B4C20E030E04AE754E401
:103160000E94BCE60E94ECEB6B017C010E94126A9B
:103170000E94F258C60ED71EE81EF91E0E94F25891
:10318000DC01CB018C199D09AE09BF09B7FD02C056
:103190000C94ED2E0E941FA1F1CF8091270288236D
:1031A00011F40C94ED2E0E94C9AA89E40E948B4C64
:1031B000882329F00E940B4C2B013C0103C0412CB9
:1031C000512C32018AE40E948B4C882329F00E9402
:1031D0000B4C4B015C0103C0812C912C540180E508
:1031E0000E948B4C882329F00E940B4C6B017C01C0
:1031F00003C0C12CD12C760181E50E948B4C882321
:1032000039F00E940B4C6CAB7DAB8EAB9FAB04C016
:103210001CAA1DAA1EAA1FAA20913E10C657DF4F46
:103220002883CA58D0406091020270910302072E91
:10323000000C880B990B0E945DE6209130023091C2
:10324000310240913202509133020E94BCE62AE0E2
:1032500037ED43E25CE30E94BCE668AB79AB8AAB36
:103260009BAB4091320450913304609134047091CF
:10327000350448AF59AF6AAF7BAF9A01AB01C301C8
:10328000B2010E94A3EAA1966CAF7DAF8EAF9FAF53
:10329000A1974090360450903704609038047090A5
:1032A0003904A3019201C501B4010E94A3EAA596C5
:1032B0006CAF7DAF8EAF9FAFA5972091AE103091D0
:1032C000AF104091B0105091B110C701B6010E94EB
:1032D000A3EAA9966CAF7DAF8EAF9FAFA99720915F
:1032E000B2103091B3104091B4105091B5106CA948
:1032F0007DA98EA99FA90E94A3EAAD966CAF7DAF70
:103300008EAF9FAFAD97C8ACD9ACEAACFBACC9826D
:10331000DA82EB82FC824D825E826F8278860E9426
:10332000F2589B01AC0128533F4F4F4F5F4FCB5793
:10333000DF4F288339834A835B83C558D040BDEC77
:103340008B2EBCEC9B2EA92CBDE3BB2E25961FAE6D
:10335000259729961FAE29972D961FAE2D9761961A
:103360001FAE61970E94C37B0E94F2588B019C01A3
:10337000CB57DF4FC880D980EA80FB80C558D0404A
:103380000C191D092E093F0937FD10C09B01AC0126
:1033900028533F4F4F4F5F4FCB57DF4F2883398321
:1033A0004A835B83C558D0400E941FA125967FADFC
:1033B000259729966FAD29972D969FAD2D976196EC
:1033C0008FAD6197272F362F492F582FC501B40194
:1033D0000E94A3EA6CAB78AF8CAF21969FAF219788
:1033E00020E030E040E85FE30E94C9EC181644F4A6
:1033F0001CAA18AE30E83CAF4FE321964FAF21979F
:103400006091AE107091AF108091B0109091B1109A
:10341000E1966CAF7DAF8EAF9FAFE19780913204A4
:1034200090913304A0913404B0913504E5968CAFAB
:103430009DAFAEAFBFAFE59721969FAD21979F930C
:10344000ACADAF93B8ADBF93ECA9EF93E196ACAC44
:10345000BDACCEACDFACE197A996ECACFDAC0EAD4B
:103460001FADA997A1962CAD3DAD4EAD5FADA19717
:10347000E5966CAD7DAD8EAD9FADE5970E94A2C582
:103480000F900F900F900F9062966FAF62976396B8
:103490007FAF639764968FAF649765969FAF65978C
:1034A000C090B210D090B310E090B410F090B5106E
:1034B000E996CCAEDDAEEEAEFFAEE99720913604D4
:1034C000309137044091380450913904ED962CAF77
:1034D0003DAF4EAF5FAFED9721963FAD21973F9344
:1034E0004CAD4F9358AD5F936CA96F93E996ACAC1C
:1034F000BDACCEACDFACE997AD96ECACFDAC0EAD9F
:103500001FADAD97A5962CAD3DAD4EAD5FADA5976A
:10351000ED966CAD7DAD8EAD9FADED970E94A2C5D1
:103520000F900F900F900F9066966FAF669767960B
:103530007FAF679768968FAF689769969FAF6997D7
:1035400089819A81AB81BC81C358DF4F888399837D
:10355000AA83BB83CD57D040CD80DE80EF80F88436
:10356000CF57DF4FC882D982EA82FB82C158D04050
:103570006A961FAE6A9725967FAD259729966FADFF
:1035800029972D969FAD2D9761968FAD6197272F27
:10359000362F492F582FBCA9A8ADFCAD2196EFAD11
:1035A00021976B2F7A2F8F2F9E2F0E94A2EA2FE652
:1035B00032E143E05BE30E9457E687FD29C125968F
:1035C0007FAD259729966FAD29972D969FAD2D97A5
:1035D00061968FAD6197272F362F492F582FBCA9A1
:1035E000A8ADFCAD2196EFAD21976B2F7A2F8F2FD1
:1035F0009E2F0E94A3EA20E030E040E05FE30E94BB
:10360000BCE6662E972E882E792E9F938F937F93FC
:103610006F93E196ACACBDACCEACDFACE197A996B4
:10362000ECACFDAC0EAD1FADA997A1962CAD3DAD98
:103630004EAD5FADA197E5966CAD7DAD8EAD9FAD06
:10364000E5970E94A2C50F900F900F900F906B9678
:103650006FAF6B976C967FAF6C976D968FAF6D97D2
:10366000C757DF4F9883C958D0407F928F929F925F
:103670006F92E996ACACBDACCEACDFACE997AD9641
:10368000ECACFDAC0EAD1FADAD97A5962CAD3DAD30
:103690004EAD5FADA597ED966CAD7DAD8EAD9FAD9A
:1036A000ED970E94A2C50F900F900F900F90162FCC
:1036B000072FB82EA92E66962FAD669767963FAD59
:1036C000679768964FAD689769965FAD6997CF57D2
:1036D000DF4F688179818A819B81C158D0400E94E7
:1036E000A3EA20E030E040E05FE30E94BCE61B017B
:1036F0002C0162962FAD629763963FAD63976496F7
:103700004FAD649765965FAD6597C358DF4F68818D
:1037100079818A819B81CD57D0400E94A3EA20E025
:1037200030E040E05FE30E94BCE69B01AC016B9699
:103730006FAD6B976C967FAD6C976D968FAD6D97F7
:10374000C757DF4F9881C958D0400E94A2EA6B0149
:103750007C0120E030E0A9010E94C9EC87FF04C091
:10376000F7FAF094F7F8F094A2019101612F702F0D
:103770008B2D9A2D0E94A2EA1B012C0120E030E043
:10378000A9010E94C9EC87FF04C057FA509457F86A
:103790005094A2019101C701B6010E94A3EA2DEC49
:1037A0003CEC4CEC5DE30E9457E618168CF56696EF
:1037B0001FAF669767960FAF67976896BFAE68971B
:1037C0006996AFAE69976B96DFAC6B976296DFAE8A
:1037D00062976C96EFAC6C976396EFAE63976D96BD
:1037E000FFAC6D976496FFAE6497C757DF4F288193
:1037F000C958D04065962FAF65976CAA98AE8CAE2D
:1038000021967FAE219731E06A963FAF6A97B3CE9B
:103810006A964FAD6A97411144C125967FAD2597B1
:1038200029966FAD29972D969FAD2D9761968FADF7
:103830006197272F362F492F582FBCA9A8ADFCAD73
:103840002196EFAD21976B2F7A2F8F2F9E2F0E94FD
:10385000A2EA6B017C012DEC3CEC4CEC5DE30E9498
:10386000C9EC18160CF41DC1A7019601C701B601D9
:103870000E94A3EA2596EFAD25972996BFAD29971B
:103880002D96AFAD2D976196FFAD61972E2F3B2FF3
:103890004A2F5F2F0E94A3EA662E972E882E792E3C
:1038A00020E030E040E85FE30E94C9EC87FFF9C008
:1038B0007F928F929F926F92E196ACACBDACCEACF2
:1038C000DFACE197A996ECACFDAC0EAD1FADA997AE
:1038D000A1962CAD3DAD4EAD5FADA197E5966CAD1B
:1038E0007DAD8EAD9FADE5970E94A2C50F900F9064
:1038F0000F900F906A966FAF6A976B967FAF6B973A
:103900006C968FAF6C976D969FAF6D977F928F92ED
:103910009F926F92E996ACACBDACCEACDFACE997B0
:10392000AD96ECACFDAC0EAD1FADAD97A5962CAD34
:103930003DAD4EAD5FADA597ED966CAD7DAD8EAD59
:103940009FADED970E94A2C50F900F900F900F9022
:10395000162F072FB82EA92E262F372F482F592F75
:10396000CF57DF4F688179818A819B81C158D040D0
:103970000E94A3EA20E030E040E05FE30E94BCE662
:103980006B017C016A962FAD6A976B963FAD6B9782
:103990006C964FAD6C976D965FAD6D97C358DF4FCA
:1039A000688179818A819B81CD57D0400E94A3EAAA
:1039B00020E030E040E05FE30E94BCE69B01AC0108
:1039C00062966FAD629763967FAD639764968FAD95
:1039D000649765969FAD65970E94A2EA1B012C0132
:1039E00020E030E0A9010E94C9EC87FF04C057FA2B
:1039F000509457F85094A701960166966FAD66975C
:103A000067967FAD679768968FAD689769969FAD0B
:103A100069970E94A2EA6B017C0120E030E0A901D5
:103A20000E94C9EC87FF04C0F7FAF094F7F8F0940D
:103A3000A2019101C701B6010E94A3EA2DEC3CEC62
:103A40004CEC5DE30E94C9EC18165CF166961FAF62
:103A5000669767960FAF67976896BFAE6897699647
:103A6000AFAE69976A965FAD6A9762965FAF6297ED
:103A70006B966FAD6B9763966FAF63976C967FADE8
:103A80006C9764967FAF64976D968FAD6D976596D2
:103A90008FAF65976CAA98AE8CAE21967FAE2197BA
:103AA000BCCE25967FAD259729966FAD29972D968B
:103AB0009FAD2D9761968FAD6197272F362F492F98
:103AC000582FBCA9A8ADFCAD2196EFAD21976B2F67
:103AD0007A2F8F2F9E2F0E94A2EA4B015C016296E3
:103AE0008FAD629763969FAD63976496AFAD649711
:103AF0006596BFAD659789839A83AB83BC836696D1
:103B00008FAD669767969FAD67976896AFAD6897DC
:103B10006996BFAD69978D839E83AF83B8877CA973
:103B200068AD9CAD21968FAD2197272F362F492F59
:103B3000582F60E070E080E89FE30E94A2EA6B01EA
:103B40007C0120913A0430913B0440913C04509117
:103B50003D040E94BCE62B013C012091B61030913F
:103B6000B7104091B8105091B910BCA9A8ADFCADE8
:103B70002196EFAD21976B2F7A2F8F2F9E2F0E94CA
:103B8000BCE69B01AC01C301B2010E94A3EA6987B4
:103B90007A878B879C8720913E0430913F04409127
:103BA000400450914104C701B6010E94BCE66B017C
:103BB0007C012091BA103091BB104091BC10509103
:103BC000BD10BCA9A8ADFCAD2196EFAD21976B2F20
:103BD0007A2F8F2F9E2F0E94BCE69B01AC01C7015C
:103BE000B6010E94A3EA6D877E878F87988BCE01EE
:103BF00001960E94DFC91CA61DA61EA61FA68981CC
:103C00009A81AB81BC8188A399A3AAA3BBA38D8110
:103C10009E81AF81B8858CA39DA3AEA3BFA38985E8
:103C20009A85AB85BC8588A799A7AAA7BBA7AE0133
:103C3000485D5F4FBE016C5D7F4FCE0180960E9454
:103C4000E5BCDE019C966D01C657DF4FE880CA587F
:103C5000D0408E01005D1F4F9E01235F3F4FAE019C
:103C6000485D5F4FBE016C5D7F4FCE0180960E9424
:103C7000EE59882329F120E030E040E85FE3BCA959
:103C8000A8ADFCAD2196EFAD21976B2F7A2F8F2F2A
:103C90009E2F0E9457E687FF13C03CA925963FAF91
:103CA000259748AD29964FAF29975CAD2D965FAF0C
:103CB0002D9721966FAD219761966FAF619752CB8B
:103CC00080E1EEEAF0E1A2E3B4E001900D928A9582
:103CD000E1F70C94ED2E0E94284E0C94ED2E80E01E
:103CE0000E9469AC0C94ED2E83E50E948B4C8823D6
:103CF00021F10E94EB4B182F863070F0E5EEF2E0D8
:103D000084918F010F5F1F4F882311F40C94ED2EC7
:103D10000E94E193F801F4CF833009F44AC130F4F2
:103D2000813091F1823009F43FC008C0843009F439
:103D30009FC1853009F4ACC101C010E00E941CACE9
:103D4000811103C0E5ECF2E013C080917C10882360
:103D500019F063E173E002C067E173E08DEB92E07C
:103D60000E9487C58AE00E94E1930E941FBD96C110
:103D700084917F01BFEFEB1AFB0A882309F48EC1FF
:103D80000E94E193F701F4CF0E94D2BD109201028C
:103D90001092000282EB92E09093A4078093A30715
:103DA0000E940D940C94ED2E8091000290910102DE
:103DB00097FF0EC0E9E8F2E084918F010F5F1F4F7B
:103DC000882311F40C94ED2E0E94E193F801F4CFB6
:103DD0000097A1F4809152028093280419821A82DC
:103DE0001B821C8218A219A21AA21BA2BE016F5F1D
:103DF0007F4FCE0180960E9468B427C0815065E055
:103E00000E946BED80FF03C024E0291B922F25E068
:103E10009202F0011124E80FF11D87FDFA95EE0FD3
:103E2000FF1FEE0FFF1FEA53FF4E80913A0490915F
:103E30003B04A0913C04B0913D0480839183A28314
:103E4000B383809128048093520280910002909164
:103E50000102893191050CF067C0109252029C0159
:103E60002F5F3F4F309301022093000265E00E94D4
:103E70006BED80FF03C024E0291B922F40913A0490
:103E800050913B0460913C0470913D0448A359A3B8
:103E90006AA37BA319821A821B821C8244E08402DB
:103EA00090011124B9016751764F4B01DB012D912F
:103EB0003D914D915C91B4E09B02C0011124FC0145
:103EC000E350F64F5F016081718182819381DE0151
:103ED00011966D01E12CF12C00EA10E40E949BB3D5
:103EE00019821A821B821C82B601CE0180960E9422
:103EF00068B4F50180819181A281B38180933204FD
:103F000090933304A0933404B0933504F40180817A
:103F10009181A281B3818093360490933704A0935A
:103F20003804B0933904BCC080E090E0A0EAB0E46B
:103F300080933A0490933B04A0933C04B0933D04D7
:103F40000E945CAD0E94126A8FEF9FEF9093010276
:103F500080930002E5E7F2E084918F010F5F1F4F2D
:103F6000882321F00E94E193F801F6CF83E992E0E3
:103F70009A83898304E610E019A308A3BE016F5F4A
:103F80007F4FCE0180960E9483B58AEB92E09A83A0
:103F9000898319A308A3BE016F5F7F4FCE0180966E
:103FA0000E9483B581E00E9469AC81E00E9449AC27
:103FB00077C088E50E948B4C8823A1F00E94DB4BE0
:103FC0001FEF160F1530A8F0EEE5F2E084918F0197
:103FD0000F5F1F4F882311F40C94ED2E0E94E19384
:103FE000F801F4CF88E50E94E1930E94A6E10C94C9
:103FF000ED2E89E50E948B4C8823A1F00E94DB4BBB
:104000000FEF060F0530A8F0E7E4F2E084918F018E
:104010000F5F1F4F882311F40C94ED2E0E94E19343
:10402000F801F4CF89E50E94E1930E94A6E10C9487
:10403000ED2E8AE50E948B4C882399F00E940B4C50
:1040400025E0129FF0011124E00FF11DEE0FFF1F7C
:10405000EE0FFF1FEA53FF4E6083718382839383C9
:1040600035C08AE50E94E1930E94A6E10C94ED2EF2
:104070008AE50E948B4C8823A1F30E940B4C60932D
:10408000C2107093C3108093C4109093C5101EC0CB
:1040900080E00E9449AC0E94D2BD18C01230B1F439
:1040A00060910002709101026931710514F069E1BB
:1040B00070E088E392E00E946EC569E170E083E3FE
:1040C00092E00E946EC58AE00E94E1930E94358DC5
:1040D0000C94ED2E80912702882311F40C94ED2E80
:1040E00089E40E948B4CE82E882321F00E94DB4B50
:1040F000062F01C000E08AE40E948B4CF82E882332
:1041000021F00E94DB4B162F01C010E0EE2011F0D1
:10411000053020F4FF2081F0153070F0ECEFF2E074
:1041200084918F010F5F1F4F882311F40C94ED2EA3
:104130000E94E193F801F4CF0E94974CEE2091F099
:1041400034E00302F0011124E350F64F80819181A5
:10415000A281B3818093AE109093AF10A093B01062
:10416000B093B110FF2091F044E01402F00111244B
:10417000E751F64F80819181A281B3818093B21083
:104180009093B310A093B410B093B51080E50E9443
:104190008B4C882319F00E94FC4B03C080E50E94E1
:1041A000424C86E40E948B4C8823D9F00E940B4C31
:1041B0006B017C0120E030E0A9010E94C9EC1816D7
:1041C00084F420E030E040E752E4C701B6010E94E9
:1041D0007FEB6093300270933102809332029093B0
:1041E00033020E9476CA0C94ED2E209327040C947F
:1041F000ED2E97E5292E92E0392E2DE4E22E20E1D6
:10420000F22E62E374E07DAB6CAB34E1C32E34E09C
:10421000D32E00E010E0D1018D911D010E948B4C46
:10422000882309F44BC00E940B4C2B013C01133036
:1042300049F0F60120813181428153810E94A2EA36
:104240002B013C01ACA9BDA92D913D914D915C91F3
:10425000C301B2010E94A2EA4B015C012DEB37E3DE
:1042600046E855EB0E94C9EC87FD0AC02DEB37E309
:1042700046E855E3C501B4010E9457E61816F4F468
:10428000133051F440923E0450923F046092400437
:104290007092410401E012C0A5019401F701608110
:1042A0007181828193810E94A3EAD7016D937D93EE
:1042B0008D939C931397812F0E94B3AD1F5FB4E041
:1042C000EB0EF11CECA9FDA93496FDABECABF4E0D0
:1042D000CF0ED11C143009F09ECF002309F4F6CE86
:1042E0000E9437B3F3CE0E94B7B50C94ED2E8091A7
:1042F0001318909114188537910511F40C94ED2E34
:104300000CF0C0C08C34910509F43CC40CF058C0CA
:104310008A31910509F42EC224F58531910509F4FD
:10432000E7C184F48231910509F4A9C5843191056E
:1043300009F49EC1419711F00C949C2E0E94E0A4B8
:104340000C94ED2E8731910509F4DCC10CF4D4C135
:104350008831910509F4ECC1499709F4F4C10C9432
:104360009C2E8F31910509F401C39CF48C31910589
:1043700009F4A6C20CF40CC28D31910511F40C9411
:10438000ED2E4E9711F00C949C2E0E9432B00C949E
:10439000ED2E8A32910509F49CC32CF4809709F420
:1043A00099C20C949C2E8133910509F4C6C38B34B9
:1043B000910511F00C949C2E0E94B7780C94ED2E70
:1043C0008A36910509F40AC5B4F58435910509F4D6
:1043D00056C5E4F48135910509F42CC54CF48D34AF
:1043E000910511F00C949C2E0E94EE780C94ED2E09
:1043F0008235910509F440C58335910511F00C947F
:104400009C2E81E0809326040C94ED2E8C35910532
:1044100009F47BC534F48535910509F45DC50C9428
:104420009C2E8836910509F4B1C38936910509F4AB
:1044300075C40C949C2E8F36910509F4E3C384F463
:104440008C36910509F431C40CF4E4C48D36910521
:1044500009F4A6C48E36910509F4C1C30C949C2EB0
:104460008137910509F42DC40CF423C482379105DA
:1044700009F4D3C58337910511F00C949C2EE3EE1B
:10448000F4E008C68E3221E0920711F40C94D82C87
:104490000CF071C08B3C910509F416C7CCF58C3833
:1044A000910509F481C4ACF48737910509F49AC6E3
:1044B0000CF44BC68837910509F497C689379105E6
:1044C00011F00C949C2E10923705109236050C9426
:1044D000ED2E8E3B910509F47DC434F48B399105A2
:1044E00009F437C40C949C2E883C910509F483C6CA
:1044F000893C910511F00C949C2EF7E5EF2EF2E02B
:10450000FF2E0FE411E1AFE5CA2EA1E1DA2EC3C6FA
:104510008C3D910511F40C946B2B9CF48D3C910512
:1045200009F463C70CF4ECC68E3C910509F4EAC7A4
:10453000833D910511F00C949C2E0E942A8C0C94C2
:10454000ED2E823E910511F40C94E62B3CF48D3D4A
:10455000910511F40C94782B0C949C2E8C3241E034
:10456000940711F40C940F2C8D32914011F40C949B
:10457000382C0C949C2E853F61E0960711F40C9426
:10458000C52DDCF58A39A1E09A0709F496C3BCF47D
:104590008033E1E09E0711F40C942F2D14F40C9459
:1045A0002C2D833621E0920709F45EC080399140BA
:1045B00011F00C949C2E0E94126A0C94ED2E853AF8
:1045C00041E0940711F40C94C22D4CF4843A9140CC
:1045D00011F00C949C2E0E94FB8D0C94ED2E8C3AC5
:1045E00071E0970709F4B1C7843F914011F00C9432
:1045F0009C2E0E9459700C94ED2E8A39B2E09B07D4
:1046000011F40C94042EB4F4873FF1E09F0711F4E9
:104610000C94CB2D14F40C94C82D883F31E09307F3
:1046200011F40C94D72D8C30924011F40C94FB2D86
:104630000C949C2E8B3853E0950711F40C94ED2EBE
:104640003CF48438934011F40C94312E0C949C2E3D
:10465000803AA3E09A0709F47CC1873E934011F4A5
:104660000C94892E0C949C2EE1EDFDE10C94AF2D61
:10467000EAE2F3E084918F010F5F1F4F882321F05E
:104680000E94E193F801F6CF1092AF0C82E69AE017
:104690000E94599A8BE1E2E6FAE0DE01159601905C
:1046A0000D928A95E1F78091600A9091610A9C834E
:1046B0008B838DEE92E09A83898340E050E0BE01C7
:1046C0006F5F7F4F80E090E00E94E082CE01019614
:1046D0000E94B5A0EBE1F3E084918F010F5F1F4FC3
:1046E000882311F40C94ED2E0E94E193F801F4CF8D
:1046F0000E94AF800C94ED2E1092310A1092320A73
:104700000C94ED2EE0911118F091121880818823FD
:1047100029F0803209F410823196F8CF40E061E050
:1047200080911118909112180E94A5D50C94ED2E2D
:104730008091320A882319F081E08093310A0E9427
:10474000B7780C94ED2E1092310A80912B078130AE
:1047500011F00C94ED2E82E080932B070E94F2580A
:1047600060932707709328078093290790932A075F
:104770000C94ED2E8091320A882311F40C94ED2EC6
:1047800083E50E948B4C81110C94F72E0C94ED2E36
:1047900083E40E94424C882309F450C0E8E6F3E029
:1047A00084918F010F5F1F4F882321F00E94E193B6
:1047B000F801F6CF8091FD0B811103C0EBE3F3E02C
:1047C00012C0BE016F5F7F4F8AEF9BE00E9421996C
:1047D0008E010F5F1F4FF80181918F01882349F1EE
:1047E0000E94E193F8CF84918F010F5F1F4F8823C0
:1047F00001F10E94E193F801F6CF06EDC02E03E02F
:10480000D02EE12CF12C20E08091100790E00E2CAE
:1048100002C0959587950A94E2F780FD23C2BFEF09
:10482000EB1AFB0AE2E0CE0ED11CF5E0EF16F10424
:1048300059F78AE00E94E1930C94ED2E8091320AA0
:10484000882339F08091310A882319F0E5E4F3E0F8
:1048500003C0E7E5F3E028C084918F010F5F1F4F8D
:10486000882321F00E94E193F801F6CF6091AB0C10
:104870007091AC0C8091AD0C9091AE0C4AE00E940E
:1048800002978FE20E94E1936091A70C7091A80CAF
:104890008091A90C9091AA0C4AE00E9402978AE0AC
:1048A0000E94E1930C94ED2E84918F010F5F1F4FB6
:1048B000882311F40C94ED2E0E94E193F801F4CFBB
:1048C00040E060E080911118909112180E94A5D5E7
:1048D0000C94ED2E8091310A81110E94126A809110
:1048E000320A882311F40C94ED2E80E50E948B4C43
:1048F000882319F00E94FC4B03C080E50E94424CC3
:10490000182F482F61E080911118909112180E9481
:10491000A5D583E50E948B4C882381F00E94DB4B58
:10492000AB01BC014093AB0C5093AC0C6093AD0C4D
:104930007093AE0C8AEF9BE00E9412988091320A2D
:10494000882319F081E08093310A11110C94ED2E27
:10495000F6CE809111189091121821E02093300A20
:1049600040E060E00E94A5D50C94ED2E0E9468788E
:104970007B018C0120E831E541E050E00E9445EAEE
:10498000C9016DE671E00E9478ED4B015C01C80140
:10499000B70120E13EE040E050E00E9445EACA0154
:1049A000B90128E130E040E050E00E9445EA762E6F
:1049B000672EC62ED72E8CE3282E312C412C512C5D
:1049C000C801B701A20191010E9445EAF62EE72E27
:1049D000CA01B901A20191010E9445EACB018E01F1
:1049E0000F5F1F4F81149104D1F0EF92FF927F93DC
:1049F0006F936F927F92BF92AF929F928F928FE947
:104A000093E09F938F931F930F930E9429E60FB615
:104A1000F894DEBF0FBECDBFE6EEFDE145C0A114A8
:104A2000B10489F0EF92FF927F936F936F927F9220
:104A3000BF92AF928FE893E09F938F931F930F9352
:104A40000E9429E6E4CFCD2879F0EF92FF927F9380
:104A50006F936F927F9283E893E09F938F931F935E
:104A60000F930E9429E6D3CF892B69F0EF92FF9232
:104A70007F936F938BE793E09F938F931F930F9395
:104A80000E9429E6C4CFEF92FF9287E793E09F93BD
:104A90008F931F930F930E9429E60F900F900F9012
:104AA0000F900F900F90B8CF84917F019FEFE91A7C
:104AB000F90A882321F00E94E193F701F5CFB801AC
:104AC00083EB93E00E9487C58AE00E94E1930C94F7
:104AD000ED2E83E50E948B4C882311F40C94ED2E6F
:104AE0000E94EB4BE82E80E50E948B4C882339F026
:104AF0000E94EB4B182F87FF03C00C94ED2E1DE096
:104B000089E40E948B4C882341F00E94FC4B811168
:104B10000C94732FEBE1F6E00BC089E40E94424C49
:104B2000F6CF3196A6E0EB34FA0711F40C94732F0C
:104B300084911813F6CF0C94482FF090200481E054
:104B4000F826F0922004EBECF3E084918F010F5FE4
:104B50001F4F882321F00E94E193F801F6CFFF2038
:104B600019F0E0ECF3E002C0E5ECF3E084918F0192
:104B70000F5F1F4F882311F40C94ED2E0E94E193D8
:104B8000F801F4CF0E94D9780C94ED2E88E690E0DD
:104B90000E94F3AD81110C94ED2E8091100783FFDC
:104BA00002C00C94ED2E83E50E948B4C882399F073
:104BB0000E940B4C0E94E7EBCB010E94E7590E9438
:104BC0000B4C20E030E044EB52E40E9457E618160C
:104BD00014F00E94EE780E94B1C70C94ED2E8EE482
:104BE0000E948B4C882311F40C94ED2E0E94DB4B19
:104BF0006093BE187093BF188093C0189093C1182B
:104C00000C94ED2E83E50E94424C882359F083E5F5
:104C10000E948B4C882319F00E94EB4B01C080E06E
:104C200080931007E6EEFDE184918F010F5F1F4F27
:104C3000811103C0E4EEF3E004C00E94E193F801A7
:104C4000F3CF84918F010F5F1F4F882321F00E94C3
:104C5000E193F801F6CF809110078111CECDE0EEFF
:104C6000F3E018C0BB24B394B20E222319F08CE2F7
:104C70000E94E193F60185919491FC0184918F014A
:104C80000F5F1F4F882321F00E94E193F801F6CFB8
:104C90002B2DC5CD84918F010F5F1F4F882309F401
:104CA000C8CD0E94E193F801F5CF109220020C9438
:104CB000ED2E8BEE93E00E94D8A00E948E860C947D
:104CC000ED2E83E50E948B4C811103C0E6EEFDE1E1
:104CD0000DC00E94EB4B8D3320F480932B020C947B
:104CE000ED2E8CE380932B020C94ED2E84918F019A
:104CF0000F5F1F4F882321F00E94E193F801F6CF48
:104D000040912B0250E060E070E084EF93E00E945D
:104D100034C58AE00E94E1930C94ED2E89E690E080
:104D20000E94F3AD811111C0EBEFF3E084918F018C
:104D30000F5F1F4F882321F00E94E193F801F6CF07
:104D40000E94F0758AE00E94E19310923F100C944B
:104D5000882F83E50E948B4C882311F40C94ED2E50
:104D60000E94EB4B182F8D3308F01CE310934C106E
:104D70000E94F2586B017C01212F30E0A8EEB3E0D5
:104D80000E9493EAC60ED71EE81EF91EC092481074
:104D9000D0924910E0924A10F0924B100C94ED2EF4
:104DA0000E9435AE0C94ED2E8091100783FF02C057
:104DB0000C94ED2E83E50E948B4C882311F40C9407
:104DC000ED2E0E940B4C0E94E7EBCB010E941A4E85
:104DD0000C94ED2E0E94F9A80C94ED2E80E50E9413
:104DE0008B4C811106C083E50E948B4C882359F0BF
:104DF00005C00E94EB4B8111F0C7F5CF0E94DB4B41
:104E00006F3F710510F06FEF70E070934304609393
:104E10004204E3C780E50E948B4C811105C01092CB
:104E2000430410924204D9C70E94DB4B672B09F060
:104E3000D4C7F5CF0E9403790E94C7B710924304EC
:104E40001092420400E010E062E370E080E090E045
:104E50000E942DB70E94C37B0F5F1F4F03311105C6
:104E600099F762E370E080E090E00E942DB70E9425
:104E7000C37B0E94A22FB1C710922604AEC783E560
:104E80000E948B4C882399F00E940B4C20E030E06C
:104E90004AE754E40E94BCE60E94ECEB60932C02CB
:104EA00070932D0280932E0290932F0296C788E56F
:104EB0000E94424C8111ACC789E50E94424C81118D
:104EC000A7C78AE50E94424C8111A2C785E40E94CF
:104ED000424C81119DC7CEC783E50E94424C882376
:104EE00009F47BC70E940B4C20E030E04AE754E411
:104EF0000E94BCE60E94ECEB609344107093451056
:104F0000809346109093471068C7B7E5CB2EB2E068
:104F1000DB2E12E9E12E10E1F12E10E0D6018D9189
:104F20006D010E94424C882309F46DC0133009F0D2
:104F300063C00E940B4C4B015C0120E030E040EA72
:104F400051E40E9457E687FF4EC0A501940160918D
:104F50009E1070919F108091A0109091A1100E94BE
:104F60007FEB2B013C019B01AC016091DF0670914E
:104F7000E0068091E1069091E2060E94BCE6609313
:104F8000DF067093E0068093E1069093E206A301AA
:104F900092016091FF067091000780910107909146
:104FA00002070E94BCE66093FF067093000780939F
:104FB00001079093020760914B1170914C11809101
:104FC0004D1190914E110E945BE6A30192010E9447
:104FD000BCE60E94ECEB60934B1170934C118093F4
:104FE0004D1190934E1180929E1090929F10A0921E
:104FF000A010B092A11007C00E940B4CF701608373
:105000007183828393831F5FF4E0EF0EF11C1430F1
:1050100009F084CF0E9452C9E0C60E94126A83E55B
:105020000E948B4C882309F451C80E94DB4B6230EC
:10503000710509F04BC80E94C3C98BE50E94E1933A
:105040006091A4187091A5188091A6189091A71846
:1050500042E00E9487974091A8185091A91860914A
:10506000AA187091AB1881E094E00E9451C540915C
:10507000AC185091AD186091AE187091AF188EEFCA
:1050800093E00E9451C58DE50E94E1938AE00E9461
:10509000E193A3C684918F010F5F1F4F882321F0F6
:1050A0000E94E193F801F6CF60E083ED94E00E9466
:1050B000028D61E08CEC94E00E94028D61E081EC55
:1050C00094E00E94028D61E081EB94E00E94028DE9
:1050D00060E088EA94E00E94028D61E08EE994E04D
:1050E0000E94028D60E084E994E00E94028D60E0FD
:1050F0008CE894E00E94028D61E08EE794E00E94CB
:10510000028D60E080E794E00E94028D60E081E61D
:1051100094E00E94028D60E083E594E00E94028D9D
:1051200060E08DE394E00E94028D60E08CE294E008
:105130000E94028D60E087E194E00E94028D61E0B0
:1051400084E094E00E94028D48C6009111181091ED
:10515000121883E0D12C40E08150E9F0D8019C91F5
:10516000292F2B7F2134C1F711962C912133A1F7E0
:10517000913421F0953421F441E002C0DD24D39430
:1051800098012E5F3F4F89012F5F3F4FF8019081BB
:105190009032C9F3E1CF442369F0E6EEFDE184915A
:1051A0007F012FEFE21AF20A882321F00E94E19397
:1051B000F701F5CFDD2069F0E9EAF5E084917F01A0
:1051C0003FEFE31AF30A882321F00E94E193F701ED
:1051D000F5CFD8018D918D01882309F42ACB0E9447
:1051E000E193F7CF0E946ABEF8C581E0809337054E
:1051F00080933605F2C588EC90E00E94F3AD8111F2
:10520000ECC584E40E94424C882309F441C00E940A
:105210000B4C6B017C0111E020E030E0A9010E9401
:1052200057E6811101C010E010932A1120E030E010
:10523000A901C701B6010E9457E6882349F10E94DF
:105240000B4CE0914E07B4E0EB9FF0011124E15DBF
:10525000FE4E608371838283938320E030E0A90156
:1052600060912F1170913011809131119091321114
:105270000E9457E681110CC080E090E0A0EEBFE3F1
:1052800080932F1190933011A0933111B09332116C
:105290000E9405B8A2C5F70181917F010E94424C8E
:1052A000882351F00E940B4C0E94ECEBD8016D93C7
:1052B0007D938D939C9313970C5F1F4FC016D1065F
:1052C00051F70E94E1C789C5E7E5EE2EE2E0FE2E28
:1052D00003EF16E0F70181917F010E94424C882381
:1052E00041F00E940B4CD8016D937D938D939C935C
:1052F00013970C5F1F4FB7E003301B0759F76DC5BD
:1053000083E50E948B4C8823A1F00E940B4C609394
:10531000EB067093EC068093ED069093EE06609397
:10532000E7067093E8068093E9069093EA0610E09A
:1053300001C011E080E50E948B4C882359F00E9447
:105340000B4C6093EB067093EC068093ED06909304
:10535000EE0610E082E50E948B4C882359F00E94F3
:105360000B4C6093EF067093F0068093F1069093D8
:10537000F20610E084E50E948B4C882359F00E94CD
:105380000B4C6093E7067093E8068093E9069093D0
:10539000EA0623C5112309F420C54091EB0650917C
:1053A000EC066091ED067091EE0683EB95E00E94AD
:1053B00051C54091EF065091F0066091F106709151
:1053C000F20680EB95E00E9451C54091E7065091AE
:1053D000E8066091E9067091EA068DEA95E00E9480
:1053E00051C58AE00E94E193F8C481E50E94424CD5
:1053F0008823C1F08091210490912204009739F014
:105400004AE050E060E070E00E94D6E403C060E053
:1054100070E0CB0160930307709304078093050746
:105420009093060783E50E94424C882351F00E9426
:105430000B4C60930B0770930C0780930D079093B0
:105440000E0784E50E94424C882351F00E940B4CC9
:1054500060930707709308078093090790930A07E2
:1054600088E50E94424C882351F00E940B4C6093C7
:10547000D3067093D4068093D5069093D60689E51B
:105480000E94424C882351F00E940B4C6093D70637
:105490007093D8068093D9069093DA068AE50E9425
:1054A000424C8823F1F00E940B4C6093DB06709312
:1054B000DC068093DD069093DE062DEC3CEC4CEC94
:1054C0005DE30E9457E6181664F0E3ECF5E0849182
:1054D0008F010F5F1F4F882321F00E94E193F80195
:1054E000F6CF85E40E94424C882309F476C40E94DA
:1054F0000B4C6093DF067093E0068093E106909377
:10550000E2066BC467E5C62E62E0D62E78E3E72E8E
:1055100075E0F72E10E0F60181916F010E94424C78
:10552000882359F00E940B4CD7016D937D938D9386
:105530009C931397812F0E94B3AD1F5FB4E0EB0ED5
:10554000F11C133041F70C9466200E9486B481113F
:1055500044C40BEF12E2E2E3F4E0FDABECAB9E01DE
:105560002F5F3F4F590154E4852E53E2952E1901C8
:10557000F8016591759185919491ACA9BDA9CD90E3
:10558000DD90ED90FD90BDABACABA70196010E9404
:10559000A2EA2B013C01F101608371838283938332
:1055A00020E030E040EA51EC0E94C9EC87FD0AC0DF
:1055B00020E030E040EA51E4C301B2010E9457E626
:1055C00018162CF4F401849118160CF456C4D10169
:1055D000CD90DD90ED90FD901D0120E030E040EA9F
:1055E00051ECC701B6010E94C9EC87FD0AC020E05A
:1055F00030E040EA51E4C701B6010E9457E61816B0
:105600004CF5E1EDFDE184918F010F5F1F4F81119A
:1056100003C0E5EFF5E004C00E94E193F801F3CF89
:1056200084918F010F5F1F4F882321F00E94E19327
:10563000F801F6CF88E290E099A388A388EC90E087
:105640009DA78CA7BE01605E7F4FCE018C960E9405
:1056500083B5C3C30C5F1F4FBFEF8B1A9B0AE7E0F4
:10566000F3E2E017F10709F083CF48E3E42E45E0C9
:10567000F42E10E0F50181919191A191B1915F011A
:10568000F70181939193A193B1937F01812F0E94A0
:10569000B3AD1F5F133071F70E94358D83E992E03F
:1056A0009DA78CA704E610E019A308A3BE01645DC2
:1056B0007F4FCE0180960E9483B58AEB92E09DA732
:1056C0008CA719A308A3BE01645D7F4FCE0180960D
:1056D0000E9483B582C383E50E948B4C882309F422
:1056E0007CC30E94DB4B709303026093020275C37C
:1056F0008DED90E00E94F3AD81116FC383E50E94B0
:105700008B4C811103C0E6EEFDE13AC000914E07DB
:1057100010E00E94DB4B000F111FF801E85CFD4F09
:105720007183608380914E0790E07C01EE0CFF1C3A
:10573000EE0CFF1C87010F5D1D4F880F991FFC01A8
:10574000E85CFD4F60817181072E000C880B990B7E
:105750000E945DE62AE037ED43E25CE30E94BCE68E
:10576000F701E55DFE4E20813181428153810E9427
:10577000BCE6D8016D937D938D939C9313972DC3B5
:1057800084918F010F5F1F4F882321F00E94E193C6
:10579000F801F6CF85E40E94E19380914E07805D89
:1057A0000E94E193E0914E07F0E0EE0FFF1FE85CEE
:1057B000FD4F6081718183E196E00E946EC585E2B4
:1057C0000E94E1938AE00E94E19307C380E50E9472
:1057D000424C882309F401C30E94DB4B6B017C011E
:1057E00083E50E948B4C882321F00E94DB4B8B01C8
:1057F00002C00FEF1FEFC8010196039708F0EDC23A
:10580000D7FCEBC28C2DEBE1F6E09491891709F4FB
:105810003FC33196B6E0EB34FB07B9F73CC383E5F1
:105820000E948B4C882319F00E94DB4B02C064E07D
:1058300071E079A368A380E50E948B4C882339F03E
:105840000E94DB4B6938E3E17E0730F402C068EE6A
:1058500073E07A83698304C088E893E19A8389833B
:10586000BE01605E7F4FCE0101960E9483B5B5C236
:1058700085E40E948B4C811110C080E50E94424C4F
:10588000882391F00E940B4C60933C0770933D0776
:1058900080933E0790933F0707C00E94EB4B8823FD
:1058A00061F3E1EDFDE171C089E40E94424C88237F
:1058B00081F00E940B4C2CEA35EC47E25EE30E943B
:1058C000BCE6609338077093390780933A0790934A
:1058D0003B0784E40E94424C882381F00E940B4CD9
:1058E0002CEA35EC47E25EE30E947FEB60934007D1
:1058F000709341078093420790934307E6EEFDE1E2
:1059000084918F010F5F1F4F882321F00E94E19344
:10591000F801F6CF40913C0750913D0760913E075A
:1059200070913F0783E596E00E9451C52CEA35EC63
:1059300047E25EE3609138077091390780913A073A
:1059400090913B070E947FEBAB01BC018FE496E096
:105950000E9451C52CEA35EC47E25EE360914007B6
:105960007091410780914207909143070E94BCE6E5
:10597000AB01BC018BE496E00E9451C58AE00E9415
:10598000E1932BC20E94E193F80184918F010F5F94
:105990001F4F8111F7CFE7E5F6E084918F010F5F8C
:1059A0001F4F882309F419C20E94E193F801F5CF33
:1059B00083E50E94424C182F882371F00E940B4C03
:1059C0000E94E7EB709326026093250221E0672B8B
:1059D00009F020E020930F0780E50E94424C8823C5
:1059E00059F02091250230912602232B11F00E94BC
:1059F000FC4B80930F07F1C11111EFC1E6EEFDE101
:105A000084918F010F5F1F4F882321F00E94E19343
:105A1000F801F6CF80910F07882319F06BE173E04E
:105A200002C06EE173E08EE796E00E9487C5609148
:105A30002502709126028DE696E00E946EC5E9E689
:105A4000F6E084918F010F5F1F4F882309F4C5C1D1
:105A50000E94E193F801F5CF0E94CB86BEC180E59C
:105A60000E94424C882351F00E940B4C60933407F3
:105A700070933507809336079093370789E40E9427
:105A8000424C882381F00E940B4C2CEA35EC47E213
:105A90005EE30E94BCE66093300770933107809309
:105AA00032079093330784E40E94424C882381F0AC
:105AB0000E940B4C2CEA35EC47E25EE30E947FEB40
:105AC00060932C0770932D0780932E0790932F07D8
:105AD000E6EEFDE184918F010F5F1F4F882321F0D7
:105AE0000E94E193F801F6CF4091340750913507B9
:105AF000609136077091370789E996E00E9451C599
:105B00002CEA35EC47E25EE3609130077091310793
:105B100080913207909133070E947FEBAB01BC016B
:105B200085E996E00E9451C52CEA35EC47E25EE338
:105B300060912C0770912D0780912E0790912F076F
:105B40000E94BCE6AB01BC0181E996E00E9451C510
:105B50008AE00E94E19341C10E94E193F80184919F
:105B60008F010F5F1F4F8111F7CFEDE9F6E08491B0
:105B70008F010F5F1F4F882309F42FC10E94E1930B
:105B8000F801F5CF0E94A38528C10E944D7025C160
:105B90000E940EC322C183E50E94424C882321F05B
:105BA0000E94FC4B91E089270E949FBE16C181E0B4
:105BB000809317070E94436A10921707882309F4FD
:105BC0000CC1E6EEFDE184918F010F5F1F4F811143
:105BD00003C0ECEAF6E004C00E94E193F801F3CFC1
:105BE00084918F010F5F1F4F882309F4F6C00E9434
:105BF000E193F801F5CF8091310A882309F4EDC0D3
:105C000081E08093340AE9C08AE50E948B4C8111BF
:105C100003C0EAEBF6E00BC00E940B4C6093371117
:105C2000709338118093391190933A11D6C08491B2
:105C30008F010F5F1F4F882321F00E94E193F8012D
:105C4000F6CF409137115091381160913911709110
:105C50003A1187EB96E00E9451C58AE00E94E193D9
:105C6000BCC08BE40E948B4C811103C0E6EEFDE1C9
:105C700036C08BE40E948B4C8823C1F00E940B4CF1
:105C80006B017C0120E030E0A9010E94C9EC87FD96
:105C90000AC020E030E040E251E4C701B6010E94B2
:105CA00057E6181634F4E9EDF6E00EC0C12CD12CFD
:105CB00076010E94126AC092E306D092E406E09256
:105CC000E506F092E60689C084918F010F5F1F4FB1
:105CD000882309F482C00E94E193F801F5CF8491F2
:105CE0008F010F5F1F4F882321F00E94E193F8017D
:105CF000F6CF4091E3065091E4066091E50670917D
:105D0000E60688EF96E00E9451C58AE00E94E19382
:105D100064C081E08093270283E50E948B4C882336
:105D200039F00E94FC4B811158C00E9467CE55C0CB
:105D300083E50E94424CF7CF0E94B7B54EC0F09069
:105D400013180E94126A10917C1080E00E9449ACE6
:105D5000FF2029F1E6EEFDE184918F010F5F1F4FD7
:105D6000882321F00E94E193F801F6CF84E50E9498
:105D7000E1936F2D70E080E090E04AE00E9402978E
:105D800080E20E94E193E5E1F7E084918F010F5FEB
:105D90001F4F882311F10E94E193F801F6CF109272
:105DA0003E10812F0E9449ACE6EEFDE184918F0107
:105DB0000F5F1F4F882321F00E94E193F801F6CF77
:105DC00060913E1070E083E097E00E946EC58AE02B
:105DD0000E94E19302C00E94B7B510923F100E944A
:105DE0004ACE96C00E94C9AA0E9476CAF6CF0E94E7
:105DF000DB4BAB01BC014093AB0C5093AC0C6093FC
:105E0000AD0C7093AE0C8AEF9BE00E941298E5CF28
:105E10000E94126A88E50E94424C882331F05F9A02
:105E2000809131048E7F8093310489E50E94424C39
:105E3000882339F08A9A479A809131048D7F809324
:105E400031048AE50E94424C882361F08091080168
:105E50008095817080930601479A809131048B7FF1
:105E60008093310485E40E94424C882309F4B5CF25
:105E7000129AB3CF0E94C7B7B0CFF7FAF094F7F8F1
:105E8000F094D101CD92DD92ED92FC9213979FCBCD
:105E90000E948BE1A2CF0E94126ABC2C60E08C2D84
:105EA0000E942AB60F3FBFEF1B0759F48C2D0E94AA
:105EB000D4B531E020E0892B09F030E0032F122F18
:105EC00005C00130110561F401E010E08B2D0E9446
:105ED000D4B58017910709F480CF0E941FA1F6CF97
:105EE00000E010E0F3CF61E0812F0E942AB66E2D12
:105EF000812F0E94FCB5F12CB701812F0E9466B65C
:105F0000193009F06ACFF0924304E092420465CF61
:105F1000C657DF4F0FB6F894DEBF0FBECDBFDF917F
:105F2000CF911F910F91FF90EF90DF90CF90BF9096
:105F3000AF909F908F907F906F905F904F903F9029
:105F40002F9008952F923F924F925F926F927F927F
:105F50008F929F92AF92BF92CF92DF92EF92FF9279
:105F60000F931F93CF93DF93CDB7DEB76F970FB625
:105F7000F894DEBF0FBECDBFC0904C04D0904D044E
:105F8000E0904E04F0904F0420E030E040EA50E40E
:105F9000C701B6010E9457E687FD19C120E030E035
:105FA00041E953E4C701B6010E94C9EC18160CF48C
:105FB0000EC110924E0E10924D0E8091090140912B
:105FC0004C0E042E000C550B817021E0822790E0CE
:105FD0004817590709F433C08091090181702827B7
:105FE00020934C0E81111BC00E94AF80E1E3FDE0C5
:105FF00084918F01882351F0082E000C990B0E9488
:10600000AA800F5F1F4FF8018491F4CF8DE090E0DC
:106010000E94AA808AE090E00E94AA8010C0E5E376
:10602000FDE084918F01882389F3082E000C990BE1
:106030000E94AA800F5F1F4FF8018491F4CF8091D6
:106040003F0E833009F44CC02CF4882351F081308A
:10605000D9F072C0843009F43EC0853009F44DC0D7
:106060006BC08091310A882309F466C081E0809377
:106070003F0E0E94F2586093430E7093440E80933B
:10608000450E9093460E58C08091310A811154C03C
:106090008091FD0B882321F082E080933F0E4CC05D
:1060A00010923F0EEDE2FDE084918F01882351F0C4
:1060B000082E000C990B0E94AA800F5F1F4FF80159
:1060C0008491F4CF8DE090E00E94AA808AE090E075
:1060D0000E94AA8031C080918C0E8823E9F22CC0E6
:1060E0008091310A811128C08091B3099091B4093F
:1060F000891B8F7009F496C01FC08091310A8111ED
:106100001BC08091B3099091B409891B8F7009F469
:10611000ABC012C08DE090E00E94AA808AE090E0BF
:106120000E94AA8010923F0E8DE09DE09093A407FC
:106130008093A3070E940D948091340E9091350EA8
:1061400003974CF571E4272E79E0372EE0E68E2E8A
:10615000EAEE9E2EA12CB12C8AE99FE00E945D4BB5
:1061600018161906C4F48091340E9091350E0497D8
:1061700094F48AE99FE00E94214B80933A0EE091CB
:106180003B0EF0913C0E8A3019F08D3009F07DC045
:10619000309709F083C08091340E9091350E0097AE
:1061A00011F40C94233F01979093350E8093340E95
:1061B0008091360E9091370E019664E070E00E9457
:1061C0008CED9093370E8093360E0C94233F809184
:1061D0004D0E90914E0E8136FAEE9F07E8F0109228
:1061E0004E0E10924D0EE9E3FDE084918F0188235D
:1061F00051F0082E000C990B0E94AA800F5F1F4FD0
:10620000F8018491F4CF8DE090E00E94AA808AE0AA
:1062100090E00E94AA80D1CE019690934E0E80937A
:106220004D0ECBCE89E19DE09093A4078093A30708
:106230000E940D9480918C0E882311F082E001C0A1
:1062400084E080933F0EE5E1FDE084918F01882397
:1062500009F438CF082E000C990B0E94AA800F5F1A
:106260001F4FF8018491F3CFE1E1FDE084918F01AC
:10627000882309F44FCF082E000C990B0E94AA80A6
:106280000F5F1F4FF8018491F3CF8A3309F480CF59
:10629000EF35F10514F40C94B73C7ACF8091380EA9
:1062A0009091390E20E6289F7001299FF00C11244F
:1062B00087010C54134FE00FF11F108261E470E06E
:1062C000C8010E94F3ED009711F40C949B3C90934D
:1062D0003E0E80933D0E801B910B8E0D9F1D60E046
:1062E00070E08B54934F0E9458E20E94E7EBCB0181
:1062F000770FAA0BBB0B8232910510F00C949B3CDC
:10630000FC018827EE58FF4F8F4F0C949FEDE8E07B
:10631000FDE084918F01882351F0082E000C990B29
:106320000E94AA800F5F1F4FF8018491F4CF20E0F4
:1063300030E040E05FE360914C0470914D04809147
:106340004E0490914F041EC0E3E0FDE084918F0164
:10635000882351F0082E000C990B0E94AA800F5F31
:106360001F4FF8018491F4CF60914A0470914B045F
:10637000072E000C880B990B0E945DE620E030E0B0
:1063800040E05FE30E94A3EA0E94E7EBCB010E949A
:10639000E44D0E94DBD78DE090E00E94AA808AE065
:1063A00090E00E94AA800C949B3CEEEFFCE084916C
:1063B0008F01882351F0082E000C990B0E94AA80AF
:1063C0000F5F1F4FF8018491F4CF20E030E040E0F0
:1063D0005FE3609146047091470480914804909176
:1063E0004904D0CFE9EFFCE084918F01882351F07C
:1063F000082E000C990B0E94AA800F5F1F4FF80116
:106400008491F4CF6091440470914504B1CF209100
:1064100042043091430444E6429FC001439F900DE3
:1064200011246FEF70E00E948CED8B0165367105D1
:1064300010F004E610E0E4EFFCE084917F01882393
:1064400059F0082E000C990B0E94AA80FFEFEF1A5A
:10645000FF0AF7018491F3CFB80180E090E036C7DE
:10646000E0EFFCE084918F01882351F0082E000CAE
:10647000990B0E94AA800F5F1F4FF8018491F4CFFF
:1064800080E290E00E94AA80ECEEFCE084918F0113
:10649000882351F0082E000C990B0E94AA800F5FF0
:1064A0001F4FF8018491F4CF60913204709133044E
:1064B00080913404909135040E94DCD780E290E012
:1064C0000E94AA80E8EEFCE084918F01882351F0BD
:1064D000082E000C990B0E94AA800F5F1F4FF80135
:1064E0008491F4CF60913604709137048091380420
:1064F000909139040E94DCD780E290E00E94AA804B
:10650000E4EEFCE084918F01882351F0082E000C0A
:10651000990B0E94AA800F5F1F4FF8018491F4CF5E
:1065200060913A0470913B0480913C0490913D0449
:106530000E94DCD780E290E0A0C58091310A8823D8
:1065400009F450C0EFEDFCE084918F01882351F0F5
:10655000082E000C990B0E94AA800F5F1F4FF801B4
:106560008491F4CF8091320A882359F18091FD0BF8
:10657000882329F18091A70C9091A80CA091A90CD7
:10658000B091AA0C0097A105B105C1F0BC01CD01E5
:106590006D597F4F8F4F9F4F24E630E040E050E031
:1065A0000E9445EA6091AB0C7091AC0C8091AD0CEF
:1065B0009091AE0C0E9445EA822F01C080E090E0ED
:1065C000E6CEEBEDFCE084918F01882309F4E3CE65
:1065D000082E000C990B0E94AA800F5F1F4FF80134
:1065E0008491F3CFE3EDFCE084918F01882309F4DB
:1065F000D2CE082E000C990B0E94AA800F5F1F4F6D
:10660000F8018491F3CFEEECFCE084918F018823B4
:1066100051F0082E000C990B0E94AA800F5F1F4FAB
:10662000F8018491F4CF8091430E9091440EA09193
:10663000450EB091460E892B8A2B8B2B09F477C01F
:106640000E94F258A50194010E9445EA69017A016D
:106650006091430E7091440E8091450E9091460ECC
:10666000A50194010E9445EA8601021B130BC80193
:106670006CE370E00E9478EDCB019927EAE0F0E04E
:10668000BF010E948CED282FCB01BF010E948CED31
:10669000805D80932904205D20932A0410922B04AE
:1066A00089E294E00E94DBD780E290E00E94AA8019
:1066B000ECECFCE084917F01882359F0082E000C5B
:1066C000990B0E94AA80FFEFEF1AFF0AF70184914D
:1066D000F3CF80E290E00E94AA80C8016CE370E0F2
:1066E0000E9478ED6AE070E00E948CED605D60933E
:1066F0002904805D80932A0410922B0489E294E09F
:106700000E94DBD780E290E00E94AA80EAECFCE0E5
:1067100084918F01882309F43ECE082E000C990B3A
:106720000E94AA800F5F1F4FF8018491F3CF80E28F
:1067300090E00E94AA80E2ECFCE084918F01882323
:1067400009F429CE082E000C990B0E94AA800F5F35
:106750001F4FF8018491F3CF10926D0E80910901C3
:1067600080FF11C0EEEBFCE084918F01882309F4D7
:1067700012CE082E000C990B0E94AA800F5F1F4FAB
:10678000F8018491F3CF83E50E9477D7882341F005
:106790000E9492D70E94ECEB7093420E6093410EE0
:1067A000EAEBFCE084918F01882351F0082E000C65
:1067B000990B0E94AA800F5F1F4FF8018491F4CFBC
:1067C0008DE090E00E94AA808AE090E00E94AA807A
:1067D00080918B0E882309F442C28091410E9091E2
:1067E000420E8430910509F4C8C08830910509F43F
:1067F0007DC1892B09F0E7C3EEEDFAE084918F01AA
:10680000882351F0082E000C990B0E94AA800F5F7C
:106810001F4FF8018491F4CF8DE090E00E94AA8090
:106820008AE090E00E94AA80E3EDFAE084918F0173
:10683000882351F0082E000C990B0E94AA800F5F4C
:106840001F4FF8018491F4CF8DE090E00E94AA8060
:106850008AE090E00E94AA80E7ECFAE084918F0140
:10686000882351F0082E000C990B0E94AA800F5F1C
:106870001F4FF8018491F4CF8DE090E00E94AA8030
:106880008AE090E00E94AA80EBEBFAE084918F010D
:10689000882351F0082E000C990B0E94AA800F5FEC
:1068A0001F4FF8018491F4CF8DE090E00E94AA8000
:1068B0008AE090E00E94AA80EDEAFAE084918F01DC
:1068C000882351F0082E000C990B0E94AA800F5FBC
:1068D0001F4FF8018491F4CF8DE090E00E94AA80D0
:1068E0008AE090E00E94AA80EFE9FAE084918F01AB
:1068F000882351F0082E000C990B0E94AA800F5F8C
:106900001F4FF8018491F4CF8DE090E00E94AA809F
:106910008AE090E00E94AA80E2E9FAE084918F0187
:10692000882351F0082E000C990B0E94AA800F5F5B
:106930001F4FF8018491F4CF8DE090E00E94AA806F
:106940008AE090E00E94AA80E5E8FAE084918F0155
:10695000882351F0082E000C990B0E94AA800F5F2B
:106960001F4FF8018491F4CF8DE090E00E94AA803F
:106970008AE090E00E94AA8026C3E7E7FAE08491CB
:106980008F01882351F0082E000C990B0E94AA80D9
:106990000F5F1F4FF8018491F4CF8DE090E00E94CB
:1069A000AA808AE090E00E94AA80E9E6FAE0849159
:1069B0008F01882351F0082E000C990B0E94AA80A9
:1069C0000F5F1F4FF8018491F4CF8DE090E00E949B
:1069D000AA808AE090E00E94AA80E3E5FAE0849130
:1069E0008F01882351F0082E000C990B0E94AA8079
:1069F0000F5F1F4FF8018491F4CF8DE090E00E946B
:106A0000AA808AE090E00E94AA80EDE3FAE08491F7
:106A10008F01882351F0082E000C990B0E94AA8048
:106A20000F5F1F4FF8018491F4CF8DE090E00E943A
:106A3000AA808AE090E00E94AA80EBE2FAE08491CA
:106A40008F01882351F0082E000C990B0E94AA8018
:106A50000F5F1F4FF8018491F4CF8DE090E00E940A
:106A6000AA808AE090E00E94AA80E9E1FAE084919D
:106A70008F01882351F0082E000C990B0E94AA80E8
:106A80000F5F1F4FF8018491F4CF8DE090E00E94DA
:106A9000AA808AE090E00E94AA80EBE0FAE084916C
:106AA0008F01882351F0082E000C990B0E94AA80B8
:106AB0000F5F1F4FF8018491F4CF8DE090E00E94AA
:106AC000AA808AE090E00E94AA80EDEFF9E084912C
:106AD0008F01882309F448CF082E000C990B0E94DF
:106AE000AA800F5F1F4FF8018491F3CFE6EFF9E022
:106AF00084918F01882351F0082E000C990B0E947D
:106B0000AA800F5F1F4FF8018491F4CF8DE090E0D1
:106B10000E94AA808AE090E00E94AA80EFEEF9E04D
:106B200084918F01882351F0082E000C990B0E944C
:106B3000AA800F5F1F4FF8018491F4CF8DE090E0A1
:106B40000E94AA808AE090E00E94AA80E8EDF9E025
:106B500084918F01882351F0082E000C990B0E941C
:106B6000AA800F5F1F4FF8018491F4CF8DE090E071
:106B70000E94AA808AE090E00E94AA80E1ECF9E0FD
:106B800084918F01882351F0082E000C990B0E94EC
:106B9000AA800F5F1F4FF8018491F4CF8DE090E041
:106BA0000E94AA808AE090E00E94AA80EAEAF9E0C6
:106BB00084918F01882351F0082E000C990B0E94BC
:106BC000AA800F5F1F4FF8018491F4CF8DE090E011
:106BD0000E94AA808AE090E00E94AA80E3E9F9E09E
:106BE00084918F01882351F0082E000C990B0E948C
:106BF000AA800F5F1F4FF8018491F4CF8DE090E0E1
:106C00000E94AA808AE090E00E94AA80E5E8F9E06C
:106C100084918F01882351F0082E000C990B0E945B
:106C2000AA800F5F1F4FF8018491F4CF8DE090E0B0
:106C30000E94AA808AE090E00E94AA80E7E7F9E03B
:106C400084918F01882309F48FCE082E000C990BB4
:106C50000E94AA800F5F1F4FF8018491F3CF8091AB
:106C6000320A882309F486C181E08093AF0C109228
:106C7000B10C1092B00C81E89AE00E94599A8BE115
:106C8000E1E8FAE0DE01159601900D928A95E1F7B0
:106C900080917F0A9091800A9C838B838DEE92E095
:106CA0009A83898340E050E0BE016F5F7F4F80E0B0
:106CB00090E00E94E082CE0101960E94B5A0C090B3
:106CC000B00CD090B10C0091410E1091420EC60153
:106CD000801B910B049720F06801F3E0CF0ED11CCC
:106CE00058E6452E59E0552E69E5662E69E0762E68
:106CF000C016D10608F467C10115110509F0A1C03D
:106D000065E37AE081E89AE00E94219962E273E00B
:106D100085E39AE00E94FEED892B09F04AC0F2015A
:106D2000849148E6E42E49E0F42E882359F0082E99
:106D3000000C990B0E94AA80FFEFEF1AFF0AF701DF
:106D40008491F3CF8DE090E00E94AA808AE090E0E9
:106D50000E94AA80F301849139E5E32E39E0F32EF5
:106D6000882359F0082E000C990B0E94AA80FFEF8F
:106D7000EF1AFF0AF7018491F3CF8DE090E00E94B3
:106D8000AA808AE090E00E94AA804AE060E070E079
:106D9000CB010E940297E9E4F9E084917F012FEF93
:106DA000E21AF20A882309F4E2C00E94E193F70193
:106DB000F4CFE5E4F9E084917F01882359F0082EAF
:106DC000000C990B0E94AA80FFEFEF1AFF0AF7014F
:106DD0008491F3CF8DE090E00E94AA808AE090E059
:106DE0000E94AA80F101849121E4E22E29E0F22E92
:106DF000882359F0082E000C990B0E94AA80FFEFFF
:106E0000EF1AFF0AF7018491F3CF8DE090E00E9422
:106E1000AA808AE090E00E94AA804AE060E070E0E8
:106E2000CB010E940297ECE3F9E084917F012FEF00
:106E3000E21AF20A882309F49AC00E94E193F7014A
:106E4000F4CF60E070E0C80101970E94A6848091B1
:106E5000330A882309F45FC0EAE3F9E084917F01F3
:106E6000882359F0082E000C990B0E94AA80FFEF8E
:106E7000EF1AFF0AF7018491F3CF85E39AE00E94AD
:106E8000DBD78DE090E00E94AA808AE090E00E942B
:106E9000AA80E8E3F9E084917F01882359F0082E65
:106EA000000C990B0E94AA80FFEFEF1AFF0AF7016E
:106EB0008491F3CF82E49AE00E94DBD78DE090E0EA
:106EC0000E94AA808AE090E00E94AA80C801A0E007
:106ED000B0E04AE0BC01CD010E940297E6E3F9E090
:106EE00084917F012FEFE21AF20A882321F00E9499
:106EF000E193F701F5CF92E4E92E9AE0F92EF7013C
:106F000081917F01882319F00E94E193F8CF8AE0F4
:106F10000E94E1932CC085E39AE00E94DBD78DE0CC
:106F200090E00E94AA808AE090E00E94AA8082E419
:106F30009AE00E94DBD78DE090E00E94AA808AE070
:106F400090E00E94AA80C801A0E0B0E04AE0BC0145
:106F5000CD010E94029782E4E82E8AE0F82EF70124
:106F600081917F01882399F20E94E193F8CF0F5F0E
:106F70001F4FBECEE7E2F9E084918F01882351F0E4
:106F8000082E000C990B0E94AA800F5F1F4FF8017A
:106F90008491F4CF8DE090E00E94AA808AE090E096
:106FA0000E94AA80E8E1F9E084918F01882309F426
:106FB000DBCC082E000C990B0E94AA800F5F1F4F9C
:106FC000F8018491F3CFE6EBFCE084918F018823F4
:106FD00009F4E1C9082E000C990B0E94AA800F5FEA
:106FE0001F4FF8018491F3CF8091310A882339F043
:106FF0000E941282A0C48091310A8823E9F00E9485
:107000002EB199C480913F0E823019F0833609F079
:1070100092C40E94F181E2EBFCE084918F0188230D
:1070200009F4B9C9082E000C990B0E94AA800F5FC1
:107030001F4FF8018491F3CF80913F0E833609F002
:107040007AC4DDCF89EA9CE00E94D8A08091B30980
:107050009091B409891B8F7009F06DC480913F0E27
:10706000823009F468C4833609F099C464C48DE0A1
:1070700090E00E94AA808AE090E00E94AA808BC9DA
:107080008091B3099091B409891B8F7009F053C4A2
:1070900080913F0E823009F44EC4833609F44BC40C
:1070A0008091FD0B8111CFC446C483E50E9477D740
:1070B000811126C083E40E9477D7882309F43BC45A
:1070C0008091B3099091B409891B8F7009F033C482
:1070D00020E030E040E251E460913A0470913B04DA
:1070E00080913C0490913D040E9457E687FF08C0C0
:1070F00086E99CE09093A4078093A3070E940D94D7
:107100000E9492D720E030E0A9010E9457E687FD57
:1071100010C00E9492D720E030E849E853E40E9472
:10712000C9EC18164CF00E9492D70E94ECEBCB01F0
:1071300005C080E090E002C083E191E00E94E75941
:10714000FAC383E50E9477D7882309F4F4C30E9429
:1071500092D720E030E0A9010E9457E687FD10C0D9
:107160000E9492D720E030E046E153E40E94C9EC4F
:1071700018164CF00E9492D70E94ECEBCB0105C090
:1071800080E090E002C086E990E00E941A4ED3C3EE
:1071900083E50E9477D78823D9F00E9492D720E018
:1071A00030E04FE753E40E94BCE620E030E048ECDA
:1071B00052E40E947FEB0E94ECEB6F3F710519F0E7
:1071C00010F06FEF70E07093430460934204E3C8E3
:1071D0008FEF90E09093430480934204DCC8809149
:1071E000B3099091B409891B8F7009F0D4C88091BC
:1071F000310A8111D0C80E948E865F9A8091310435
:107200008E7F809331048A9A479A809131048D7FD2
:1072100080933104809108018095817080930601EC
:10722000479A809131048B7F80933104129AB3C8BE
:1072300083E50E9477D7882319F10E9492D720E036
:1072400030E040E252E40E9457E687FD0FC00E9402
:1072500092D720E030EC49E754E40E94C9EC1816BC
:1072600044F00E9492D70E94E7EB05C068E270E00C
:1072700002C067EE73E070930302609302025BC387
:10728000E0E9FCE084918F01882351F0082E000C86
:10729000990B0E94AA800F5F1F4FF8018491F4CFD1
:1072A000C0900202D09003020D2C000CEE08FF08E3
:1072B000F7FE0EC06DE28AE99FE00E94D44A66277D
:1072C0007727CB016C197D098E099F094AE003C01D
:1072D0004AE0C701B6010E949BD75DC88091B309FF
:1072E0009091B409891B8F7009F025C380913F0EDE
:1072F000823009F420C3833609F0EBC21CC38091AD
:10730000B3099091B409891B8F7009F044C880912A
:107310003F0E823009F43FC8833609F0B6C33BC83C
:107320008091B3099091B409891B8F7009F003C350
:1073300080913F0E823009F4FEC2833609F0FBC40F
:10734000FAC28091B3099091B409891B8F7009F03A
:10735000F2C280913F0E823009F4EDC2833609F00B
:1073600020C5E9C28091B3099091B409891B8F703F
:1073700009F0E1C280913F0E823009F4DCC283360D
:1073800009F045C5D8C280916D0E811103C00E94DD
:10739000AF80C4C18E3271F580916E0E8E3209F0CD
:1073A00046C18091D20B882309F4B8C181508093E3
:1073B000D20B882361F090E001974FE1489F900144
:1073C000499F300D1124C9018456954F02C08EE5A6
:1073D0009AE02BE1FC013496A1E8BAE001900D920D
:1073E0002A95E1F7FC01828193819093800A809332
:1073F0007F0A94C18C3309F01AC164E273E08DE610
:107400009EE00E94FEED892B21F481E080938B0E9B
:1074100085C163E373E08DE69EE00E94FEED892B5B
:1074200079F4E4EFF8E084918F010F5F1F4F882318
:1074300021F00E94E193F801F6CF86ED98E0E4C0D8
:107440006AE473E08DE69EE00E94FEED892B79F4FC
:10745000E2EBF8E084918F010F5F1F4F882321F04A
:107460000E94E193F801F6CF8EE998E0CDC061E685
:1074700073E08DE69EE00E94FEED892B79F4E3E84F
:10748000F8E084918F010F5F1F4F882321F00E9445
:10749000E193F801F6CF8EE798E0B6C06FE673E0AF
:1074A0008DE69EE00E94FEED892B79F4E3E6F8E09C
:1074B00084918F010F5F1F4F882321F00E94E19379
:1074C000F801F6CF8EE598E09FC06DE773E08DE69A
:1074D0009EE00E94FEED892B79F4E3E4F8E08491CC
:1074E0008F010F5F1F4F882321F00E94E193F80165
:1074F000F6CF8AE398E088C06BE873E08DE69EE003
:107500000E94FEED892B71F407E118E0F8018491E7
:10751000882329F00F5F1F4F0E94E193F7CF80E18E
:1075200098E072C061EA73E08DE69EE00E94FEED95
:10753000892B79F4E1EFF7E084918F010F5F1F4F02
:10754000882321F00E94E193F801F6CF8AEE97E0BC
:107550005BC063EB73E08DE69EE00E94FEED892B3D
:1075600079F4E2EDF7E084918F010F5F1F4F8823DC
:1075700021F00E94E193F801F6CF81EC97E044C03E
:107580006EEB73E08DE69EE00E94FEED892B79F4B0
:10759000E8EAF7E084918F010F5F1F4F882321F005
:1075A0000E94E193F801F6CF86E997E02DC06AECDE
:1075B00073E08DE69EE00E94FEED892B79F4EBE707
:1075C000F7E084918F010F5F1F4F882321F00E9405
:1075D000E193F801F6CF89E697E016C068ED73E015
:1075E0008DE69EE00E94FEED892BA9F4EFE4F7E022
:1075F00084918F010F5F1F4F882321F00E94E19338
:10760000F801F6CF8DE397E09093A4078093A3074A
:107610000E940D9483C065EE73E08DE69EE00E94AB
:10762000FEED892B09F07AC010928B0E77C01D8277
:1076300018861C821B828DEE92E09A83898380914A
:10764000840A811103C06EE57AE002C06DE77AE03A
:107650006115710519F06C5F7F4F02C060E070E04A
:1076600021E04DE65EE0CE0105960E94889E8823CB
:1076700061F18BE1FE013596A1E8BAE001900D922F
:107680008A95E1F72B813C813093800A20937F0A11
:107690008091D20B8A3008F03DC091E0980F909312
:1076A000D20BFFE18F9FC0011124DC01A056B54F22
:1076B0004BE1E1E8FAE001900D924A95E1F7FC0117
:1076C000E456F54F3383228325C0E6EEFDE1849135
:1076D0008F010F5F1F4F882321F00E94E193F80173
:1076E000F6CFE7E2F7E084918F010F5F1F4F882309
:1076F00021F00E94E193F801F6CF0DE61EE0F801BB
:1077000081918F01882319F00E94E193F8CF8AE0DC
:107710000E94E193CE0101960E94B5A010926D0ED9
:107720008091090180FF07C1E4EDFBE084918F01A6
:10773000882311F40C94CB31082E000C990B0E9475
:10774000AA800F5F1F4FF8018491F2CF8FE40E944F
:1077500077D781110C94CB3183E40E9477D70C94B6
:10776000CB3183E50E9477D7811159C08FE40E9405
:1077700077D7882319F08CE99BE007C084E50E9445
:1077800077D7882349F084E79BE09093A407809300
:10779000A3070E940D9443C083E40E9477D78823F7
:1077A00019F08BE49BE0F1CF81E50E9477D7882325
:1077B00019F083E29BE0E9CF88E40E9477D7882321
:1077C000C9F0EFE1FBE084918F01882351F0082E8E
:1077D000000C990B0E94AA800F5F1F4FF801849143
:1077E000F4CF8DE090E00E94AA808AE090E00E94B1
:1077F000AA8015C08CE40E9477D7882381F0EBE142
:10780000FBE084918F01882361F3082E000C990B13
:107810000E94AA800F5F1F4FF8018491F4CFE3EE1E
:10782000FBE084918F01882311F40C94CB31082E56
:10783000000C990B0E94AA800F5F1F4FF8018491E2
:10784000F2CF8091B3098091B4090C94CB3183E5D8
:107850000E9477D7882309F46EC083EF9AE0909353
:10786000A4078093A3070E940D94E3EEFBE08491AC
:107870008F01882311F40C94CB31082E000C990B46
:107880000E94AA800F5F1F4FF8018491F2CFEEEEA5
:10789000FAE084918F01882351F0082E000C990B97
:1078A0000E94AA800F5F1F4FF8018491F4CFE9EE88
:1078B000FAE084918F01882311F40C94CB31082EC7
:1078C000000C990B0E94AA800F5F1F4FF801849152
:1078D000F2CF88E50E9477D7811106C089E50E9422
:1078E00077D7882309F4C3C088E50E9477D7882317
:1078F00041F08AE89CE09093A4078093A3070E943C
:107900000D9489E50E9477D7882341F084E89CE0B4
:107910009093A4078093A3070E940D948AE50E9488
:1079200077D7882341F08EE79CE09093A40780935B
:10793000A3070E940D948091380E9091390E019604
:1079400064E070E00E948CED9093390E8093380EC5
:107950008091340E9091350E01969093350E809360
:10796000340E10923C0E10923B0E0C94AC304091B1
:10797000380E5091390E9F012F5F3F4F30933C0ED0
:1079800020933B0E90E6949F9001959F300D11241B
:107990002C54334FE20FF31F80830C94AC300091D2
:1079A0003D0E10913E0E780124E0E20EF11C6AE2D9
:1079B00070E0C7010E94F3EDF80124812F3221F419
:1079C000B8016B5F7F4F03C02C3339F4B7018DE6EC
:1079D0009EE00E9407EE0C94CB3110926D0E009742
:1079E00019F0FC013197108280913D0E90913E0E6E
:1079F00040E061E004960E94A5D58091FD0B8823AC
:107A000089F0E5EAFCE084918F01882309F42FCB0B
:107A1000082E000C990B0E94AA800F5F1F4FF801DF
:107A20008491F3CFE1EAFCE084918F01882309F48B
:107A30001ECB082E000C990B0E94AA800F5F1F4FCF
:107A4000F8018491F3CF0E94F181EDE9FCE084918B
:107A50008F01882311F40C94CB31082E000C990B64
:107A60000E94AA800F5F1F4FF8018491F2CF8AE530
:107A70000E9477D7811138CF83E40E9477D788237B
:107A800009F459CF8AE79CE050CF86E40E9477D76B
:107A9000882309F44DC10E9492D70E94ECEB8B0120
:107AA00086E79CE09093A4078093A3070E940D941F
:107AB00088E50E9477D7882309F451C00E9492D7A5
:107AC0002B013C012DEC3CEC4CE45EE30E9457E6BC
:107AD0009E012F5F3F4F7901181674F020E030E0CF
:107AE000A901C301B2010E94C9EC18162CF41F931E
:107AF0000F938BE69CE005C12DEC3CEC4CEC5DEB70
:107B0000C301B2010E9457E618167CF020E030E075
:107B100040E85FEBC301B2010E94C9EC18162CF4D7
:107B20001F930F938FE59CE0ECC01F930F93C3014D
:107B3000B2010E94E7EB7F936F9385E59CE09F93F2
:107B40008F93FF92EF920E9429E60FB6F894DEBF62
:107B50000FBECDBFCE0101960E94E893DFC089E53C
:107B60000E9477D7882309F441C00E9492D72B0145
:107B70003C012DEC3CEC4CE45EE30E9457E6FE0138
:107B800031967F01181674F020E030E0A901C3019E
:107B9000B2010E94C9EC18162CF41F930F938AE4CB
:107BA0009CE0AFC02DEC3CEC4CEC5DEBC301B201B2
:107BB0000E9457E618167CF020E030E040E85FEBCA
:107BC000C301B2010E94C9EC18162CF41F930F9345
:107BD0008EE39CE096C01F930F93C301B2010E94F5
:107BE000E7EB7F936F9384E39CE0A9CF8AE50E9443
:107BF00077D7882309F441C00E9492D72B013C011A
:107C00002DEC3CEC4CE45EE30E9457E6FE0131961D
:107C10007F01181674F020E030E0A901C301B20121
:107C20000E94C9EC18162CF41F930F9389E29CE074
:107C300068C02DEC3CEC4CEC5DEBC301B2010E9442
:107C400057E618167CF020E030E040E85FEBC30117
:107C5000B2010E94C9EC18162CF41F930F938DE10A
:107C60009CE04FC01F930F93C301B2010E94E7EB4A
:107C70007F936F9383E19CE062CF85E40E9477D786
:107C8000882309F44BC00E9492D72B013C012DECB4
:107C90003CEC4CE45EE30E9457E6FE0131967F0126
:107CA000181674F020E030E0A901C301B2010E946F
:107CB000C9EC18162CF41F930F9388E09CE021C0A8
:107CC0002DEC3CEC4CEC5DEBC301B2010E9457E69D
:107CD00018167CF020E030E040E85FEBC301B20111
:107CE0000E94C9EC18162CF41F930F938CEF9BE0A5
:107CF00008C0C301B2010E94E7EB7F936F9381EF4D
:107D00009BE09F938F93FF92EF920E9429E60F9042
:107D10000F900F900F900F900F901CCF8DEE9BE067
:107D20009093A4078093A3070E940D940C94CB31E9
:107D300000E010E0B5CE20E030E040E251E4609198
:107D40003A0470913B0480913C0490913D040E9460
:107D500057E687FF08C086EE9BE09093A4078093C8
:107D6000A3070E940D9482E390E0909345048093D2
:107D700044040E94AA7688EC90E00E94E759E3EE62
:107D8000FBE084918F01882311F40C94CB31082EF1
:107D9000000C990B0E94AA800F5F1F4FF80184917D
:107DA000F2CF20E030E040E251E460913A0470917B
:107DB0003B0480913C0490913D040E9457E687FF6C
:107DC00008C08CED9BE09093A4078093A3070E94CA
:107DD0000D9480E590E090934504809344040E94C4
:107DE000AA7680EF90E00E94E759E3EEFBE08491F1
:107DF0008F01882311F40C94CB31082E000C990BC1
:107E00000E94AA800F5F1F4FF8018491F2CF80E09B
:107E100090E00E94E75910924504109244040E9499
:107E2000AA76E8EDFBE084918F01882311F40C948D
:107E3000CB31082E000C990B0E94AA800F5F1F4FB8
:107E4000F8018491F2CF6F960FB6F894DEBF0FBEA3
:107E5000CDBFDF91CF911F910F91FF90EF90DF90F9
:107E6000CF90BF90AF909F908F907F906F905F90DA
:107E70004F903F902F9008952F923F924F925F9294
:107E80006F927F928F929F92AF92BF92CF92DF922A
:107E9000EF92FF920F931F93CF93DF93CDB7DEB78F
:107EA00062970FB6F894DEBF0FBECDBFF8948FEF88
:107EB0009FEF90938900809388002AE02A8B212CE1
:107EC000312C78948091A2049091A304A091A404F1
:107ED000B091A504892B8A2B8B2B09F00FC28091BE
:107EE0001A078823E1F010921A07809118079091E1
:107EF0001907892B09F402C210925A04109219072B
:107F0000109218079091B3098091B409981709F459
:107F1000F5C18091B4098F5F8F708093B40980910F
:107F2000180790911907892B09F4E8C140919E0424
:107F300050919F046091A0047091A10480919A04D3
:107F400090919B04A0919C04B0919D040091910498
:107F500010E020E030E0841B950BA60BB70B081750
:107F600019072A073B0710F4D901C801E82F840F2D
:107F7000951FA61FB71F80939E0490939F04A09304
:107F8000A004B093A1042091840030918500245E68
:107F90003F4F40917604509177046091780470913E
:107FA00079048091660490916704A0916804B0916F
:107FB0006904840F951FA61FB71F809376049093C2
:107FC0007704A0937804B0937904B7FD1CC0889A15
:107FD0008091821090918310A0918410B0918510AF
:107FE00040910402042E000C550B660B770B840F96
:107FF000951FA61FB71F8093821090938310A093A4
:108000008410B093851040917A0450917B04609164
:108010007C0470917D0480916A0490916B04A0911E
:108020006C04B0916D04840F951FA61FB71F809339
:108030007A0490937B04A0937C04B0937D04B7FDF5
:108040001CC08E9A8091861090918710A091881004
:10805000B091891040910502042E000C550B660B5F
:10806000770B840F951FA61FB71F809386109093E0
:108070008710A0938810B093891040917E0450918E
:108080007F04609180047091810480916E049091CE
:108090006F04A0917004B0917104840F951FA61F06
:1080A000B71F80937E0490937F04A0938004B093C5
:1080B0008104B7FD3FC080915404F09106028823EB
:1080C000C9F08091520482FF02C0F7FD06C0809182
:1080D0005104882311F40C94E64880915204909145
:1080E000530493FF02C0F7FD0CC08091500481112E
:1080F00008C006C080910B018095887080930901AB
:10810000419A40918A1050918B1060918C1070911F
:108110008D108F2FFF0F990BAA0BBB0B840F951F90
:10812000A61FB71F80938A1090938B10A0938C107A
:10813000B0938D1040918204509183046091840427
:10814000709185048091720490917304A0917404DD
:10815000B0917504840F951FA61FB71F80938204EA
:1081600090938304A0938404B0938504B7FD3AC030
:1081700040918E1050918F106091901070919110DD
:10818000C09007020C2C000CDD08EE08FF084C0D17
:108190005D1D6E1D7F1D40938E1050938F10609358
:1081A000901070939110409162045091630460911B
:1081B000640470916504841B950BA60BB70B809328
:1081C000820490938304A0938404B09385049091D7
:1081D000550480918F0493FF02C0815001C08F5FCE
:1081E00080938F048091760490917704A091780415
:1081F000B0917904B7FD15C04091620450916304B9
:108200006091640470916504841B950BA60BB70BF9
:108210008093760490937704A0937804B0937904C4
:10822000889880917A0490917B04A0917C04B0910D
:108230007D04B7FD15C040916204509163046091C4
:10824000640470916504841B950BA60BB70B809397
:108250007A0490937B04A0937C04B0937D048E9861
:1082600080917E0490917F04A0918004B09181045C
:10827000B7FD3AC040916204509163046091640478
:1082800070916504841B950BA60BB70B80937E043D
:1082900090937F04A0938004B09381048091540450
:1082A0008823E1F08091520482FF04C0809106028D
:1082B00087FD05C080915104882309F48FC7809100
:1082C00052049091530493FF04C08091060287FDED
:1082D0000BC080915004811107C005C080910B0133
:1082E0008870809309014198E15041F080918400A9
:1082F0009091850082179307C8F34BCE80911102AD
:1083000090911202A0911302B0911402892B8A2B32
:108310008B2B09F08AC080919004882309F453C004
:1083200080909E0490909F04A090A004B090A1041F
:10833000C0908B04D0908C04E0908D04F0908E045B
:1083400040918F04C814D904EA04FB0480F480919E
:108350005B0490915C0420915F04309160042817C5
:10836000390728F4415040938F04019714C08C14AE
:108370009D04AE04BF04E0F480915B0490915C0422
:1083800020915D0430915E048217930788F44F5F5B
:1083900040938F04019690935C0480935B0440911A
:1083A0000D0250910E0260910F02709110020EC0EA
:1083B0008FEF9FEFDC0180930D0290930E02A0934C
:1083C0000F02B09310024FEF5FEFBA0180918F045C
:1083D00087FD02C0169A01C0169880918400909182
:1083E00085004C9620918F042223B9F0149A209195
:1083F0008F0427FF02C02F5F01C0215020938F04FC
:10840000149820918F04222369F3209184003091E5
:10841000850028173907C8F3E5CF40931102509320
:10842000120260931302709314028091A20490913F
:10843000A304A091A404B091A504892B8A2B8B2BB3
:1084400009F049C6A0911807B0911907109711F4C7
:108450000C94904A80909E0490909F04A090A00459
:10846000B090A10440919A0450919B0460919C04A7
:1084700070919D0484169506A606B706D8F0109252
:108480005A0410921907109218079091B30980911D
:10849000B409981711F40C94904A8091B4098F5F35
:1084A0008F708093B40940EDC42E47E0D42EE12CA8
:1084B000F12C1AC44091960450919704609198044D
:1084C00070919904481559056A057B0508F4AAC1FD
:1084D000409192045091930460919404709195049A
:1084E000D6960D911D912D913C91D997401751072A
:1084F0006207730708F077C14115510561057105E1
:1085000049F48090560490905704A0905804B0907D
:10851000590464C1E12CF980842E952F862F0A819D
:108520001B81FD81EE813F8128859C80E091EF17C2
:10853000E89D912CFF273091F017389D900CF11D8C
:108540001090F117189CF00DE99F900CF11D399FC8
:10855000F00DE89FF00D092D1F2F099DE12D332708
:1085600022270F9FE00D311D2E1D199DE00D311D9D
:108570002E1D1F9F300D211D032F122F099DF12C41
:10858000332722270F9FF00C311D2E1D199DF00C53
:10859000311D2E1D1F9F300D211D032F122FEE2781
:1085A0008090560490915704809158040090B20432
:1085B0000E2809F483C03091AE04309FE1198E0873
:1085C0009E098E092091AF04209FE01981089E0921
:1085D0008E09F090B004F09E801891098E09319FA9
:1085E000E01981089E098E09219F801891098E0942
:1085F000F19E90198109099DF12C332722270F9FA5
:10860000F00C311D2E1D199DF00C311D2E1D1F9FCC
:10861000300D211D032F122F3091AA04309FE10D40
:108620008E1C9E1D8E1D2091AB04209FE00D811C91
:108630009E1D8E1DF090AC04F09E800C911D8E1D31
:10864000319FE00D811C9E1D8E1D219F800C911D70
:108650008E1DF19E900D811D099DF12C332722273F
:108660000F9FF00C311D2E1D199DF00C311D2E1D7C
:108670001F9F300D211D032F122F3091A604309F14
:10868000E1198E089E098E092091A704209FE01908
:1086900081089E098E09F090A804F09E8018910927
:1086A0008E09319FE01981089E098E09219F80184B
:1086B00091098E09F19E9019810982C03091AE0412
:1086C000309FE10D8E1C9E1D8E1D2091AF04209FBA
:1086D000E00D811C9E1D8E1DF090B004F09E800C5C
:1086E000911D8E1D319FE00D811C9E1D8E1D219FB1
:1086F000800C911D8E1DF19E900D811D099DF12C08
:10870000332722270F9FF00C311D2E1D199DF00CD1
:10871000311D2E1D1F9F300D211D032F122F309153
:10872000AA04309FE1198E089E098E092091AB049E
:10873000209FE01981089E098E09F090AC04F09EFC
:10874000801891098E09319FE01981089E098E09D0
:10875000219F801891098E09F19E90198109099D28
:10876000F12C332722270F9FF00C311D2E1D199D50
:10877000F00C311D2E1D1F9F300D211D032F122FB8
:108780003091A604309FE10D8E1C9E1D8E1D209100
:10879000A704209FE00D811C9E1D8E1DF090A80453
:1087A000F09E800C911D8E1D319FE00D811C9E1D41
:1087B0008E1D219F800C911D8E1DF19E900D811D9F
:1087C00011249C82F9820A831B83FD83EE833F83FD
:1087D0002887912C992AA12CB12CA82A8DE395E108
:1087E00021E0298B14C0D2968D909D90AD90BC90C5
:1087F000D597F4CFB694A79497948794D988DD0C35
:10880000D98A049625E18935920709F4EDC4FC0163
:108810000591159125913491081519052A053B05F7
:1088200048F3E2C440908B0450908C0460908D0417
:1088300070908E04481459046A047B0408F0C3C184
:1088400080918A04811121C0FD01EE5BFF4FE08021
:10885000F180028113817896208131814281538198
:10886000D2966D917D918D919C91D5970E9480C4F7
:10887000DD24D394D0928A04E0911807F09119076F
:1088800082A993A9A4A9B5A98EC14091860450914B
:1088900087046091880470918904DA960D911D9186
:1088A0002D913C91DD97401751076207730708F03F
:1088B00073C1411551056105710549F48091560454
:1088C00090915704A0915804B09159046CC1F0E004
:1088D000E985842F352F262FAA857B856C855D85BC
:1088E000BE854F859889B091EF17B89F612D5527A8
:1088F0004091F017489F600D511D1090F117189E80
:10890000500DB39F600D511D439F500DB29F500DF0
:10891000A62F752FA69FB12D44279927A59FB00D8F
:10892000411D9F1F769FB00D411D9F1F759F400DDC
:10893000911DA42F792FA69FE12D44279927A59F4C
:10894000E00D411D9F1F769FE00D411D9F1F759FEC
:10895000400D911DA42F792FBB2780915604309193
:108960005704209158040090B2040F2A09F483C0E0
:108970004091AE044A9FB1198F0B3F0B2F0B909182
:10898000AF049A9FB01981093F0B2F0BE091B004FF
:10899000EA9F801931092F0B479FB01981093F0BBE
:1089A0002F0B979F801931092F0BE79F3019210951
:1089B000A69FE12D44279927A59FE00D411D9F1FEC
:1089C000769FE00D411D9F1F759F400D911DA42FA7
:1089D000792F4091AA044A9FB10D8F1F3F1F2F1F6F
:1089E0009091AB049A9FB00D811D3F1F2F1FE09106
:1089F000AC04EA9F800D311D2F1F479FB00D811DD4
:108A00003F1F2F1F979F800D311D2F1FE79F300D98
:108A1000211DA69FE12D44279927A59FE00D411D0B
:108A20009F1F769FE00D411D9F1F759F400D911D5B
:108A3000A42F792F4091A6044A9FB1198F0B3F0BA9
:108A40002F0B9091A7049A9FB01981093F0B2F0B10
:108A5000E091A804EA9F801931092F0B479FB019B4
:108A600081093F0B2F0B979F801931092F0BE79F2F
:108A70003019210982C04091AE044A9FB10D8F1F69
:108A80003F1F2F1F9091AF049A9FB00D811D3F1F74
:108A90002F1FE091B004EA9F800D311D2F1F479FCB
:108AA000B00D811D3F1F2F1F979F800D311D2F1F60
:108AB000E79F300D211DA69FE12D44279927A59FF3
:108AC000E00D411D9F1F769FE00D411D9F1F759F6B
:108AD000400D911DA42F792F4091AA044A9FB119EE
:108AE0008F0B3F0B2F0B9091AB049A9FB01981090C
:108AF0003F0B2F0BE091AC04EA9F801931092F0B3B
:108B0000479FB01981093F0B2F0B979F801931099F
:108B10002F0BE79F30192109A69FE12D44279927A4
:108B2000A59FE00D411D9F1F769FE00D411D9F1FDA
:108B3000759F400D911DA42F792F4091A6044A9F47
:108B4000B10D8F1F3F1F2F1F9091A7049A9FB00D4B
:108B5000811D3F1F2F1FE091A804EA9F800D311D4A
:108B60002F1F479FB00D811D3F1F2F1F979F800D07
:108B7000311D2F1FE79F300D211D1124E987AA8782
:108B80007B876C875D87BE874F87988B90E0932BA0
:108B9000A0E0B0E0A22B07C0A65ABF4F8D919D91D7
:108BA0000D90BC91A02D2DE335E141E0498BF901F9
:108BB0004591559165917491481759076A077B074C
:108BC00008F49CC3AAC380918F048823E1F0FD01BF
:108BD000E85BFF4F4081518160E070E000910D0241
:108BE00010910E0220910F02309110024017510790
:108BF0006207730741F01092110210921202109254
:108C00001302109214024091090250910A026091DD
:108C10000B0270910C0277FF5FC0AE5ABF4FCD9030
:108C2000DD90ED90FC908DE395E121E0FC01459114
:108C30005591659174914C155D056E057F0550F455
:108C4000F694E794D794C794220F049675E189357A
:108C5000970761F72093910480E2C816D104E104DC
:108C6000F10428F470E2C72ED12CE12CF12C90E213
:108C7000C91AD108E108F108C114A8E0DA06E10434
:108C8000F10408F406C4B4E0DB9EC0011124835C47
:108C90009E4EFC01329625913491EC2D6627E39F80
:108CA000A001E29F410D561F0694461F561F112436
:108CB00060E070E0FC0125913491C901A0E0B0E0D2
:108CC000841B950BA60BB70B8093090290930A02A5
:108CD000A0930B02B0930C02C0900902D0900A023C
:108CE000E0900B02F0900C02809118079091190708
:108CF000892B09F0E8C10E94FFC490931907809363
:108D00001807892B09F4DFC1E0911807F0911907C2
:108D1000808183FF3EC085899689A789B08D809325
:108D2000821090938310A0938410B0938510818D4E
:108D3000928DA38DB48D8093861090938710A0930D
:108D40008810B0938910858D968DA78DB0A18093E2
:108D50008A1090938B10A0938C10B0938D1081A1EA
:108D600092A1A3A1B4A180938E1090938F10A09391
:108D70009010B09391109091B3098091B409981715
:108D800009F4B9CF8091B4098F5F8F708093B409D3
:108D9000B2CFC588D688E788F08C81E0C114D104B1
:108DA000E104F10409F480E0018D128D238D348DEE
:108DB000011511052105310509F08260458D568D9B
:108DC000678D70A1411551056105710509F0846039
:108DD00080935A041092860410928704109288049B
:108DE00010928904109292041092930410929404A9
:108DF0001092950485A196A1A7A1B0A580939A048D
:108E000090939B04A0939C04B0939D048824992480
:108E10005401881A990AAA0ABB0A80928204909285
:108E20008304A0928404B092850480927E04909280
:108E30007F04A0928004B092810480927A04909280
:108E40007B04A0927C04B0927D0480927604909280
:108E50007704A0927804B0927904CC0CDD1CEE1C4F
:108E6000FF1CC0926604D0926704E0926804F092FE
:108E70006904000F111F221F331F00936A0410930F
:108E80006B0420936C0430936D04440F551F661FD0
:108E9000771F40936E0450936F0460937004709337
:108EA000710441A152A163A174A1440F551F661F13
:108EB000771F40937204509373046093740470930B
:108EC0007504880F991FAA1FBB1F8093620490939B
:108ED0006304A0936404B093650410929E041092FE
:108EE0009F041092A0041092A10482A593A5A4A5AA
:108EF000B5A58093960490939704A0939804B0939B
:108F0000990486A597A5A0A9B1A980938B049093F5
:108F10008C04A0938D04B0938E0481A5809361048A
:108F2000DF01A95BBF4F9C9190939004992339F185
:108F300015962D913C9111973093600420935F0416
:108F400012972D913C91119730935E0420935D040C
:108F50001092110210921202109213021092140237
:108F600012972D913C91A90160E070E040930D02B1
:108F700050930E0260930F02709310020CC088246D
:108F80008A94982C540180920D0290920E02A09225
:108F90000F02B0921002EA5BFF4F908120915504BE
:108FA00092130AC02091080230E0482F082E000CCE
:108FB000550B4217530731F09093550480930802E4
:108FC0000E94D2C48091370581110E94E2BD2FEF2B
:108FD0003FEFA9012093090230930A0240930B024C
:108FE00050930C02E0911807F0911907DF01DE960B
:108FF000ED90FD900D911C9122A933A944A955A98A
:10900000EA5AFF4F60817181828193810E9480C4FE
:1090100010928A04E0911807F0911907EA5AFF4F5D
:1090200080809180A280B3808DE395E121E0FC01F6
:109030004591559165917491481559056A057B05CF
:1090400058F4B694A79497948794220F0496A9E5B0
:10905000B5E1A817B90759F720939104B0E28B1630
:109060009104A104B10428F4B0E28B2E912CA12C20
:10907000B12C30E2831A9108A108B108811448E0AC
:109080009406A104B10408F428C254E0959EC001DE
:109090001124835C9E4EFC01329625913491782DEB
:1090A0006627739FA001729F410D561F0694461FAD
:1090B000561F1124FC01C590D490E12CF12CC41A48
:1090C000D50AE108F108C092A204D092A304E0926C
:1090D000A404F092A5040091A2041091A30420918D
:1090E000A4043091A50440911102509112026091A4
:1090F000130270911402F02E198BF22FE32F4017F8
:1091000051076207730720F4F42E598BF62FE72FCF
:109110008F2D9989AF2FBE2F0097E1E0AE07B105E3
:1091200020F08FEF9FEFA0E0B0E0081B190B2A0B97
:109130003B0B0093A2041093A3042093A404309348
:10914000A5044F3FFFEF5F076F077F0761F0481BE4
:10915000590B6A0B7B0B40931102509312026093E0
:10916000130270931402F8942091840030918500CA
:10917000205F3F4F4A8941504A8B442341F0280EDB
:10918000391E2216330610F40C94613F01C01901F8
:109190003092890020928800789462960FB6F894F5
:1091A000DEBF0FBECDBFDF91CF911F910F91FF901A
:1091B000EF90DF90CF90BF90AF909F908F907F9077
:1091C0006F905F904F903F902F90089580910B018A
:1091D00080958870809309010C946D4080910B01FB
:1091E0008870809309016BC839893093910480E2BB
:1091F00088169104A104B10428F430E2832E912C46
:10920000A12CB12C30E2831A9108A108B108811475
:1092100088E09806A104B10420F1E4E09E9EC0011C
:109220001124835C9E4EFC01329625913491F82DD9
:10923000EE27F39F7001F29FE10CFE1E0694EE1ED6
:10924000FE1E1124FC01C590D490860120E030E080
:10925000480159018E189F08A108B10875016401E1
:1092600022C0950184013695279517950795F80139
:10927000EC7FCF01835C924FFC01C590D490FC0140
:10928000329625913491E82DE770E29FC001E39F6B
:10929000900D112423E0969587952A95E1F7C81A39
:1092A000D90AE12CF12C4C0D5D1D6E1D7F1D4093E4
:1092B0009204509393046093940470939504909156
:1092C000900480918F04992309F474C0882309F4D1
:1092D0000BCDA85BBF4F8D919C91A0E0B0E0409179
:1092E0000D0250910E0260910F02709110028417CE
:1092F0009507A607B70709F060C0F6CCB695A79505
:1093000097958795D988DD0CD98A2C5F3F4F49E521
:1093100055E14217530709F04ACC598950939104FB
:1093200080329105A105B10520F480E290E0A0E033
:10933000B0E08097A109B109811558E09507A10512
:10934000B10508F443C074E0979F90011124235C99
:109350003E4EF901329645915491EE27859FB0011A
:10936000849F610D7E1F06946E1F7E1F1124F901DC
:10937000C590D490E12CF12CC61AD70AE108F10867
:109380008091860490918704A0918804B09189040B
:109390008C0D9D1DAE1DBF1D809386049093870488
:1093A000A0938804B093890480919004811130C007
:1093B00080918F04882309F497CC109211021092A7
:1093C000120210921302109214028ECCAC01BD0155
:1093D0007695679557954795FA01EC7F9F01235C39
:1093E000324FF901C590D490F901329645915491CC
:1093F0008770849F9001859F300D1124F3E036958E
:109400002795FA95E1F7C21AD30AE12CF12CB8CFCF
:109410008989480E511C611C711C8091180790911C
:109420001907481459046A047B04D8F420918F0466
:10943000222309F459CCFC01E85BFF4F20813181E4
:10944000A90160E070E000910D0210910E022091E0
:109450000F0230911002401751076207730709F499
:1094600043CC109211021092120210921302109229
:109470001402FC01E85BFF4F80819181A0E0B0E025
:1094800080930D0290930E02A0930F02B0931002EE
:109490002BCCD701C601B695A79597958795FC016A
:1094A000EC7FCF01835C924FFC0125913491FC014C
:1094B0003296459154916C2D6770649FC001659FF1
:1094C000900D112463E0969587956A95E1F7281B26
:1094D000390BC901A0E0B0E0F7CBD501C401B695C6
:1094E000A79597958795FC01EC7FCF01835C924F00
:1094F000FC01C590D490FC01329625913491482D01
:109500004770429FC001439F900D1124A3E09695A0
:109510008795AA95E1F7C81AD90AE12CF12CD3CD89
:1095200080EDC82E87E0D82EE12CF12CE4CBCF9231
:10953000DF92EF92FF92CF93DF936B017C01EA0100
:1095400021E338E040EA50EC0E94C9EC87FD23C0DB
:1095500022E430E04CE553E4C701B6010E9457E62F
:109560001816CCF0C880D980EA80FB802FE632E163
:1095700043E85AEBC701B6010E94C9EC87FD0BC056
:10958000C1E022E430E04CE553E4C701B6010E949B
:1095900057E618160CF4C0E08C2FDF91CF91FF90A6
:1095A000EF90DF90CF9008950F931F93CF93DF93A9
:1095B000FC01A685B7858D0100581F4FE801888101
:1095C000998101968F779927AD014E575F4FEA0138
:1095D0002881398128173907D1F3E8012881398199
:1095E000A20FB31F6C93A685B785A058BF4F1196E5
:1095F0009C938E93A689B7892C9181E090E0078C8B
:1096000002C0880F991F0A94E2F7822B8C9381E0A5
:1096100081A30488F589E02D80818064808381E0C6
:1096200090E0DF91CF911F910F910895FC0181A1EE
:10963000882329F0A489B5898C9186FFFBCF11A2DC
:109640000895FC01A485B585FD01E058FF4F2081F8
:1096500031813296808191812817390779F0808194
:109660009181A80FB91F8C91208131812F5F3F4FCD
:109670002F7733273183208390E008958FEF9FEF7A
:109680000895DC011C96ED91FC911D97DF01A05817
:10969000BF4F2D913C91119712968D919C911197EE
:1096A0002817390739F08D919C91E80FF91F8081B7
:1096B00090E008958FEF9FEF0895FC012485358594
:1096C000F901E058FF4F80819181329620813181EC
:1096D00080589F4F821B930B60E870E00C948CEDD8
:1096E0000895089580E090E00895CF92DF92EF9280
:1096F000FF92C0903002D0903102E0903202F090A0
:109700003302FC0180819181A281B3818093300278
:1097100090933102A0933202B09333020E9476CA32
:10972000C0923002D0923102E0923202F0923302C3
:10973000FF90EF90DF90CF900895809196189091D0
:109740009718981759F0E92FF0E0EA5EF74E8081FC
:109750009F5F9F779093971890E008958FEF9FEF0A
:1097600008951F920F920FB60F9211240BB60F920D
:109770002F938F939F93EF93FF9320919718E091EE
:10978000961881E08E0F8F779091C600281729F0E8
:10979000F0E0EA5EF74E9083E82FE0939618FF9191
:1097A000EF919F918F912F910F900BBE0F900FBE55
:1097B0000F901F901895809121049091220400979A
:1097C00031F04AE050E060E070E00C94ABE360E020
:1097D00070E0CB010895EFDF97FD0AC0ECDF6F3F2B
:1097E00071058105910509F02CF4E5DF862F0895B8
:1097F00080E008958FEF08958091210490912204D4
:10980000892B31F0E8DF91E0811103C090E001C0C5
:1098100091E0892F08950F931F93CF938091210496
:1098200090912204009711F1FC018F01C1912C2F1E
:109830002F7DA9F0C53411F0C536B9F7F8011082B3
:1098400060E070E080912104909122040E9458E22F
:10985000F801C083562F472F382F292F0BC060E007
:1098600070E0CF911F910F910C9458E250E040E0CE
:1098700030E020E0652F742F832F922FCF911F911E
:109880000F91089581548A3108F042C0E82FF0E02A
:1098900040910D1850910E1860910F18709110188A
:1098A00004C076956795579547958A95D2F7842F8A
:1098B000817040FF2FC0ED50F84E9081992309F13F
:1098C000E0917210F0917310E90FF11D908120ED7D
:1098D000290F2A3098F09E3211F491810CC09D32EC
:1098E00011F09B3271F4918120ED290F2A3030F074
:1098F0009E3239F4928190539A3018F42E2F9F2F74
:1099000002C020E090E02093210490932204089567
:1099100080E008950895B6DF882341F081E020912A
:10992000210430912204232B09F480E0089580E182
:10993000E2E3F4E0AEEAB0E101900D928A95E1F73E
:1099400008952F923F924F925F926F927F928F92E3
:109950009F92AF92BF92CF92DF92EF92FF920F93BE
:109960001F93CF93DF9300D01F921F92CDB7DEB726
:109970007C018B016A0119018090320490903304BC
:10998000A0903404B0903504A5019401FC016081DD
:109990007181828193810E9457E6F1E0FD838111FC
:1099A00012C0209136043091370440913804509110
:1099B0003904F80160817181828193810E9457E6A8
:1099C000811101C01D82F601408051806280738048
:1099D0002091150230911602409117025091180201
:1099E000C301B2010E9457E6882309F453C0409294
:1099F000150250921602609217027092180220E02F
:109A000030E040E450E46091FB067091FC068091E8
:109A1000FD069091FE060E947FEB69837A838B831B
:109A20009C838092AE109092AF10A092B010B09232
:109A3000B1108091360490913704A0913804B09110
:109A400039048093B2109093B310A093B410B093E4
:109A5000B510F60180819181A281B3818093B61007
:109A60009093B710A093B810B093B91080913E04B2
:109A700090913F04A0914004B09141048093BA10AA
:109A80009093BB10A093BC10B093BD10CE01019673
:109A90002CDE4DDFFD81FF2309F16090F706709009
:109AA000F8068090F9069090FA06A090F306B09020
:109AB000F406C090F506D090F6069501A601B30114
:109AC000C4010E94C9EC181614F05301640120E08F
:109AD00030E040E251E4B501C6010CC020E030E0C6
:109AE00040EC5FE36091FF067091000780910107F1
:109AF000909102070E947FEB69837A838B839C831A
:109B000020912004222349F0AB01BC018DE595E1B1
:109B10000E9451C58AE00E94E193F7018081918102
:109B2000A281B3818093AE109093AF10A093B01038
:109B3000B093B110F80180819181A281B3818093AB
:109B4000B2109093B310A093B410B093B510F1017C
:109B500020813181428153816091BA107091BB1094
:109B60008091BC109091BD100E94A3EA6093BA103E
:109B70007093BB108093BC109093BD10CE010196E2
:109B8000B4DDD5DE0F900F900F900F900F90DF9106
:109B9000CF911F910F91FF90EF90DF90CF90BF90EA
:109BA000AF909F908F907F906F905F904F903F907D
:109BB0002F90089580E1EEEAF0E1A2E3B4E0019095
:109BC0000D928A95E1F708959C0197FD0EC08436A9
:109BD000910584F064E670E00E948CEDCB016AE0B0
:109BE00070E00E948CED805D06C0319521953109B1
:109BF0008DE201C080E280932D042A30310564F0AB
:109C0000EAE0F0E0C901BF010E948CEDCB01BF0189
:109C10000E948CED805D01C080E280932E04C9011A
:109C20006AE070E00E948CED805D80932F048DE2ED
:109C300094E008958E3691051CF02EE680E002C077
:109C4000282F892F20934404809345040C94AA76EE
:109C50002F923F924F925F926F927F928F929F923C
:109C6000AF92BF92CF92DF92EF92FF920F931F932A
:109C7000CF93DF93CDB7DEB7C455D1090FB6F894B3
:109C8000DEBF0FBECDBFECE1F8E184918F010F5F25
:109C90001F4F882321F00E94E193F801F6CF0E9424
:109CA00086B481110C940A5880E090E0A0E8BFE3EC
:109CB0008093A6109093A710A093A810B093A9101A
:109CC00080E090E0A0ECB0E48093AA109093AB10F9
:109CD000A093AC10B093AD108DEC9CECACE4BEE363
:109CE0008093A2109093A310A093A410B093A510FA
:109CF00080E090E0A8ECB1E48093240590932505E2
:109D0000A0932605B09327058CE390E0909323055C
:109D10008093220588EC90E09093210580932005A4
:109D200010921F058FE4F7DD882311F074DD04C065
:109D300060E070E080E190E46BAF7CAF8DAF9EAFF0
:109D400083E4E9DD882311F057DD02C083E49ADD66
:109D500061968FAF61978BE4DEDD882311F04CDDD7
:109D600002C08BE48FDD60968FAF609782E4D3DD15
:109D70008823E9F050DD0E94E7EB709323056093A0
:109D800022056115710599F06852710965367105F2
:109D900070F0E7EEF7E184918F010F5F1F4F88238A
:109DA00011F40C940A580E94E193F801F4CF8CE46A
:109DB000B2DD882351F12FDD6B017C016093A2108D
:109DC0007093A3108093A4109093A51020E030E02E
:109DD000A9010E94C9EC87FD0AC020E030E040E004
:109DE00050E4C701B6010E9457E6181674F4EFEB71
:109DF000F7E184918F010F5F1F4F882311F40C94BA
:109E00000A580E94E193F801F4CF81E53BDD8823F5
:109E100009F440C08091210490912204892B19F407
:109E2000E4E9F7E12BC0F7DC6B017C016093AA1039
:109E30007093AB108093AC109093AD102DEC3CEC74
:109E40004CE45DE30E94C9EC87FD0AC020E030E0ED
:109E500040E751E4C701B6010E9457E61816D4F452
:109E6000E3E6F7E184918F010F5F1F4F882311F420
:109E70000C940A580E94E193F801F4CF84918F0169
:109E80000F5F1F4F882311F40C940A580E94E1932E
:109E9000F801F4CF83E53FDD882319F1BCDC4B01E9
:109EA0005C012DEC3CEC4CEC5DE30E94C9EC87FDC1
:109EB0000AC020E030E040E85FE3C501B4010E9441
:109EC00057E61816ACF4ECE3F7E184918F010F5FCD
:109ED0001F4F882311F40C940A580E94E193F80153
:109EE000F4CF5DEC852E5CEC952EA92C5EE3B52EAF
:109EF00080E5C8DC882309F443C080912104909157
:109F00002204892B71F4E4E0F7E184918F010F5F63
:109F10001F4F882311F40C940A580E94E193F80112
:109F2000F4CF80911F058F5F80931F0574DC6B0158
:109F30007C016093240570932505809326059093FA
:109F4000270520E030E0A9010E94C9EC87FD0AC086
:109F500020E030E048EC51E4C701B6010E9457E62A
:109F6000181674F4ECEDF6E184918F010F5F1F4F2A
:109F7000882311F40C940A580E94E193F801F4CF5D
:109F800086E4C9DC882319F146DC6B017C0120E002
:109F900030E040E85FE30E94C9EC87FD0AC020E0A2
:109FA00030E040E850E4C701B6010E9457E61816B9
:109FB000A4F4E3EBF6E184918F010F5F1F4F882338
:109FC00011F40C940A580E94E193F801F4CFC12CCB
:109FD000D12C40EEE42E4FE3F42EA7019601C701E9
:109FE000B6010E94BCE69B01AC0160E070E084E435
:109FF00090E40E947FEB2091A6103091A710409131
:10A00000A8105091A9100E94BCE62B013C01A501AB
:10A010009401C501B4010E94BCE6A70196010E940B
:10A02000BCE62CEE31E548EB5DE30E947FEB9B0143
:10A03000AC01C301B2010E94BCE66093A61070930C
:10A04000A7108093A8109093A91088E464DC88235B
:10A05000C9F0E1DB0E94E7EB7093210560932005D6
:10A06000655A71096437710568F0E5E8F6E1849195
:10A070008F010F5F1F4F882309F4CCC70E94E19323
:10A08000F801F5CF85E5FEDB8823E9F00E94F25860
:10A09000611571058105910511F00E944FE28091D3
:10A0A000210490912204892B11F0B5DB04C060E0FB
:10A0B00070E088E492E460931B0570931C05809324
:10A0C0001D0590931E0582E5DDDB81110DC0E1E5E4
:10A0D000F6E184918F010F5F1F4F882309F49AC71F
:10A0E0000E94E193F801F5CF809121049091220420
:10A0F000892BA9F060DB2F967FAF6EAF2F971616D6
:10A1000017069CF0EDE1F6E184918F010F5F1F4F80
:10A11000882309F47FC70E94E193F801F5CF8AE113
:10A1200090E02F969FAF8EAF2F9788E5F4DB8823C2
:10A1300061F071DB209114043091150440911604F4
:10A14000509117040E94A2EA08C0609132047091F5
:10A150003304809134049091350460931705709313
:10A1600018058093190590931A0589E5D4DB882397
:10A1700061F051DB209118043091190440911A04C8
:10A1800050911B040E94A2EA08C0609136047091AD
:10A1900037048091380490913904609313057093CB
:10A1A000140580931505909316056091170570911D
:10A1B00018058091190590911A0543E155E0B7D92A
:10A1C00081110DC0E3EFF5E184918F010F5F1F4F07
:10A1D000882309F41FC70E94E193F801F5CF84E4B6
:10A1E00051DB91E089270E9449AC20E030E040EA51
:10A1F00050E460913A0470913B0480913C0490914A
:10A200003D040E9457E687FF14C0198A1A8A1B8AE8
:10A210001C8A80E090E0A0EAB0E489839A83AB8353
:10A22000BC83BE016F5E7F4FCE0101960E9468B471
:10A23000C1DCD8D76B017C01A8E8CA0EA3E1DA1E05
:10A24000E11CF11C8091220590912305F3DC6091C3
:10A25000220570912305072E000C880B990B0E9494
:10A260005DE69B01AC0160914604709147048091CA
:10A270004804909149040E94A2EA4B015C0120E04D
:10A2800030E0A9010E94C9EC87FF04C0B7FAB0947E
:10A29000B7F8B09420E030E040E450E4C501B401E8
:10A2A0000E94C9EC1816F4F49DD7DC01CB018C197F
:10A2B0009D09AE09BF09B7FD0EC094D76B017C01A3
:10A2C000B8E8CB0EB3E1DB1EE11CF11C0E94F07577
:10A2D0008AE00E94E1930E941FA1809196188093CA
:10A2E0009718B5CF80912005909121050E94E759DC
:10A2F0006091200570912105072E000C880B990BA9
:10A300000E945DE69B01AC0160914C0470914D048C
:10A3100080914E0490914F040E94A2EA4B015C018F
:10A3200020E030E0A9010E94C9EC87FF04C0B7FA21
:10A33000B094B7F8B09420E030E040E450E4C501B8
:10A34000B4010E94C9EC1816F4F44CD7DC01CB011F
:10A350008C199D09AE09BF09B7FD0EC043D76B012B
:10A360007C01E8E8CE0EE3E1DE1EE11CF11C0E9458
:10A37000F0758AE00E94E1930E941FA180919618D7
:10A3800080939718B5CF10923E0410923F0410921C
:10A390004004109241040E9437B380911F05882326
:10A3A00099F1C5DA209124053091250540912605C3
:10A3B000509127056091BA107091BB108091BC102C
:10A3C0009091BD100E94A3EA6093BA107093BB10E5
:10A3D0008093BC109093BD1020E030E040E751E442
:10A3E0006091FF067091000780910107909102072C
:10A3F0000E947FEB69837A838B839C83CE010196D5
:10A4000074D995DA0E9444B180E2E3EFF4E0DF0111
:10A41000282F1D922A95E9F7E3EDF4E0DF01282FBC
:10A420001D922A95E9F7E3EBF4E0DF011D928A958E
:10A43000E9F77DDA8091A2109091A310A091A41069
:10A44000B091A5108093B6109093B710A093B81058
:10A45000B093B91019821A821B821C829E012F5F51
:10A460003F4F46EB50E162EB70E18EEA90E169DA32
:10A470009E01255C3F4F46EB50E162EB70E18EEAB6
:10A4800090E15FDA6196BFAD6197BB2329F066E387
:10A4900074E082E394E004C063E175E087E195E055
:10A4A0000E94A7D8298F3A8F4B8F5C8F6D8F7E8F3C
:10A4B0003FAF2D962FAF2D972D96EFAD2D97E7FD42
:10A4C00081C4FFADF7FD7EC424E0E202F001112457
:10A4D000E350F64F40805180628073803FAD84E04E
:10A4E0003802F0011124E751F64FD080C18032804C
:10A4F00023808D2D9C2DA32DB22D8FAB98AFA9AFAE
:10A50000BAAFAE01495C5F4FB201C30110D88823D6
:10A5100009F45CC420E030E040EA50E4B201C30139
:10A520000E94A3EAF62E072F182FE92E862F902FD0
:10A53000A12FBE2D8BAB9CABADABBEAB8D2D9C2D9F
:10A54000A32DB22D8FA798ABA9ABBAAB2D969FAD1B
:10A550002D97911152C0AFADA11105C05F2D402FB5
:10A56000312F2E2D04C0542D452D362D272D852F0E
:10A57000942FA32FB22F8BAB9CABADABBEABBFADBB
:10A58000B43034F4F42C052D162DE72CBB2369F0E0
:10A5900020E030E040EA50E46D2D7C2D832D922D9B
:10A5A0000E94A2EA362F272F03C09601832D922DF9
:10A5B000432F522FBC014FA758AB69AB7AABEFAD1D
:10A5C000E4300CF0A7C020E030E040EA50E46D2D0C
:10A5D0007C2D832D922D0E94A3EA21966FAF2197A7
:10A5E00023967FAF239725968FAF259727969FAF0A
:10A5F0002797FFADF11185C099C02D962FAD2D97EE
:10A6000024300CF453C03FAD34305CF020E030E037
:10A6100040EA50E4B201C3010E94A2EA362F272F7C
:10A6200003C0342D252DC301432F522FBC014BAB4A
:10A630005CAB6DAB7EAB8FAD8111E3C420E030E04D
:10A6400040EA50E4B201C3010E94A2EAF62E072FAD
:10A65000182FE92E20E030E040EA50E46D2D7C2DEB
:10A66000832D922D0E94A3EA6FA778AB89AB9AAB9A
:10A670009FAD992309F44EC020E030E040EA50E459
:10A680006D2D7C2D832D922D0E94A2EA21966FAF15
:10A69000219723967FAF239725968FAF25972796EF
:10A6A0009FAF2797AFADA43064F140C0BFADB111EB
:10A6B0000DC020E030E040EA50E4B201C3010E9446
:10A6C000A2EAF62E072F182FE92E0FC0EFADE430C7
:10A6D000B4F120E030E040EA50E4B201C3010E944E
:10A6E000A2EA6BAB7CAB8DAB9EAB2196DFAE219724
:10A6F0002396CFAE239725963FAE259727962FAE6C
:10A70000279732ED832E33E5932E3BE7A32E31E4DA
:10A71000B32E29C02196DFAE21972396CFAE239783
:10A7200025963FAE259727962FAE279722ED822EAE
:10A7300023E5922E2BEFA22E20E4B22E14C02196F8
:10A74000DFAE21972396CFAE239725963FAE259770
:10A7500027962FAE279792ED892E93E5992E9BEFA2
:10A76000A92E91E4B92E8BA99CA9ADA9BEA92C96BE
:10A770008CAF9DAFAEAFBFAF2C979C01AD01B201C6
:10A78000C3010E94A2EA698B7A8B8B8B9C8B4FA4AE
:10A7900058A869A87AA8A30192016D2D7C2D832D5C
:10A7A000922D0E94A2EA6D8B7E8B8F8B988F2C96B8
:10A7B0002CAD3DAD4EAD5FAD2C97609132047091E4
:10A7C000330480913404909135040E94A2EA2C96BF
:10A7D0006CAF7DAF8EAF9FAF2C97A30192016091BC
:10A7E00036047091370480913804909139040E94A6
:10A7F000A2EA2B013C018F2D902FA12FBE2D898322
:10A800009A83AB83BC8321968FAD219723969FAD0E
:10A8100023972596AFAD25972796BFAD27978D83B4
:10A820009E83AF83B8878091A2109091A310A091CE
:10A83000A410B091A51089879A87AB87BC872DECAF
:10A840003CEC4CEC5CE3C501B4010E94BCE62091F9
:10A85000A6103091A7104091A8105091A9100E9405
:10A86000BCE620913E0430913F0440914004509159
:10A8700041040E94A3EA6D877E878F87988B2C9670
:10A880002CAD3DAD4EAD5FAD2C97CA01B9010E9414
:10A89000BCE66B017C01A3019201C301B2010E94DD
:10A8A000BCE69B01AC01C701B6010E94A3EA20E00F
:10A8B00030E040E050E40E94C9EC18160CF046C0AD
:10A8C0000E9444B11BA21CA21DA21EA220E030E0E7
:10A8D00040E05FE360913A0470913B0480913C0456
:10A8E00090913D040E94A3EA6F8F78A389A39AA355
:10A8F0009E012D5D3F4FAE01415E5F4F66E374E008
:10A9000082E394E01ED81BA21CA21DA21EA220E07E
:10A9100030E040E05FE36091A2107091A31080915D
:10A92000A4109091A5100E94A3EA6F8F78A389A329
:10A930009AA39E012D5D3F4FAE01415E5F4FBE0168
:10A94000615D7F4FCE01C3960E94A14C1F8E18A25D
:10A9500019A21AA29E01215E3F4F42EA50E1BE01B8
:10A96000615D7F4FCE01C3960E94A14C0E9470B1E1
:10A970004090300250903102609032027090330269
:10A98000E090F706F090F8060091F9061091FA06AB
:10A99000A090F306B090F406C090F506D090F606AD
:10A9A0009501A601B701C8010E94C9EC181614F45C
:10A9B0007501860120E030E040E251E4B701C801B2
:10A9C0000E947FEB609330027093310280933202D9
:10A9D0009093330240E0BE016F5E7F4FCE0101963F
:10A9E0000E94EBA4409230025092310260923202F7
:10A9F000709233020E94974CADEFB9E02496BFAF3E
:10AA0000AEAF249722961FAE1EAE229701E010E053
:10AA100021960FAC219702C0000F111F0A94E2F794
:10AA20002296EEADFFAD229731962296FFAFEEAFA4
:10AA3000229721E030E021960FAC219702C0220F2F
:10AA4000331F0A94E2F763963FAF2EAF639783EB11
:10AA5000282E84E0382E83EF94E02A969FAF8EAFA5
:10AA60002A97A3EDB4E02896BFAFAEAF2897E9EEE2
:10AA7000F9E02696FFAFEEAF26972A962EAD3FADB2
:10AA80002A9765963FAF2EAF6597D9018D919C911E
:10AA90009C0120233123232B09F4ADC06396EEAD36
:10AAA000FFAD63978E239F23892B09F4A4C02896BA
:10AAB000AEADBFAD28978D919C9180239123892BBA
:10AAC00009F099C020E030E040E050E42496AEADBB
:10AAD000BFAD24976D917D918D919C910E94A3EAC9
:10AAE0006B017C0120E030E040E050E42496EEADC4
:10AAF000FFAD249764817581868197810E94A2EAC7
:10AB00004B015C0120E030E040E850ECC701B601A9
:10AB10000E9457E687FD70C120E030E04BE553E42A
:10AB2000C701B6010E94C9EC181634F4C12CD12C0F
:10AB3000BBE5EB2EB3E4FB2ECBA6DCA6EDA6FEA672
:10AB40002696AEADBFAD26974D905D906D907C90F2
:10AB500020E030E040E85FE3C301B2010E9457E625
:10AB600087FD51C120E030E04BE553E4C301B20161
:10AB70000E94C9EC181634F4412C512CFBE56F2EC1
:10AB8000F3E47F2E4F8E58A269A27AA24FA258A654
:10AB900069A67AA620E030E040E850ECC501B40197
:10ABA0000E9457E687FD36C120E030E04BE553E4D4
:10ABB000C501B4010E94C9EC181634F4812C912C03
:10ABC0007BE5A72E73E4B72E8BA29CA2ADA2BEA2FA
:10ABD000AE01495D5F4FC701B6010E94974A8111DE
:10ABE00020C12896EEADFFAD289780819181802B02
:10ABF000912B918380832A962EAD3FAD2A972E5FAD
:10AC00003F4F2A963FAF2EAF2A976596AEADBFADA8
:10AC100065978D919C9180239123892B09F4A6C07F
:10AC2000F9018081918180239123892B09F49EC0B1
:10AC3000F1018081918180239123892B09F096C0B5
:10AC400020E030E040E050E42696AEADBFAD269760
:10AC50006D917D918D919C910E94A3EA2B013C0105
:10AC600020E030E040E050E42696EEADFFAD2697C0
:10AC700064817581868197810E94A2EA4B015C0103
:10AC80002496AEADBFAD2497CD90DD90ED90FC90B5
:10AC900020E030E040E850ECC701B6010E9457E6E2
:10ACA00087FDFFC020E030E04BE553E4C701B6016B
:10ACB0000E94C9EC181634F4C12CD12C5BE5E52EAA
:10ACC00053E4F52ECBA2DCA2EDA2FEA2CBA6DCA61D
:10ACD000EDA6FEA620E030E040E85FE3C301B2014C
:10ACE0000E9457E687FDE4C020E030E04BE553E4E6
:10ACF000C301B2010E94C9EC181634F4412C512C46
:10AD00003BE5632E33E4732E4FA258A669A67AA6BC
:10AD100020E030E040E85FE3C501B4010E9457E65F
:10AD200087FDCDC020E030E04BE553E4C501B40120
:10AD30000E94C9EC181634F4812C912C9BE5A92EA5
:10AD400093E4B92E8F8E98A2A9A2BAA2AE01495D52
:10AD50005F4FC701B6010E94974A8111B7C0F10148
:10AD600080819181802B912B91838083F2E02F0E43
:10AD7000311C28962EAD3FAD28972E5F3F4F289669
:10AD80003FAF2EAF289726968EAD9FAD269704969F
:10AD900026969FAF8EAF26979DEB291694E0390635
:10ADA00009F06BCE2496AEADBFAD249714962496D1
:10ADB000BFAFAEAF24972296EEADFFAD2297359789
:10ADC00009F024CE80919618809397182F962EAD77
:10ADD0003FAD2F97215031092F963FAF2EAF2F97C0
:10ADE000232B09F4B3C02D963FAD2D9737FDAEC090
:10ADF0008FAD87FF47CBAAC0C12CD12CA0E8EA2E8B
:10AE0000A0ECFA2E99CE412C512CE0E86E2EEFE307
:10AE10007E2EB8CE812C912C60E8A62E60ECB62E4A
:10AE2000D3CEAE01415E5F4FC501B4010E94974A87
:10AE3000882309F4D6CE80912004882321F1B7011C
:10AE4000A6018DEC95E10E9451C54FA158A569A5B9
:10AE50007AA587EC95E10E9451C54BA15CA16DA13B
:10AE60007EA18DEB95E10E9451C54F8D58A169A13E
:10AE70007AA187EB95E10E9451C589E20E94E19396
:10AE80008AE00E94E1939E01215E3F4FAE014D5D3D
:10AE90005F4FBE01695D7F4FCE018B960E94A0B1CE
:10AEA000A0CEC12CD12C40E8E42E40ECF42E0ACFE9
:10AEB000412C512C20E8622E2FE3722E25CF812CBD
:10AEC000912C80E8A82E8FE3B82E3CCFAE01415ED6
:10AED0005F4FC701B6010E94974A882309F43FCF0C
:10AEE00080912004882321F1B701A60183E995E12F
:10AEF0000E9451C54FA158A569A57AA58DE895E195
:10AF00000E9451C54BA15CA16DA17EA183E895E192
:10AF10000E9451C54F8D58A169A17AA18DE795E195
:10AF20000E9451C589E20E94E1938AE00E94E19368
:10AF30009E01215E3F4FAE014D5D5F4FBE01695DD9
:10AF40007F4FCE018B960E94A0B109CF0E9444B1E1
:10AF500080E090E0A0EAB0E48093B6109093B71040
:10AF6000A093B810B093B91019821A821B821C8268
:10AF70009E012F5F3F4F46EB50E162EB70E18EEA9E
:10AF800090E10E94A14C8091170590911805A09125
:10AF90001905B0911A058093AE109093AF10A0934D
:10AFA000B010B093B1108091130590911405A09149
:10AFB0001505B09116058093B2109093B310A0932D
:10AFC000B410B093B51019821A821B821C829E01A4
:10AFD0002F5F3F4F46EB50E162EB70E18EEA90E16C
:10AFE0000E94A14C6096FFAD6097F11113C01092C2
:10AFF0004504109244040E94AA7680E090E0E7D1D4
:10B0000009C02FADF42C052D162DE72C24300CF0A3
:10B0100033CB20CBCC5ADF4F0FB6F894DEBF0FBE38
:10B02000CDBFDF91CF911F910F91FF90EF90DF90F7
:10B03000CF90BF90AF909F908F907F906F905F90D8
:10B040004F903F902F9008951F920F920FB60F923E
:10B0500011240BB60F922F933F938F939F93EF93EF
:10B06000FF932091120F3091130F8091140F909144
:10B07000150F2817390731F4809131018F7D8093A6
:10B08000310114C0E091140FF091150FEE56F14FFD
:10B0900020818091140F9091150F01968F77992739
:10B0A0009093150F8093140F20933601FF91EF9129
:10B0B0009F918F913F912F910F900BBE0F900FBEDC
:10B0C0000F901F9018951F920F920FB60F92112498
:10B0D0000BB60F922F934F935F938F939F93EF93A2
:10B0E000FF938091300182FD1CC020913601809138
:10B0F000960F9091970F4091980F5091990F01964C
:10B100008F7799274817590771F0E091960FF091C2
:10B11000970FEA5EF04F20839093970F8093960FDE
:10B1200002C080913601FF91EF919F918F915F91C5
:10B130004F912F910F900BBE0F900FBE0F901F904D
:10B140001895CF92DF92EF92FF920F931F93CF93B8
:10B15000DF936C017A018B01C0E0D0E0CE15DF05F2
:10B1600081F0D8016D918D01D601ED91FC91019096
:10B17000F081E02DC6011995892B11F02196EECFB3
:10B180007E01C701DF91CF911F910F91FF90EF904A
:10B19000DF90CF9008950E94B3ED3FB7F89480916F
:10B1A000CF069091D006A091D106B091D20626B5D7
:10B1B000A89B05C02F3F19F00196A11DB11D3FBFEF
:10B1C000BA2FA92F982F8827820F911DA11DB11D7D
:10B1D000BC01CD0142E0660F771F881F991F4A9579
:10B1E000D1F708952FB7F8946091CB067091CC06F3
:10B1F0008091CD069091CE062FBF08951F920F9299
:10B200000FB60F9211242F933F938F939F93AF9379
:10B21000BF938091CB069091CC06A091CD06B091C2
:10B22000CE063091CA0623E0230F2D3720F4019675
:10B23000A11DB11D05C026E8230F0296A11DB11D59
:10B240002093CA068093CB069093CC06A093CD069C
:10B25000B093CE068091CF069091D006A091D106F2
:10B26000B091D2060196A11DB11D8093CF06909397
:10B27000D006A093D106B093D206BF91AF919F9113
:10B280008F913F912F910F900FBE0F901F901895A7
:10B290001F920F920FB60F9211240BB60F922F939D
:10B2A0003F934F935F936F937F938F939F93AF934E
:10B2B000BF93EF93FF9380912B0590912C05A09164
:10B2C0002D05B0912E05892B8A2B8B2B59F190914E
:10B2D0002A05E0912805F09129058081892780833E
:10B2E00080912B0590912C05A0912D05B0912E05F4
:10B2F000181619061A061B060CF056C080912B056D
:10B3000090912C05A0912D05B0912E050197A109D2
:10B31000B10980932B0590932C05A0932D05B09334
:10B320002E0542C080911902E9E4F8E1E4919FEF13
:10B3300090931902E230C9F050F4EE2399F0E13015
:10B3400081F590916F009D7F90936F002AC0E4304B
:10B3500019F1E0F0E53029F5909173009D7F90930D
:10B3600073001FC010926E001CC0909170009D7FF2
:10B370009093700091E09093B0009091B100987F0D
:10B3800094609093B1001092B3000BC09091710043
:10B390009D7F9093710005C0909172009D7F909366
:10B3A000720060E00E94FCB5FF91EF91BF91AF91F8
:10B3B0009F918F917F916F915F914F913F912F91CD
:10B3C0000F900BBE0F900FBE0F901F90189590938B
:10B3D0004B0480934A0480E00C94F6762F923F92BF
:10B3E0004F925F926F927F928F929F92AF92BF9295
:10B3F000CF92DF92EF92FF920F931F93CF93DF9341
:10B40000CDB7DEB7C857D1090FB6F894DEBF0FBE6F
:10B41000CDBFE0914A07F0914B07EF2B11F00C9450
:10B42000AE622896DFAECEAE28976E2C79016A0107
:10B430005B01FC0120813181428153816C962CAFEC
:10B440003DAF4EAF5FAF6C9720919210309193104B
:10B4500040919410509195106C966CAD7DAD8EAD71
:10B460009FAD6C970E94BCE60E94D4ECE0966CAF56
:10B470007DAF8EAF9FAFE097D5018D919D910D90DF
:10B48000BC91A02DA0968CAF9DAFAEAFBFAFA097E3
:10B4900020919610309197104091981050919910EA
:10B4A000BC01CD010E94BCE60E94D4ECE4966CAFD6
:10B4B0007DAF8EAF9FAFE497D6012D913D914D9119
:10B4C0005C91A4962CAF3DAF4EAF5FAFA497209197
:10B4D0009A1030919B1040919C1050919D10A49611
:10B4E0006CAD7DAD8EAD9FADA4970E94BCE60E9471
:10B4F000D4ECE8966CAF7DAF8EAF9FAFE897D701E5
:10B500002D913D914D915C9122962CAF3DAF4EAF68
:10B510005FAF229720919E1030919F104091A01014
:10B520005091A11022966CAD7DAD8EAD9FAD22974E
:10B530000E94BCE60E94D4EC60966CAF7DAF8EAFEB
:10B540009FAF60978091100783FF1CC060962CAD61
:10B550003DAD4EAD5FAD60972093E5093093E609B0
:10B560004093E7095093E80922968CAD9DADAEADAE
:10B57000BFAD22978093D5099093D609A093D709A0
:10B58000B093D809D801BC91B9A7F801F181F9AB02
:10B59000D8011296BC91BEABF801F381FAAF80914D
:10B5A000B3099091B409891B8F708F3019F40E94F0
:10B5B0001FA1F5CF0091B309E9960FAFE9978091EC
:10B5C000B309082F10E01CA30BA38091D909909117
:10B5D000DA09A091DB09B091DC09E0968CAC9DAC56
:10B5E000AEACBFACE097881A990AAA0ABB0A809150
:10B5F000DD099091DE09A091DF09B091E009E496A0
:10B600002CAC3DAC4EAC5FACE497281A390A4A0A20
:10B610005B0A8091E1099091E209A091E309B09160
:10B62000E409E8962CAD3DAD4EAD5FADE897281B23
:10B63000390B4A0B5B0B2DA33EA34FA358A7809158
:10B64000E5099091E609A091E709B091E8096096B3
:10B650000CAD1DAD2EAD3FAD6097081B190B2A0B2D
:10B660003B0B0DA71EA72FA738AB012B022B032BDB
:10B6700009F4BCC080910F0781114BC060914C044C
:10B6800070914D0480914E0490914F040E94E7EB1D
:10B690002091250230912602621773070CF039C001
:10B6A00060962CAD3DAD4EAD5FAD60972093E50942
:10B6B0003093E6094093E7095093E80922968CAD50
:10B6C0009DADAEADBFAD22978093D5099093D609BD
:10B6D000A093D709B093D809E6EEFDE184918F01DC
:10B6E0000F5F1F4F811103C0EDEBF9E104C00E9411
:10B6F000E193F801F3CF84918F010F5F1F4F8823EF
:10B7000021F00E94E193F801F6CF1DA61EA61FA608
:10B7100018AA94E0699E800111240F5D1D4F6DA54C
:10B720007EA58FA598A90E945DE6D8012D913D9137
:10B730004D915C910E94BCE66B017C0120E030E001
:10B74000A9010E94C9EC87FF04C0F7FAF094F7F84A
:10B75000F09460919E1070919F108091A010909134
:10B76000A1100E94E7EB9B01AC01A8ECB0E00E94A5
:10B7700083EA0E945DE6A70196010E9457E687FFD3
:10B7800039C060960CAD1DAD2EAD3FAD60970093F6
:10B79000E5091093E6092093E7093093E80922961A
:10B7A0002CAD3DAD4EAD5FAD22972093D5093093C2
:10B7B000D6094093D7095093D809E6EEFDE184916C
:10B7C0008F010F5F1F4F811103C0EEE9F9E104C043
:10B7D0000E94E193F801F3CF84918F010F5F1F4F17
:10B7E000882321F00E94E193F801F6CF1DA61EA642
:10B7F0001FA618AAD501C4018827B7FD83959927EC
:10B80000AA27BB27782E57FE03C0382F3260732E2D
:10B810008DA19EA1AFA1B8A5B7FF03C0972D9460DD
:10B82000792E0DA51EA52FA538A937FF03C0172D0A
:10B830001860712E24E0629E800111240F5D1D4F5F
:10B840006DA57EA58FA598A90E945DE6D8012D91D2
:10B850003D914D915C910E94BCE66B017C0120E022
:10B8600030E0A9010E94C9EC87FF04C0C701B601FE
:10B87000905802C0C701B60120E030E040E05FE32D
:10B880000E94A3EA0E94ECEB6AAB7BAB8CAB9DAB56
:10B8900088E60BA11CA1809FF001819FF00D11246F
:10B8A000E159FE4E1082EA5BFF4F7082B501A401A0
:10B8B000B7FE07C044275527BA01481959096A0934
:10B8C0007B0988E60BA11CA1809FF001819FF00DF0
:10B8D0001124E159FE4E458B568B678B708F2C9649
:10B8E0002CAE3DAE4EAE5FAE2C9757FE0DC08827F6
:10B8F0009927DC0182199309A409B5092C968CAF0C
:10B900009DAFAEAFBFAF2C9728E60BA11CA1209F27
:10B91000F001219FF00D1124E159FE4E2C968CADC3
:10B920009DADAEADBFAD2C97818F928FA38FB48F9D
:10B930000DA11EA12FA138A537FF07C03095209576
:10B94000109501951F4F2F4F3F4FE8E67E2EABA17C
:10B95000BCA17A9EF0017B9EF00D1124E159FE4EB0
:10B96000058F168F278F30A38AA99BA9ACA9BDA9E3
:10B9700081A392A3A3A3B4A323964FAF2397752EBD
:10B98000F62FE72F2C968CAD9DADAEADBFAD2C97AD
:10B99000481759076A077B0778F429969FAD2997BE
:10B9A00023969FAF23972A967FAC2A972B96FFADBD
:10B9B0002B972C96EFAD2C9723968FAD2397972D31
:10B9C000AF2FBE2F80179107A207B30710F4D9013C
:10B9D000C8010AA91BA92CA93DA980179107A20794
:10B9E000B30710F4D901C80128E60BA11CA1209FC0
:10B9F000F001219FF00D1124E159FE4E85A396A37D
:10BA0000A7A3B0A70697A105B10508F4A0C5DF015B
:10BA1000AE59BF4F80914204909143048D939C9303
:10BA200061A6452B462B472B09F05F9888E60BA1B2
:10BA30001CA1809FF001819FF00D1124E159FE4E61
:10BA4000818D928DA38DB48D892B8A2B8B2B11F038
:10BA50008A98479888E60BA11CA1809FF001819FDE
:10BA6000F00D1124E159FE4E858D968DA78DB0A164
:10BA7000892B8A2B8B2B31F0809108018170809368
:10BA8000060147982AA93BA94CA95DA9232B242B81
:10BA9000252B09F465C580911507882319F081507D
:10BAA00080931507611004C0129880E280931507F7
:10BAB00060900B0770900C0700910D0710910E0716
:10BAC0009301A80169A579A98EA99AAD0E9457E6AC
:10BAD00087FF04C069A679AA0EAB1AAFC501B401ED
:10BAE0000E945DE620915F113091601140916111DB
:10BAF000509162110E94BCE626966CAF7DAF8EAF6E
:10BB00009FAF2697698B7A8B8B8B9C8BC201B1017F
:10BB10000E945DE62091631130916411409165119E
:10BB2000509166110E94BCE62B013C016D8B7E8B0F
:10BB30008F8B988F6DA17EA18FA198A50E945DE645
:10BB400020916711309168114091691150916A11EB
:10BB50000E94BCE64B015C01698F7A8F8B8F9C8FB2
:10BB600020916B1130916C1140916D1150916E11BB
:10BB7000C701B6010E94BCE66B017C016D8F7E8F10
:10BB80008F8F98A388E60BA11CA1809FF001819F55
:10BB9000F00D1124E159FE4E258936894789508DD3
:10BBA0002DA33EA34FA358A72630310541055105CB
:10BBB00008F4DFC42896AEADBFAD2897CD90DD90D8
:10BBC000ED90FC9020E030E0A901C701B6010E9491
:10BBD00057E68111EDC426962CAD3DAD4EAD5FAD5F
:10BBE0002697CA01B9010E94BCE66B017C01A30142
:10BBF0009201C301B2010E94BCE69B01AC01C701E6
:10BC0000B6010E94A3EA6B017C01A5019401C50164
:10BC1000B4010E94BCE69B01AC01C701B6010E94C1
:10BC2000A3EA0E940EED28E60BA11CA1209FF001C3
:10BC3000219FF00D1124E159FE4E65877687878795
:10BC4000908B88E60BA11CA1809FF001819FF00DD5
:10BC50001124E159FE4E4584568467847088A301FF
:10BC6000920160E070E080E89FE30E947FEB6496C1
:10BC70006CAF7DAF8EAF9FAF649729A539A94EA950
:10BC80005AAD0E94BCE64B015C018091B3099091D2
:10BC9000B109891B8F7027968FAF2797A501940153
:10BCA00060E074E284E799E40E947FEB0E94D4ECA8
:10BCB0006B017C0127968FAD27978250863008F460
:10BCC00086C4A5019401C301B2010E94BCE69B0198
:10BCD000AC010E94BCE668966CAF7DAF8EAF9FAFA3
:10BCE000689788E6ABA1BCA18A9F80018B9F100D4D
:10BCF000112401591E4E68962CAD3DAD4EAD5FAD81
:10BD00006897D80111962D933D934D935C931497AA
:10BD100095962D913D914D915C9198972EAB3FABAF
:10BD200048AF59AFCA01B9010E945BE66AAF7BAF69
:10BD30008CAF9DAF9B01AC01C501B4010E94BCE674
:10BD40000E9469EB0E94ECEBA8966CAF7DAF8EAFC2
:10BD50009FAFA897F801EE5AFF4F608371838283EB
:10BD600093838E010F5E1F4F2A961FAF0EAF2A9747
:10BD70000051110924961FAF0EAF249703EF16E070
:10BD8000AC961FAF0EAFAC978E010F5D1F4F1AA37D
:10BD900009A324960EAD1FAD2497AA961FAF0EAF30
:10BDA000AA97312C212C10E819A70FE309AB2A968A
:10BDB000AEADBFAD2A972D913D914D915D912A96E3
:10BDC000BFAFAEAF2A97C501B4010E94BCE66B01BC
:10BDD0007C01AA96EEADFFADAA9761937193819312
:10BDE0009193AA96FFAFEEAFAA9720E030E0A901A9
:10BDF0000E94C9EC87FF04C0F7FAF094F7F8F094BA
:10BE0000AC96AEADBFADAC974D905D906D907D9012
:10BE1000AC96BFAFAEAFAC97A7019601C301B2011C
:10BE20000E9457E687FD0DC409A11AA12A962EADDE
:10BE30003FAD2A970217130709F0B9CF20E030E091
:10BE400040E85FE3632D722D89A599A90E9457E60A
:10BE500087FF58C07E0131E1E30EF11C24960EAD40
:10BE60001FAD2497232D322D49A559A9D8016D91D5
:10BE70007D918D919C910E94BCE6F8016193719334
:10BE8000819391938F01EE16FF0661F728E60BA1CF
:10BE90001CA1209FC001219F900D11249C012159BC
:10BEA0003E4E790189010E5A1F4FA8966CAD7DADAB
:10BEB0008EAD9FADA8970E945BE6232D322D49A53C
:10BEC00059A90E94BCE60E94ECEBD8016D937D93CA
:10BED0008D939C931397232D322D49A559A9632D3A
:10BEE000722D89A599A90E94BCE668962CAD3DAD3E
:10BEF0004EAD5FAD68970E94BCE6F7016183728327
:10BF0000838394832AAD3BAD4CAD5DAD64966CAD3F
:10BF10007DAD8EAD9FAD64970E94BCE669A77AA700
:10BF20008BA79CA70DA11EA12FA138A5012B022B29
:10BF3000032B09F09EC388E62BA13CA1829F8001C0
:10BF4000839F100D112401591E4EF801818D928D91
:10BF5000A38DB48D892B8A2B8B2B09F08AC3858DF9
:10BF6000968DA78DB0A1892B8A2B8B2B09F081C3CD
:10BF70002091EF063091F0064091F1065091F206C3
:10BF800069A57AA58BA59CA50E94BCE60E9469EBD9
:10BF90000E94ECEB2B013C01F801E95BFF4F1082A2
:10BFA00088E62BA13CA1829F8001839F100D112464
:10BFB00001591E4EF801E25AFF4F408251826282BF
:10BFC0007382C301B2010E945BE629A53AA54BA585
:10BFD0005CA50E947FEB6AAF7BAF8CAF9DAFD801B1
:10BFE00051966D937D938D939C935497F801E95BE3
:10BFF000FF4F8081882381F17801B8E4EB0EF11CBA
:10C0000037962091E3063091E4064091E506509181
:10C01000E60660817181828193810E94BCE62AAD2F
:10C020003BAD4CAD5DAD0E94BCE620919E103091C1
:10C030009F104091A0105091A1100E94BCE69B015E
:10C04000AC0160E074E284EF99E40E947FEB0E940F
:10C05000ECEBF7017183608388E60BA11CA1809F44
:10C06000F001819FF00D1124E159FE4E21813281B2
:10C07000438154812C962CAF3DAF4EAF5FAF2C97D0
:10C08000CA01B9010E940EED362E272E8C0143ED18
:10C0900056E062965FAF4EAF62973E0151E1650E8A
:10C0A000711C83ED96E09FAB8EAB24964EAC5FACDB
:10C0B00024973DA62DA209A719AB1AAAD201CD90AB
:10C0C000DD90ED90FD902D0120E030E0A901C70149
:10C0D000B6010E94C9EC87FF04C0F7FAF094F7F8A4
:10C0E000F094EEA9FFA981909190A190B190FFAB3F
:10C0F000EEABA7019601C501B4010E9457E687FD8A
:10C10000D8C564147504D1F627965FAD27975523DB
:10C1100009F448C6C090B509D090B609E090B709B7
:10C12000F090B8092DEB37E346E855E3C701B601B7
:10C130000E9457E687FD36C6C701B6010E940EED84
:10C140006B017C019B01AC01632D722DC8010E9423
:10C1500057E687FD03C03C2C2D2C87019601A701D3
:10C16000632D722DC8010E947FEB68966CAF7DAF86
:10C170008EAF9FAF689789EB99E028969FAF8EAFFF
:10C18000289720E030E040E85FE32AAB3BAB4CABC4
:10C190005DAB1EAA2896AEADBFAD28972D913D91FF
:10C1A0004D915D912896BFAFAEAF289768966CAD64
:10C1B0007DAD8EAD9FAD68970E94BCE64B015C01E2
:10C1C0002496EEADFFAD2497C190D190E190F1900F
:10C1D0002496FFAFEEAF2497FEA9FF2391F02AA982
:10C1E0003BA94CA95DA90E94BCE64B015C012AA9B0
:10C1F0003BA94CA95DA9C701B6010E94BCE66B0131
:10C200007C01A7019601C501B4010E94C9EC20E0A0
:10C2100030E0A90118160CF092C5C701B6010E94C2
:10C22000C9EC18160CF486C520E030E0A901C50160
:10C23000B4010E9457E687FD7DC52601370177FAD4
:10C24000709477F87094A3019201C501B4010E9423
:10C25000C9EC181614F4240135016296AEADBFADD9
:10C260006297CD90DD90ED90FD906296BFAFAEAF3E
:10C270006297A3019201C701B6010E9457E687FFAA
:10C2800015C0A3019201C701B6010E947FEB9B017B
:10C29000AC016AA97BA98CA99DA90E94BCE66AABE6
:10C2A0007BAB8CAB9DABBEA9BF5FBEABE9ECF9E04D
:10C2B00028962EAD3FAD2897E217F30709F06ACF15
:10C2C0003EA9332361F02AA93BA94CA95DA9632D9E
:10C2D000722DC8010E94BCE6362E272E8C0124EA5E
:10C2E00030E74DE75FE3632D722DC8010E94BCE685
:10C2F0006B017C01209111073091120740911307C7
:10C30000509114070E9457E687FD42C58DA59DA157
:10C31000A9A5B9A98093110790931207A0931307B9
:10C32000B093140728E64BA15CA1249FC001259F70
:10C33000900D1124DC01A159BE4E7D01232D322D1B
:10C34000A801632D722DC8010E94BCE6F701618728
:10C350007287838794876AAD7BAD8CAD9DAD905815
:10C360009B01AC010E94A3EAD7011D962D913D913E
:10C370004D915C9150970E94BCE69B01AC016BE033
:10C3800077ED83E29BE30E94A2EA9B01AC018BE084
:10C3900097EDA3E2BBE3F70185839683A783B0877C
:10C3A00010812C966CAD7DAD8EAD9FAD2C970E940B
:10C3B00057E618160CF4FBC483E0182B88E62BA173
:10C3C0003CA1829FF001839FF00D1124E159FE4EA4
:10C3D000108380E1FE013196A9EBB9E001900D9246
:10C3E0008A95E1F72C968CAD9DADAEADBFAD2C9787
:10C3F0008093B5099093B609A093B709B093B80993
:10C40000E0960CAD1DAD2EAD3FADE0970093D90980
:10C410001093DA092093DB093093DC09E4962CAD04
:10C420003DAD4EAD5FADE4972093DD093093DE095D
:10C430004093DF095093E009E8968CAD9DADAEAD19
:10C44000BFADE8978093E1099093E209A093E309D7
:10C45000B093E40960960CAD1DAD2EAD3FAD609775
:10C460000093E5091093E6092093E7093093E80962
:10C470006C962CAD3DAD4EAD5FAD6C972093C90968
:10C480003093CA094093CB095093CC09A0968CAD48
:10C490009DADAEADBFADA0978093CD099093CE0971
:10C4A000A093CF09B093D009A4960CAD1DAD2EADCD
:10C4B0003FADA4970093D1091093D2092093D309DB
:10C4C0003093D40922962CAD3DAD4EAD5FAD229791
:10C4D0002093D5093093D6094093D7095093D809B2
:10C4E0009091B3098091B409981303C084E68093B6
:10C4F000B009E9968FADE9978F5F8F708093B3098C
:10C500008091B3099091B20981508F70891351C401
:10C510001091B4091BA30091B3090DA728E61BA134
:10C520000DA51013D1C4812C912CA12CB12C1DA2CE
:10C5300019A619AA1EAE212C312C00E010E02DA561
:10C540003BA12313CEC42114310409F07FC580918F
:10C550006F00826080936F0081E0ECC680E0EAC6E5
:10C5600060900707709008070091090710910A076B
:10C57000A7CA818D928DA38DB48D0697A105B105B3
:10C5800008F018CB858D968DA78DB0A10697A105D3
:10C59000B10508F00FCB20E030E0A901C701B601DA
:10C5A0000E94C9EC87FF04C0F7FAF094F7F8F09402
:10C5B00088E60BA11CA1809FF001819FF00D112442
:10C5C000E159FE4EC586D686E786F08A3ACB809141
:10C5D000030790910407A0910507B0910607C816BC
:10C5E000D906EA06FB0608F06CCB8C199D09AE094A
:10C5F000BF09BC01CD01660F771F881F991F2796C1
:10C600004FAD2797042F10E020E030E0A9019801FA
:10C610000E9445EACA01B9010E945BE60E94D4EC7F
:10C620006C0D7D1D8E1D9F1D0E945BE69B01AC0164
:10C6300060E074E284E799E40E947FEB4B015C01C7
:10C6400040CBA7019601C301B2010E947FEB7B01A1
:10C650008C019B01AC01632D722D89A599A90E94C3
:10C66000C9EC18160CF0E0CB3E2C2F2C09A719AB07
:10C67000DBCB0AA91BA92CA93DA9012B022B032B5B
:10C6800049F02091EB063091EC064091ED06509177
:10C69000EE0608C02091E7063091E8064091E906D1
:10C6A0005091EA0669A57AA58BA59CA50E94BCE6D7
:10C6B0000E9469EB0E94ECEB2B013C012AA93BA9EB
:10C6C0004CA95DA9232B242B252BC9F020E030E0B9
:10C6D000A9016091E3067091E4068091E5069091CE
:10C6E000E6060E9457E6882351F081E00DA51EA5BD
:10C6F0002FA538A910161106120613060CF080E0BB
:10C7000098E62BA13CA1929F8001939F100D1124CC
:10C7100001591E4E180137E4230E311CD1018C93B0
:10C72000882309F4B3C02091C9093091CA09409106
:10C73000CB095091CC096C966CAD7DAD8EAD9FADA3
:10C740006C970E94A2EA6DA77EA78FA798AB209155
:10C75000CD093091CE094091CF095091D009A096D2
:10C760006CAD7DAD8EAD9FADA0970E94A2EA4B014E
:10C770005C012091D1093091D2094091D3095091A7
:10C78000D409A4966CAD7DAD8EAD9FADA4970E94EB
:10C79000A2EA6B017C012DA53EA54FA558A9CA01AF
:10C7A000B9010E94BCE66DA77EA78FA798ABA50133
:10C7B0009401C501B4010E94BCE69B01AC016DA5CA
:10C7C0007EA58FA598A90E94A3EA4B015C01A70151
:10C7D0009601C701B6010E94BCE69B01AC01C501F0
:10C7E000B4010E94A3EA0E940EED6B017C0120912E
:10C7F000D5093091D6094091D7095091D809229690
:10C800006CAD7DAD8EAD9FAD22970E94A2EAA701CF
:10C8100096010E947FEB6B017C01F801E25BFF4F08
:10C82000608371838283938320E030E040E450E4AE
:10C830000E94C9EC18161CF4F101108227C0209147
:10C84000E3063091E4064091E5065091E606C70103
:10C85000B6010E94BCE69B01AC016091DF067091BD
:10C86000E0068091E1069091E2060E947FEB29A507
:10C870003AA54BA55CA50E94BCE60E94ECEB6415B2
:10C8800075058605970510F42B013C0180913B113D
:10C8900090913C11A0913D11B0913E110EA91FA99C
:10C8A00028AD39AD80179107A207B30708F4DFC0A0
:10C8B0002DA13EA14FA158A5232B242B252B41F1BF
:10C8C00060913F11709140118091411190914211FE
:10C8D0006415750586059705D8F42EA93FA948ADBE
:10C8E00059AD0E9436EA6B017C012DA13EA14FA1FA
:10C8F00058A5C301B2010E9436EAC616D706E8065B
:10C90000F90630F4C701B6010E9445EA29013A014F
:10C9100088E60BA11CA1809FF001819FF00D1124DE
:10C92000E159FE4EC18CD28CE38CF48CC114D1043D
:10C93000E104F10431F1609143117091441180914F
:10C940004511909146116415750586059705C8F443
:10C950002EA93FA948AD59AD0E9436EA4B015C01B2
:10C96000A7019601C301B2010E9436EA8616970616
:10C97000A806B90630F4C501B4010E9445EA2901B0
:10C980003A0188E60BA11CA1809FF001819FF00D68
:10C990001124E159FE4EC58CD68CE78CF0A0C11451
:10C9A000D104E104F10431F1609147117091481113
:10C9B0008091491190914A11641575058605970576
:10C9C000C8F42EA93FA948AD59AD0E9436EA4B01E3
:10C9D0005C01A7019601C301B2010E9436EA8616E6
:10C9E0009706A806B90630F4C501B4010E9445EACD
:10C9F00029013A0188E60BA11CA1809FF001819FCB
:10CA0000F00D1124E159FE4EC1A0D2A0E3A0F4A084
:10CA1000C114D104E104F10409F4C2CA60914B11BC
:10CA200070914C1180914D1190914E1164157505C6
:10CA30008605970508F0B4CA2EA93FA948AD59AD9F
:10CA40000E9436EA4B015C01A7019601C301B201C5
:10CA50000E9436EA86169706A806B90608F0A0CA0C
:10CA6000C501B4010E9445EA29013A0199CA2DA1E4
:10CA70003EA14FA158A5232B242B252BC9F1609152
:10CA80003F117091401180914111909142116415B4
:10CA900075058605970560F50E945BE62AAD3BADFE
:10CAA0004CAD5DAD0E94BCE66B017C016DA17EA129
:10CAB0008FA198A50E945BE64B015C01C301B20106
:10CAC0000E945BE6A50194010E94BCE69B01AC01BB
:10CAD000C701B6010E9457E687FF0AC0A50194016D
:10CAE000C701B6010E947FEB0E94ECEB2B013C01D9
:10CAF00088E60BA11CA1809FF001819FF00D1124FD
:10CB0000E159FE4E818C928CA38CB48C81149104DB
:10CB1000A104B104B9F16091431170914411809165
:10CB2000451190914611641575058605970550F5D8
:10CB30000E945BE62AAD3BAD4CAD5DAD0E94BCE60C
:10CB40006B017C01C501B4010E945BE64B015C01F5
:10CB5000C301B2010E945BE6A50194010E94BCE6FC
:10CB60009B01AC01C701B6010E9457E687FF0AC0CE
:10CB7000A5019401C701B6010E947FEB0E94ECEB76
:10CB80002B013C0188E60BA11CA1809FF001819F35
:10CB9000F00D1124E159FE4E858C968CA78CB0A027
:10CBA00081149104A104B104B9F16091471170910D
:10CBB00048118091491190914A11641575058605B7
:10CBC000970550F50E945BE62AAD3BAD4CAD5DADDF
:10CBD0000E94BCE66B017C01C501B4010E945BE6CA
:10CBE0004B015C01C301B2010E945BE6A501940107
:10CBF0000E94BCE69B01AC01C701B6010E9457E64A
:10CC000087FF0AC0A5019401C701B6010E947FEB0E
:10CC10000E94ECEB2B013C0188E60BA11CA1809F3C
:10CC2000F001819FF00D1124E159FE4EC1A0D2A068
:10CC3000E3A0F4A0C114D104E104F10409F4B0C9E3
:10CC400060914B1170914C1180914D1190914E114A
:10CC5000641575058605970508F0A2C90E945BE674
:10CC60002AAD3BAD4CAD5DAD0E94BCE64B015C0115
:10CC7000C701B6010E945BE66B017C01C301B201F2
:10CC80000E945BE6A70196010E94BCE69B01AC01F5
:10CC9000C501B4010E9457E687FF82C9A70196012A
:10CCA000C501B4010E947FEB0E94ECEB2B013C011B
:10CCB00077C9FAA9FF2331F1A5019401632D722DE3
:10CCC000C8010E94BCE64B015C012DA53DA149A510
:10CCD00059A9C701B6010E94BCE69B01AC01C50180
:10CCE000B4010E9457E687FF22C0A7019601C50143
:10CCF000B4010E947FEB6DA77DA389A799AB21E0CA
:10CD00002AABFFC9A7019601C501B4010E947FEBC0
:10CD10009B01AC016DA57DA189A599A90E94BCE6E6
:10CD20006DA77DA389A799AB31E03AABEAC941E091
:10CD30004AABE7C9A7019601C501B40113C0C701F9
:10CD4000B6010E9457E687FD09C020E030E0A90146
:10CD5000C501B4010E94C9EC18164CF4A501940158
:10CD6000C701B6010E94A2EA2B013C0176CA240148
:10CD7000350177FA709477F87094A3019201C70196
:10CD8000B6010E9457E687FD68CA2601370165CAC9
:10CD90002DA53DA149A559A9C701B6010E9457E695
:10CDA00087FFB4CA3DA42DA009A519A9AFCA81E087
:10CDB00004CBF090B3098FEF8F0D8F708BA3B090E1
:10CDC000B2098091B309B81609F454C0C12CD12C12
:10CDD0000BA10B1509F44EC0602E712C28E6269D80
:10CDE0008001279D100D112401591E4ED8018C91F0
:10CDF00083FD2BC00EAF1AAB0115110541F1199639
:10CE0000BC91BDA7F801F285FDA3D8011B96BC918A
:10CE1000B9A7F801F485F9ABD80115962D903D908E
:10CE20004D905C901897A20191016DA57DA189A5F7
:10CE30009F2F0E9457E6811186C1C114D10439F099
:10CE4000F601808180FD7FC102C0CEAEDAAA8BA13F
:10CE500081508F708BA38091B2098B1103C0CEAC2F
:10CE6000DAA8B6CF0BA10B1529F081E08B0D8F70DE
:10CE7000B82EF1CF1091B2091BA3C12CD12C8091F7
:10CE8000B3090BA1801709F443CB802E912C28E61F
:10CE9000289D8001299D100D112401591E4ED80195
:10CEA0008C9183FD0AC05801C114D10439F0C60128
:10CEB0000E943B7F811102C0C5C156018BA18F5FCB
:10CEC0008F708BA36501DBCF802F81508F70289FDF
:10CED000F0011124E159FE4E908193FF24CB8DA7E0
:10CEE0001ECB48E6439FC0011124DC01A159BE4E70
:10CEF0001D018C9183FD19C015966D917D918D91C9
:10CF00009C9118970E940EEDF62EE72ED82EC92E72
:10CF10000115110509F48CC0F801808180FD0AC05B
:10CF2000D1018C9180FD06C083C0FDA0E9A4D9A8E1
:10CF3000CEAC83C0F801808181608083C8010E94EB
:10CF40003B7F811171C0F80161817281838194817D
:10CF50000E940EED2B013C019B01AC0160E070E0F2
:10CF600080E89FE30E947FEB4B015C019B01AC01D9
:10CF70006F2D7E2D8D2D9C2D0E94BCE669837A83BA
:10CF80008B839C832DA139A549A95EADC501B40150
:10CF90000E94BCE6698B7A8B8B8B9C8BAE014F5FBA
:10CFA0005F4FBE016F5E7F4FC8010E946AB8F801F3
:10CFB000E95BFF4F80818823B9F12091E30630912E
:10CFC000E4064091E5065091E6063796608171814E
:10CFD000828193810E94BCE620919E1030919F1027
:10CFE0004091A0105091A1100E94BCE64B015C0141
:10CFF0009B01AC01C301B2010E94BCE60E94ECEBB4
:10D00000F801E65BFF4F71836083A50194016F2DEA
:10D010007E2D8D2D9C2D0E94BCE60E94ECEBF8012C
:10D02000E45BFF4F71836083D8018C918E7F8C937A
:10D030008F2C9E2CAD2CBC2C81018BA18F5F8F700F
:10D040008BA3FDA2E9A6D9AACEAE79CAF10180814F
:10D0500081608083C8010E943B7F81116FC0D10134
:10D0600011966D917D918D919C9114970E940EED7A
:10D070006B017C019B01AC0160E070E080E89FE304
:10D080000E947FEB2B013C012DEC3CEC4CE45DE37A
:10D090000E94BCE669837A838B839C839401A501FB
:10D0A000C301B2010E94BCE6698B7A8B8B8B9C8B8F
:10D0B000AE014F5F5F4FBE016F5E7F4FC1010E94A7
:10D0C0006AB8F101E95BFF4F80818823B9F12091B3
:10D0D000E3063091E4064091E5065091E606379666
:10D0E00060817181828193810E94BCE620919E10B3
:10D0F00030919F104091A0105091A1100E94BCE669
:10D100004B015C019B01AC01C701B6010E94BCE66A
:10D110000E94ECEBF101E65BFF4F718360832DEC25
:10D120003CEC4CE45DE3C501B4010E94BCE60E9406
:10D13000ECEBF101E45BFF4F71836083F1018081CF
:10D140008E7F808304CA28E6269DF001279DF00D7E
:10D150001124E159FE4E808181FD43C0C114D104E8
:10D1600041F0D6011596CD90DD90ED90FC9018978A
:10D1700008C08BE0C82E87EDD82E83E2E82E8BE323
:10D18000F82EB8E6B69DF001B79DF00D1124E159D7
:10D19000FE4E81899289A389B489BC01CD01905842
:10D1A0009B01AC010E94A3EAF801258536854785DD
:10D1B00050890E94BCE69B01AC01C701B6010E94E8
:10D1C000A2EAE62E872E982EA92E262F372F482F3B
:10D1D000592F6DA57DA189A599A90E9457E687FFC2
:10D1E00004C0EDA48DA099A4A9A82E2D382D492DF9
:10D1F0005A2DC201B1010E9457E6882309F427CEB7
:10D20000F8E6F69DC001F79D900D11249C0121596F
:10D210003E4E6901D9018C9181608C93C8010E94B6
:10D220003B7F882329F0F60180818E7F80830FCE9B
:10D230008E2D982DA92DBA2DF60185839683A7836F
:10D24000B08705CED6018C9181FD52C0D6011596CE
:10D250002D913D914D915C9118972DA73EA74FA719
:10D2600058AB1501B5E02B0E311CF80145805680F6
:10D2700067807084A30192016DA57EA58FA598A9F2
:10D280000E9457E687FF34C0F60181899289A389FD
:10D29000B489BC01CD0190589B01AC010E94A3EA66
:10D2A000D6011D962D913D914D915C9150970E9414
:10D2B000BCE69B01AC016DA57EA58FA598A90E9437
:10D2C000A2EA6B017C019B01AC01C301B2010E9487
:10D2D000C9EC18166CF4D8018C9181608C93C5014F
:10D2E0000E943B7F8823E1F0F80180818E7F80835C
:10D2F00018E6189DF001199DF00D1124E159FE4E1C
:10D300002185328543855485658176818781908525
:10D310000E9457E68111D2CD0BA10093B209CECD68
:10D32000D101CD92DD92ED92FC9213970BA1009367
:10D33000B209DECFC858DF4F0FB6F894DEBF0FBE7C
:10D34000CDBFDF91CF911F910F91FF90EF90DF90B4
:10D35000CF90BF90AF909F908F907F906F905F9095
:10D360004F903F902F9008958091B3099091B40908
:10D37000891B8F708F3019F40E941FA1F5CF809107
:10D38000B3098F5F8F70E091B30998E69E9FF0011B
:10D390001124E159FE4EDF011D929A95E9F798E0BC
:10D3A00090834091D9095091DA096091DB0970911D
:10D3B000DC09458B568B678B708F4091DD0950914E
:10D3C000DE096091DF097091E009418F528F638F10
:10D3D000748F4091E1095091E2096091E3097091E5
:10D3E000E409458F568F678F70A34091E5095091EE
:10D3F000E6096091E7097091E80941A352A363A38C
:10D4000074A32091B3099091B409291303C094E641
:10D410009093B0098093B30980916F0082608093EC
:10D420006F0008959091B3098091B409981306C0D4
:10D4300080914A0790914B07892B19F00E941FA1F8
:10D44000F1CF0895CF93DF938B3D9240B1F0E1EDA2
:10D45000FDE18491EF012196882321F00E94E19360
:10D46000FE01F7CFE8EDF9E18491EF0121968823E1
:10D4700031F00E94E193FE01F7CF80E001C081E02E
:10D48000DF91CF9108952F923F924F925F926F92CA
:10D490007F928F929F92AF92BF92CF92DF92EF9244
:10D4A000FF920F931F93CF93DF93CDB7DEB7C7578C
:10D4B000D1090FB6F894DEBF0FBECDBF2DB63EB674
:10D4C000A7961FAE1EAEA79784E690E0A9969FAFE1
:10D4D0008EAFA99701E09E012B593F4F44E050E0E9
:10D4E000BE01655A7F4FCE0189599F4F0E9412D0CD
:10D4F0009E012B593F4F42E050E0BE0167597F4FDC
:10D50000CE0189599F4F0E9412D043E050E0BE01E6
:10D51000655A7F4F8FED92E00E940EEE892B09F441
:10D520003FC06F968FAD6F97882339F08FE36C966D
:10D530008FAF6C976D961FAE6D97E6EEFDE184910F
:10D540007F012FEFE21AF20A811103C0EBE9FAE141
:10D5500004C00E94E193F701F2CF84917F013FEF75
:10D56000E31AF30A882321F00E94E193F701F5CF33
:10D57000BE01655A7F4F82E99AE10E9487C5E4E8BF
:10D58000FAE184917F019FEFE91AF90A882321F0DB
:10D590000E94E193F701F5CF81E08093160754C50F
:10D5A000EDB7FEB7E696FFAFEEAFE6976B961CAE13
:10D5B0001DAE1EAE1FAE6B97A7961FAE1EAEA797F1
:10D5C00001E09E012B593F4F41E050E0BE01605900
:10D5D0007F4FCE0189599F4F0E9412D080E1EBE529
:10D5E000F2E0DE01919601900D928A95E1F780E1DB
:10D5F000EBE6F2E0DE01519601900D928A95E1F79B
:10D6000080E1EBE7F2E0DE01119601900D928A9540
:10D61000E1F7E1964FADE19750E04D5F5F4F440F6A
:10D62000551F440F551F2DB73EB7241B350B0FB6A2
:10D63000F8943EBF0FBE2DBF8DB79EB701967C01FB
:10D6400000E09E012B593F4FBC01CE0189599F4FED
:10D650000E9412D09E012B593F4F44E050E063E0FE
:10D6600077E0CE0189599F4F0E9412D0E1968FAC8E
:10D67000E197912C93E0890E911C880C991C880CE1
:10D68000991CEDB7FEB7E819F9090FB6F894FEBF7B
:10D690000FBEEDBF2DB73EB72F5F3F4F69018DB76E
:10D6A0009EB7881999090FB6F8949EBF0FBE8DBF1B
:10D6B000EDB7FEB731965F019E012B593F4FA40194
:10D6C000B601CE0189599F4F0E9412D09E012B595D
:10D6D0003F4FA401B501CE0189599F4F0E9412D03E
:10D6E00010911707112309F4A7C000E09E012B59E0
:10D6F0003F4F44E050E06BEE76E0CE0189599F4FFA
:10D700000E9412D09E012B593F4F44E050E06FEE33
:10D7100076E0CE0189599F4F0E9412D09E012B596D
:10D720003F4F44E050E067EE76E0CE0189599F4FCD
:10D730000E9412D09E012B593F4F44E050E06BE015
:10D7400077E0CE0189599F4F0E9412D09E012B593C
:10D750003F4F44E050E067E077E0CE0189599F4FAA
:10D760000E9412D09E012B593F4F40E150E063EDE3
:10D7700076E0CE0189599F4F0E9412D09E012B590D
:10D780003F4F44E050E0BE01695A7F4FCE018959B6
:10D790009F4F0E9412D09E012B593F4F4CE050E00A
:10D7A00068E375E0CE0189599F4F0E9412D09E0117
:10D7B0002B593F4F44E050E063E371E1CE018959BA
:10D7C0009F4F0E9412D09E012B593F4F44E050E0E2
:10D7D000BE01695A7F4FCE0189599F4F0E9412D0D6
:10D7E00001E09E012B593F4F41E050E0BE016159DD
:10D7F0007F4FCE0189599F4F0E9412D09E012B5915
:10D800003F4F41E050E0BE0162597F4FCE01895940
:10D810009F4F0E9412D011118AC06B968CAD9DADA6
:10D82000AEADBFAD6B978093C2109093C310A09321
:10D83000C410B093C5107BC0E1968FADE19790E026
:10D84000029623EF36E0E4963FAF2EAFE497B501A2
:10D85000DE011196E2E98E2EE0E19E2EAE014F5ED2
:10D860005F4FFFE4AF2EF1E1BF2EE896FFAEEEAEC4
:10D87000E8977E0131E2E30EF11C20E030E08217F0
:10D8800093072CF0E896EEADFFADE89701C0F701E5
:10D890004080518062807380F50141925192619283
:10D8A00071925F018217930714F0F60101C0FA012B
:10D8B0004080518062807380F40141925192619264
:10D8C00071924F018217930734F0FB014080518021
:10D8D0006280738005C04D905D906D907C90139731
:10D8E000E496EEADFFADE497419251926192719250
:10D8F000E496FFAFEEAFE4972F5F3F4F6C5F7F4F33
:10D900001496F4E0CF0ED11C4C5F5F4FE896EEAD5D
:10D91000FFADE8973496E896FFAFEEAFE897F4E0F6
:10D92000EF0EF11C2430310509F0A9CFDECEE096D0
:10D930008FADE097853099F4AF968FADAF97853076
:10D9400071F400E09E012B593F4F44E650E066EC35
:10D9500070E1CE0189599F4F0E9412D024C011114D
:10D9600002C00E94D2BDE0968FADE097AF96CFACDB
:10D97000AF978C9D60011124E12CF12CEC14FD0477
:10D9800091F000E09E012B593F4F44E050E0BE0172
:10D99000695A7F4FCE0189599F4F0E9412D02FEFB5
:10D9A000E21AF20AEBCF00E09E012B593F4F44E010
:10D9B00050E0BE016D5A7F4FCE0189599F4F0E94A2
:10D9C00012D01AE0115079F000E09E012B593F4F20
:10D9D00044E050E0BE01695A7F4FCE0189599F4F04
:10D9E0000E9412D0EFCF01E09E012B593F4F41E042
:10D9F00050E0BE0163597F4FCE0189599F4F0E946D
:10DA000012D09E012B593F4F41E050E0BE016459B6
:10DA10007F4FCE0189599F4F0E9412D000E09E0196
:10DA20002B593F4F44E050E0BE01635C7F4FCE0175
:10DA300089599F4F0E9412D09E012B593F4F44E0BD
:10DA400050E0BE016F5C7F4FCE0189599F4F0E940D
:10DA500012D0AE968FADAE97AD96CFACAD978C9DF4
:10DA600060011124E12CF12C00E09E012B593F4F65
:10DA7000CE14DF0471F044E050E0BE01695A7F4FDC
:10DA8000CE0189599F4F0E9412D03FEFE31AF30A4B
:10DA9000EBCF41E050E0BE016F587F4FCE01895976
:10DAA0009F4F0E9412D09E012B593F4F41E050E002
:10DAB000BE0165597F4FCE0189599F4F0E9412D0F8
:10DAC0009E012B593F4F44E050E0BE01695A7F4F01
:10DAD000CE0189599F4F0E9412D09E012B593F4F72
:10DAE00044E050E0BE01695A7F4FCE0189599F4FF3
:10DAF0000E9412D09E012B593F4F44E050E067E353
:10DB000071E1CE0189599F4F0E9412D09E012B597D
:10DB10003F4F44E050E0BE01615B7F4FCE01895929
:10DB20009F4F0E9412D09E012B593F4F44E050E07E
:10DB3000BE01655B7F4FCE0189599F4F0E9412D075
:10DB40009E012B593F4F44E050E0BE01695B7F4F7F
:10DB5000CE0189599F4F0E9412D010E000E09E0133
:10DB60002B593F4F44E050E0BE01695A7F4FCE0130
:10DB700089599F4F0E9412D0111110C06B96CCACE6
:10DB8000DDACEEACFFAC6B9720E030E84BE355E446
:10DB9000C701B6010E9457E6811103C054E0F52E7B
:10DBA00033C080911707811108C0C0923C07D09202
:10DBB0003D07E0923E07F0923F0700E09E012B599F
:10DBC0003F4F44E050E068E377E0CE0189599F4F32
:10DBD0000E9412D09E012B593F4F44E050E060E478
:10DBE00077E0CE0189599F4F0E9412D09E012B5998
:10DBF0003F4F44E050E0BE01695A7F4FCE01895942
:10DC00009F4F0E9412D012C0FA94FF2079F000E0DA
:10DC10009E012B593F4F44E050E0BE01695A7F4FAF
:10DC2000CE0189599F4F0E9412D0EECF1F5F153051
:10DC300009F094CF00E09E012B593F4F42E050E0A5
:10DC4000BE016D597F4FCE0189599F4F0E9412D05E
:10DC50009E012B593F4F44E050E0BE01695A7F4F6F
:10DC6000CE0189599F4F0E9412D06B96CCACDDAC8F
:10DC7000EEACFFAC6B9720E030E84BE355E4C70116
:10DC8000B6010E9457E6882329F180911707811178
:10DC900008C0C0923407D0923507E0923607F09260
:10DCA000370700E09E012B593F4F44E050E060E30E
:10DCB00077E0CE0189599F4F0E9412D09E012B59C7
:10DCC0003F4F44E050E06CE277E0CE0189599F4F2E
:10DCD0000E9412D000E09E012B593F4F42E050E0DD
:10DCE000BE016F597F4FCE0189599F4F0E9412D0BC
:10DCF0009E012B593F4F41E050E0BE016F587F4FCE
:10DD0000CE0189599F4F0E9412D019E0115000E0B6
:10DD10009E012B593F4F112359F044E050E0BE01C2
:10DD2000695A7F4FCE0189599F4F0E9412D0EECF82
:10DD300041E050E06AE271E1CE0189599F4F0E94B3
:10DD400012D0F12C00E09E012B593F4F44E050E0EF
:10DD5000BE01695A7F4FCE0189599F4F0E9412D050
:10DD600010911707111110C0F1100EC06B968CADF9
:10DD70009DADAEADBFAD6B9780932F1190933011D9
:10DD8000A0933111B0933211F39485E0F812DACFF9
:10DD9000111102C00E94D2C44CE0F42EFA94F1108A
:10DDA00003C03CE0F32E0FC000E09E012B593F4F13
:10DDB00042E050E0BE01615A7F4FCE0189599F4F2A
:10DDC0000E9412D0EBCFFA9400E09E012B593F4FF6
:10DDD000FF2059F044E050E0BE016D5B7F4FCE0163
:10DDE00089599F4F0E9412D0EECF46E050E0BE010D
:10DDF000635C7F4FCE0189599F4F0E9412D09E01D4
:10DE00002B593F4F44E050E063EE76E0CE01895954
:10DE10009F4F0E9412D09E012B593F4F4CE050E083
:10DE2000BE016F5C7F4FCE0189599F4F0E9412D077
:10DE30002CE1F22EFA94F11003C094E0F92E1DC0EB
:10DE400000E09E012B593F4F44E050E0BE01695A6B
:10DE50007F4FCE0189599F4F0E9412D0EBCF00E037
:10DE60009E012B593F4F44E050E0BE01695A7F4F5D
:10DE7000CE0189599F4F0E9412D0FA94F110EFCF32
:10DE80008BE0F82EFA94FF2079F000E09E012B59E8
:10DE90003F4F44E050E0BE01695A7F4FCE0189599F
:10DEA0009F4F0E9412D0EECFA9968EAD9FADA9973D
:10DEB00084569109C7DA80931607882309F1E6EEA4
:10DEC000FDE184917F019FEFE91AF90A882321F08F
:10DED0000E94E193F701F5CFA9966EAD7FADA997AA
:10DEE000645671098CE79AE10E946EC56BED72E091
:10DEF00084E79AE10E946EC58AE00E94E19399C08E
:10DF0000A7962EAD3FADA797AB968EAD9FADAB97C5
:10DF10002817390709F44BC081E080931607E1ED1B
:10DF2000FDE184917F012FEFE21AF20A811103C013
:10DF3000E4E5FAE104C00E94E193F701F2CF849195
:10DF40007F013FEFE31AF30A882321F00E94E19357
:10DF5000F701F5CFAB966EAD7FADAB9780E090E06B
:10DF60004AE00E940297EFE4FAE184917F019FEF7B
:10DF7000E91AF90A882321F00E94E193F701F5CF0D
:10DF8000A7966EAD7FADA79780E090E04AE00E9433
:10DF90000297EFE3FAE184917F012FEFE21AF20A90
:10DFA000882309F446C00E94E193F701F4CF1111D0
:10DFB00042C0E6EEFDE184917F013FEFE31AF30AF0
:10DFC000811103C00FED12E004C00E94E193F7013C
:10DFD000F2CFF80181918F01882319F00E94E1931B
:10DFE000F8CFA9966EAD7FADA9976456710982E20C
:10DFF0009AE10E946EC5A7964EAD5FADA79760E00F
:10E0000070E085E19AE10E9434C5E2E1FAE1849191
:10E010007F012FEFE21AF20A811107C080911607E3
:10E02000811109C00E94D3D006C00E94E193F7017C
:10E03000EECF112399F3E6968EAD9FADE6970FB61E
:10E04000F8949EBF0FBE8DBF80911707811102C04B
:10E050000E949FBE9091160781E089270FB6F89421
:10E060003EBE0FBE2DBEC958DF4F0FB6F894DEBFBF
:10E070000FBECDBFDF91CF911F910F91FF90EF9019
:10E08000DF90CF90BF90AF909F908F907F906F90D8
:10E090005F904F903F902F90089581E080931707F5
:10E0A000F2D9109217078111EEC90E940EC381E0C8
:10E0B00008958F929F92AF92BF92CF92DF92EF928C
:10E0C000FF920F931F93CF93DF93CDB7DEB7CA5A5A
:10E0D000D1090FB6F894DEBF0FBECDBFE9961CAED6
:10E0E0001DAE1EAE1FAEE9978091EC039091ED033B
:10E0F000A091EE03B091EF03ED968CAF9DAFAEAF64
:10E10000BFAFED97C556DF4F19821882CB59D0406B
:10E1100084E690E0C356DF4F99838883CD59D04081
:10E12000109216079E0125563F4F44E050E0BE0175
:10E1300067587F4FCE0183569F4F0E945FD0C356D2
:10E14000DF4F88819981CD59D0400296C356DF4F69
:10E1500099838883CD59D040C556DF4F19821882E4
:10E16000CB59D04081E0CD55DF4F8883C35AD04092
:10E170009E0125563F4F41E050E0BE016D557F4F57
:10E18000CE0183569F4F0E945FD09E0125563F4F80
:10E1900040E150E06FE471E1CE0183569F4F0E9451
:10E1A0005FD09E0125563F4F44E050E063E077E0AA
:10E1B000CE0183569F4F0E945FD09E0125563F4F50
:10E1C00040E150E062E970E1CE0183569F4F0E942A
:10E1D0005FD09E0125563F4F40E150E063EF76E06F
:10E1E000CE0183569F4F0E945FD09E0125563F4F20
:10E1F00044E050E06BEE76E0CE0183569F4F0E94E4
:10E200005FD09E0125563F4F44E050E06FEE76E030
:10E21000CE0183569F4F0E945FD09E0125563F4FEF
:10E2200044E050E067EE76E0CE0183569F4F0E94B7
:10E230005FD09E0125563F4F44E050E06BE077E011
:10E24000CE0183569F4F0E945FD09E0125563F4FBF
:10E2500044E050E067E077E0CE0183569F4F0E9494
:10E260005FD09E0125563F4F40E150E063ED76E0E0
:10E27000CE0183569F4F0E945FD08AE097EDA3EABC
:10E28000BCE3E9968CAF9DAFAEAFBFAFE9979E01FF
:10E2900025563F4F44E050E0BE016B587F4FCE0102
:10E2A00083569F4F0E945FD09E0125563F4F4CE002
:10E2B00050E068E375E0CE0183569F4F0E945FD027
:10E2C00080917D1090917E10A0917F10B091801070
:10E2D000C358DF4F88839983AA83BB83CD57D0402F
:10E2E0009E0125563F4F44E050E0BE0163587F4FEA
:10E2F000CE0183569F4F0E945FD085E0CC55DF4F03
:10E300008883C45AD040CB55DF4F8883C55AD0404C
:10E310009E0125563F4F44E050E062EC70E1CE0193
:10E3200083569F4F0E945FD09E0125563F4F41E08C
:10E3300050E0BE016C557F4FCE0183569F4F0E9427
:10E340005FD09E0125563F4F41E050E0BE016B5526
:10E350007F4FCE0183569F4F0E945FD09E0125566E
:10E360003F4F44E650E066EC70E1CE0183569F4F8C
:10E370000E945FD0CF57DF4F188219821A821B820A
:10E38000C158D0409E0125563F4F44E050E0BE01A9
:10E390006F577F4FCE0183569F4F0E945FD0E99603
:10E3A0001CAE1DAE1EAE1FAEE9971AE0115071F003
:10E3B0009E0125563F4F44E050E0BE016B587F4F11
:10E3C000CE0183569F4F0E945FD0F0CF83E0CA55A5
:10E3D000DF4F8883C65AD040C955DF4F8883C75A5C
:10E3E000D040CB57DF4F188219821A821B82C55842
:10E3F000D040C757DF4F188219821A821B82C95832
:10E40000D040E9961CAE1DAE1EAE1FAEE9979E0130
:10E4100025563F4F41E050E0BE016A557F4FCE0187
:10E4200083569F4F0E945FD09E0125563F4F41E08B
:10E4300050E0BE0169557F4FCE0183569F4F0E9429
:10E440005FD09E0125563F4F44E050E0BE01675724
:10E450007F4FCE0183569F4F0E945FD09E0125566D
:10E460003F4F44E050E0BE016B577F4FCE018356D3
:10E470009F4F0E945FD00AE010E00150110971F037
:10E480009E0125563F4F44E050E0BE016B587F4F40
:10E49000CE0183569F4F0E945FD0EFCFC855DF4F0C
:10E4A0001882C85AD0408FEFC755DF4F8883C95AAA
:10E4B000D0409E0125563F4F41E050E0BE016855D7
:10E4C0007F4FCE0183569F4F0E945FD09E012556FD
:10E4D0003F4F41E050E0BE0167557F4FCE0183566C
:10E4E0009F4F0E945FD0E9961CAE1DAE1EAE1FAEC0
:10E4F000E9979E0125563F4F44E050E0BE016B581E
:10E500007F4FCE0183569F4F0E945FD09E012556BC
:10E510003F4F44E050E0BE016B587F4FCE01835621
:10E520009F4F0E945FD09E0125563F4F44E050E030
:10E5300067E371E1CE0183569F4F0E945FD08091C7
:10E540008B0290918C02A0918D02B0918E02C357E4
:10E55000DF4F88839983AA83BB83CD58D0408091B5
:10E560008F0290919002A0919102B0919202CF56A9
:10E57000DF4F88839983AA83BB83C159D040CB5690
:10E58000DF4F19821882C559D040C956DF4F198212
:10E590001882C759D0409E0125563F4F44E050E0B5
:10E5A000BE0163577F4FCE0183569F4F0E945FD0BD
:10E5B0009E0125563F4F44E050E0BE016F567F4F0D
:10E5C000CE0183569F4F0E945FD09E0125563F4F3C
:10E5D00044E050E0BE016B567F4FCE0183569F4F03
:10E5E0000E945FD010E0C12C80E8D82E8BE3E82E8B
:10E5F00085E4F82E812C912C90E8A92E9FE3B92E6A
:10E60000111138C09E0125563F4F44E050E06CE3A5
:10E6100077E0CE0183569F4F0E945FD09E01255622
:10E620003F4F44E050E068E377E0CE0183569F4FD0
:10E630000E945FD09E0125563F4F44E050E060E4C9
:10E6400077E0CE0183569F4F0E945FD0E9968CAE53
:10E650009DAEAEAEBFAEE9979E0125563F4F44E05A
:10E6600050E0BE016B587F4FCE0183569F4F0E94F2
:10E670005FD02AC0E996CCAEDDAEEEAEFFAEE99734
:10E680009E0125563F4F44E050E0BE016B587F4F3E
:10E69000CE0183569F4F0E945FD0E9961CAE1DAEFF
:10E6A0001EAE1FAEE99704E0015071F09E012556A1
:10E6B0003F4F44E050E0BE016B587F4FCE01835680
:10E6C0009F4F0E945FD0F0CF1F5F153009F098CFA9
:10E6D00084E190E0C156DF4F99838883CF59D040C1
:10E6E0009E0125563F4F42E050E0BE0161567F4FEC
:10E6F000CE0183569F4F0E945FD09E0125563F4F0B
:10E7000044E050E064E377E0CE0183569F4F0E94DF
:10E710005FD09E0125563F4F44E050E060E377E034
:10E72000CE0183569F4F0E945FD09E0125563F4FDA
:10E7300044E050E06CE277E0CE0183569F4F0E94A8
:10E740005FD080E290E0CF55DF4F99838883C15A34
:10E75000D0409E0125563F4F42E050E0BE016F552C
:10E760007F4FCE0183569F4F0E945FD0C655DF4F2B
:10E770001882CA5AD04080E2E3E9F2E0DE019D96B9
:10E7800001900D928A95E1F79E0125563F4F41E099
:10E7900050E0BE0166557F4FCE0183569F4F0E94C9
:10E7A0005FD09E0125563F4F40E250E0BE01635DC1
:10E7B0007F4FCE0183569F4F0E945FD09E0125560A
:10E7C0003F4F41E050E06AE271E1CE0183569F4F36
:10E7D0000E945FD010E011110EC080912F11909116
:10E7E0003011A0913111B0913211E9968CAF9DAFEB
:10E7F000AEAFBFAFE9979E0125563F4F44E050E0D2
:10E80000BE016B587F4FCE0183569F4F0E945FD051
:10E810001F5F153001F7BE01635B7F4F86E1FB018F
:10E8200011928A95E9F79E0125563F4F46E150E047
:10E83000CE0183569F4F0E945FD08CE2E3EBF2E063
:10E84000DE01119601900D928A95E1F79E01255601
:10E850003F4F4CE250E0BE016F5F7F4FCE018356C9
:10E860009F4F0E945FD0BE0161597F4F86E0FB0140
:10E8700011928A95E9F79E0125563F4F46E050E0F8
:10E88000CE0183569F4F0E945FD09E0125563F4F79
:10E8900044E050E063EE76E0CE0183569F4F0E9445
:10E8A0005FD0BE016D597F4F8CE0FB0111928A95BC
:10E8B000E9F79E0125563F4F4CE050E0CE018356CC
:10E8C0009F4F0E945FD0E9961CAE1DAE1EAE1FAEDC
:10E8D000E9971CE1115071F09E0125563F4F44E02D
:10E8E00050E0BE016B587F4FCE0183569F4F0E9470
:10E8F0005FD0F0CFE9961CAE1DAE1EAE1FAEE997FD
:10E9000014E0115071F09E0125563F4F44E050E055
:10E91000BE016B587F4FCE0183569F4F0E945FD040
:10E92000F0CFE9961CAE1DAE1EAE1FAEE9971BE000
:10E93000115071F09E0125563F4F44E050E0BE015A
:10E940006B587F4FCE0183569F4F0E945FD0F0CF10
:10E9500080911607811167C0C356DF4FE880F980A8
:10E96000CD59D040F4E6EF1AF108C556DF4F888143
:10E970009981CB59D040C756DF4F99838883C959B5
:10E98000D04084E690E0C356DF4F99838883CD5909
:10E99000D0409E0125563F4F44E050E06FED72E0BD
:10E9A000CE0183569F4F0E945FD09E0125563F4F58
:10E9B00042E050E0BE0167567F4FCE0183569F4F25
:10E9C0000E945FD0E6EEFDE184918F010F5F1F4F43
:10E9D000882321F00E94E193F801F6CFB70180E08F
:10E9E0009AE10E946EC5C756DF4F48815981C959C7
:10E9F000D04060E070E083EF99E10E9434C5E0EF21
:10EA0000F9E184918F010F5F1F4F882321F00E944D
:10EA1000E193F801F6CFC7010E94226A9091160790
:10EA2000892B809316079091160781E08927C65598
:10EA3000DF4F0FB6F894DEBF0FBECDBFDF91CF9191
:10EA40001F910F91FF90EF90DF90CF90BF90AF900C
:10EA50009F908F900895FF920F931F93CF93DF9312
:10EA60008C01EB01F42E80E20E94E1938FEFF81607
:10EA700011F084E501C082E40E94E1938AE30E94E0
:10EA8000E193F801608171818281938142E00E946B
:10EA90008797488159816A817B818FE49DE10E943B
:10EAA00051C562E070E080E090E0DF91CF911F916E
:10EAB0000F91FF900C942DB78F929F92AF92BF92BF
:10EAC000CF92DF92EF92FF920F931F93CF93DF933A
:10EAD000F0E2FF2EE12CAE2DB0E0BD016F0D711DF7
:10EAE000759567956E1511F0F6120BC0E2E3FBE128
:10EAF00065917491072E000C880B990B0E945DE6BE
:10EB000062C09B0121503109220F331F220F331F96
:10EB1000F901EC54F54E05911491AB01440F551FCA
:10EB2000440F551FFA01EC54F54EC591D49180174E
:10EB3000910714F4F62ED1CFC817D90714F4E62E96
:10EB4000CACFF901EA54F54EE590F490FA01EA547F
:10EB5000F54EC590D490BC01601B710B072E000CC4
:10EB6000880B990B0E945DE64B015C01B6016E19A2
:10EB70007F09072E000C880B990B0E945DE69B0114
:10EB8000AC01C501B4010E94BCE64B015C01C01B95
:10EB9000D10BBE01DD0F880B990B0E945DE69B0136
:10EBA000AC01C501B4010E947FEB4B015C01B701D0
:10EBB000FF0C880B990B0E945DE69B01AC01C5011F
:10EBC000B4010E94A3EADF91CF911F910F91FF90B2
:10EBD000EF90DF90CF90BF90AF909F908F9008956F
:10EBE0000F931F93CF93DF93CDB7DEB728970FB660
:10EBF000F894DEBF0FBECDBF60914A0470914B0404
:10EC0000072E000C880B990B0E945DE66D837E83B6
:10EC10008F83988780914C0490914D04A0914E046D
:10EC2000B0914F0489839A83AB83BC834DEFBE01BF
:10EC30006B5F7F4FCE0101960EDF609144047091AF
:10EC40004504072E000C880B990B0E945DE66D832E
:10EC50007E838F8398878091460490914704A0918A
:10EC60004804B091490489839A83AB83BC834FEFF6
:10EC7000BE016B5F7F4FCE010196EDDEE7E5FDE162
:10EC800084918F010F5F1F4F882321F00E94E19331
:10EC9000F801F6CFE0914E07F0E0E45BF84F6081B9
:10ECA00070E080E090E00E946D97E2E5FDE18491E4
:10ECB0008F010F5F1F4F882321F00E94E193F8011D
:10ECC000F6CF60914D0770E080E090E00E946D9774
:10ECD00028960FB6F894DEBF0FBECDBFDF91CF915F
:10ECE0001F910F9108950F930FB70F9300916E002E
:10ECF0000B7F00936E0078940F930BB70F930CB7B4
:10ED00000F921F922F933F934F935F936F937F9335
:10ED10008F939F93AF93BF93EF93FF931124EFD201
:10ED2000FF91EF91BF91AF919F918F917F916F91E3
:10ED30005F914F913F912F911F900F900CBF0F91BA
:10ED40000BBF0F910460F89400936E000F910FBFFA
:10ED50000F911895CF92DF92EF92FF92C0904604E8
:10ED6000D0904704E0904804F09049046091440436
:10ED70007091450466507109072E000C880B990BA1
:10ED80000E945DE69B01AC01C701B6010E9457E6F7
:10ED900087FF1FC020E030E040E050E4C701B6012B
:10EDA0000E94A3EA0E94ECEB7093860760938507AC
:10EDB0000E94F258DC01CB01805A9541AF4FBF4F02
:10EDC0008093810790938207A0938307B093840771
:10EDD00008C0109281071092820710928307109248
:10EDE0008407FF90EF90DF90CF900895CF92DF924D
:10EDF000EF92FF92C0904C04D0904D04E0904E04EE
:10EE0000F0904F0460914A0470914B04695071096D
:10EE1000072E000C880B990B0E945DE69B01AC014C
:10EE2000C701B6010E9457E687FF1FC020E030E00F
:10EE300040EA50E4C701B6010E94A3EA0E94ECEB4D
:10EE40007093800760937F070E94F258DC01CB012A
:10EE500088549747AF4FBF4F80937B0790937C07B1
:10EE6000A0937D07B0937E0708C010927B07109295
:10EE70007C0710927D0710927E07FF90EF90DF9045
:10EE8000CF9008958F929F92AF92BF92CF92DF92D0
:10EE9000EF92FF920F931F93CF93DF93F0E4FF2E37
:10EEA000E12CAE2DB0E0BD016F0D711D759567951C
:10EEB0006E1511F0F6120BC0E4EAFCE16591749155
:10EEC000072E000C880B990B0E945DE662C09B0127
:10EED00021503109220F331F220F331FF901EA5548
:10EEE000F44E05911491AB01440F551F440F551F6B
:10EEF000FA01EA55F44EC591D4918017910714F4A4
:10EF0000F62ED1CFC817D90714F4E62ECACFF901CF
:10EF1000E855F44EE590F490FA01E855F44EC590AA
:10EF2000D490BC01601B710B072E000C880B990B51
:10EF30000E945DE64B015C01B6016E197F09072E48
:10EF4000000C880B990B0E945DE69B01AC01C5018A
:10EF5000B4010E94BCE64B015C01C01BD10BBE0199
:10EF6000DD0F880B990B0E945DE69B01AC01C5018A
:10EF7000B4010E947FEB4B015C01B701FF0C880BD1
:10EF8000990B0E945DE69B01AC01C501B4010E9492
:10EF9000A3EADF91CF911F910F91FF90EF90DF9047
:10EFA000CF90BF90AF909F908F90089560E0809138
:10EFB00091079091920780DD60934C0470934D040B
:10EFC00080934E0490934F0480918F079091900707
:10EFD00059DF6093460470934704809348049093EC
:10EFE0004904A8951092490708957F928F929F92A5
:10EFF000AF92BF92CF92DF92EF92FF920F931F9347
:10F00000CF93DF9320E030E048E452E460914C0479
:10F0100070914D0480914E0490914F040E94C9EC70
:10F0200018164CF4EAE3FBE1E491C1E001C0CC0F17
:10F03000EA95EAF701C0C0E084E3E82E8BE1F82E00
:10F040000AE31BE196E0A92E912CD0E0CC24C394D6
:10F05000D12CF7017490F801849077FC23C0892D9E
:10F0600090E0082C02C0959587950A94E2F780FD00
:10F0700019C0BE01082C02C0759567950A94E2F785
:10F080006170B62EB1946B2D872D0E94FCB56B2D4F
:10F0900070E0872D0E9466B6C60101C0880F8A9471
:10F0A000EAF7982AAA94FFEFEF1AFF0A0F5F1F4FA3
:10F0B000A110CFCFDF91CF911F910F91FF90EF90D3
:10F0C000DF90CF90BF90AF909F908F907F900895EA
:10F0D0000F931F9380912B07813019F40E94F258EF
:10F0E00008C06091270770912807809129079091A7
:10F0F0002A0700915307109154072091550730912A
:10F100005607601B710B820B930B28EE33E040E037
:10F1100050E00E9445EA80914F0790915007A091DE
:10F120005107B0915207BC01CD01620F731F841FBC
:10F13000951F1F910F91089510922B07109253075E
:10F1400010925407109255071092560710922707F5
:10F15000109228071092290710922A0710924F0741
:10F160001092500710925107109252070895809103
:10F170002B078130E1F0823051F4AADF60934F0712
:10F1800070935007809351079093520701C0D4DFCA
:10F1900081E080932B070E94F2586093530770938D
:10F1A0005407809355079093560781E0089580E0B7
:10F1B000089580912B07813079F482E080932B07AA
:10F1C0000E94F258609327077093280780932907BD
:10F1D00090932A0781E0089580E0089580912B079D
:10F1E0008150823010F080E0089510922B070E9429
:10F1F000F25860932707709328078093290790930C
:10F200002A0781E008951092480780E090E00E946C
:10F21000E75910924504109244049CDDDFDF80E042
:10F2200090E00E94E75910924C072C9810924504E8
:10F230001092440410924D078091020180728093D5
:10F2400000010895DF92EF92FF920F931F93CF93E7
:10F25000DF93F82ED62EE72E8A018091270288238D
:10F2600009F439C0E1EDFDE18491EF012196882395
:10F2700021F00E94E193FE01F7CFED2DFE2D849148
:10F28000EF012196882321F00E94E193FE01F7CF40
:10F29000E5E4FBE18491EF012196882321F00E94AF
:10F2A000E193FE01F7CFF7FC0BC06F2DFF0C770B3E
:10F2B000880B990B0E946D978AE00E94E1930BC026
:10F2C000E0E4FBE18491EF012196882321F00E9484
:10F2D000E193FE01F7CF80915707811108C010928A
:10F2E000270281E080935707C8010E94D8A0DF91D0
:10F2F000CF911F910F91FF90EF90DF9084CFEF920D
:10F30000FF920F931F93CF93DF9380912A028F3741
:10F31000A0F08F5790914C079093A207992311F07A
:10F320002C9A01C02C9820914D072093A107909111
:10F330000201222369F090950BC09091A2078917D2
:10F3400008F02C989091A107891728F0909102015C
:10F350009072909300018F5F80932A029091A00792
:10F3600081E089278093A0078091290285301CF4D1
:10F37000C1E0C80F01C0C0E0823009F4B4C054F449
:10F38000882301F1813009F0E3C088E080937B009D
:10F3900085E4C0C0843009F4C5C00CF4B7C0853022
:10F3A00009F0D6C090919F07911102C080939F07EA
:10F3B00080919F07815080939F07882309F4C8C0DC
:10F3C000C5E0C6C0809128028F5F80311CF4809315
:10F3D0002802BEC01092280280914907811113C0F3
:10F3E000809195079091960790939207809391074B
:10F3F00080919307909194079093900780938F0743
:10F4000081E0809349078AE0E5E9F7E0DF011D929A
:10F410008A95E9F71092940710929307009191074B
:10F420001091920711950195110980914A049091CC
:10F430004B04D1E0181619062CF080914C0781116D
:10F4400001C0D0E08091320590913305919581956E
:10F4500091098017910734F44DED5CE16EEF7CE18A
:10F4600080E0F0DE80911C0290911D0291958195C3
:10F4700091090817190744F4DD2331F040E15DE1FB
:10F4800061E37DE180E0DEDE8091440490914504FB
:10F4900011E0181619062CF080914D07811101C05A
:10F4A00010E0E0908F07F0909007809130059091E8
:10F4B00031058E159F0534F04DEE5CE16EEF7CE179
:10F4C0008FEFC0DE80911A0290911B02E816F906B8
:10F4D0000CF43EC01123E1F140E25DE161E37DE126
:10F4E0008FEFB0DE35C080917A0086FD2EC080910E
:10F4F0007800909179002091950730919607820FBE
:10F50000931F909396078093950722C088E080937D
:10F510007B0086E480937C0080917A0080648093F5
:10F520007A0016C080917A0086FD11C08091780023
:10F53000909179002091930730919407820F931F47
:10F54000909394078093930703C0C2E001C0C4E086
:10F55000C09329028091370581110E94E2BD8091FC
:10F560004A0790914B070097A9F0019790934B079A
:10F5700080934A07892B71F483E49DE19093A4075B
:10F580008093A307DF91CF911F910F91FF90EF9090
:10F590000C940D94DF91CF911F910F91FF90EF90FC
:10F5A00008952F923F924F925F926F927F928F9227
:10F5B0009F92AF92BF92CF92DF92EF92FF920F9302
:10F5C0001F93CF93DF9300D01F92CDB7DEB75C01BE
:10F5D0007A8369834A01170107FD07C0802F002E37
:10F5E000000C990B9C838B8304C0E1E0F0E0FC836A
:10F5F000EB83F90140805180628073808B819C8114
:10F60000880F991F880F991F9C838B838957984F68
:10F610007C01A3019201FC0160817181828193814F
:10F620000E9457E6882391F0F7014082518262825E
:10F63000738211E020E030E0A901C301B2010E9411
:10F64000C9EC18160CF010E0F5011083F50180816B
:10F650008230D1F0833009F45EC0813009F07CC083
:10F66000EB81FC81E957F84F208131814281538140
:10F67000F40160817181828193810E9457E687FD48
:10F680006BC082E0F50180838B819C818957984F04
:10F690009C838B83B60180E090E00E945BE69B0137
:10F6A000AC01EB81FC8160817181828193810E9438
:10F6B000A2EA9B01AC01F401608171818281938196
:10F6C0000E94C9EC87FD14C00E94F2586B017C01B6
:10F6D0009101A8EEB3E00E9493EAC60ED71EE81E81
:10F6E000F91EE981FA81C082D182E282F38234C0BC
:10F6F0000E94F258E981FA81C080D180E280F380D3
:10F70000DC01CB018C199D09AE09BF09B7FD24C0EE
:10F7100083E0F50180830F3F19F046EA5CE102C007
:10F7200049EB5CE16DEC7CE1802F0F900F900F9026
:10F730000F90DF91CF911F910F91FF90EF90DF908D
:10F74000CF90BF90AF909F908F907F906F905F9081
:10F750004F903F902F9076CD0F900F900F900F907D
:10F76000DF91CF911F910F91FF90EF90DF90CF909D
:10F77000BF90AF909F908F907F906F905F904F90D1
:10F780003F902F9008954F925F926F927F928F9249
:10F790009F92AF92BF92CF92DF92EF92FF920F9320
:10F7A0001F93CF93DF93CDB7DEB760970FB6F89472
:10F7B000DEBF0FBECDBF80914907811117C0609693
:10F7C0000FB6F894DEBF0FBECDBFDF91CF911F9172
:10F7D0000F91FF90EF90DF90CF90BF90AF909F90F0
:10F7E0008F907F906F905F904F900895DFDB0E9425
:10F7F000F2584B015C0160914A0470914B04072E52
:10F80000000C880B990B0E945DE669837A838B83D9
:10F810009C8344E1C42ED12C5CE3E52EF12C00E066
:10F820009E012F5F3F4F4CE454E067E777E086E7A7
:10F8300097E0B7DEC0904C04D0904D04E0904E04A9
:10F84000F0904F046091340570913505072E000C3F
:10F85000880B990B0E945DE69B01AC01C701B601C4
:10F860000E94C9EC18160CF009C160911E0270913B
:10F870001F02072E000C880B990B0E945DE69B016E
:10F88000AC01C701B6010E9457E687FFF7C000919F
:10F890004A0410914B04B801012E000C880B990BFF
:10F8A0000E945DE6A70196010E94A2EA2B013C019D
:10F8B00020ED3CEC4CE45DE3609140077091410722
:10F8C00080914207909143070E94BCE66D837E833E
:10F8D0008F83988720916D0730916E0740916F0755
:10F8E00050917007C701B6010E94A2EA9B01AC01CA
:10F8F0006D817E818F8198850E94BCE66D837E83B9
:10F900008F83988723E333E343E75FE360916907DD
:10F9100070916A0780916B0790916C070E94BCE61A
:10F920009B01AC016D817E818F8198850E94A3EA45
:10F930006D837E838F8398876093690770936A07CE
:10F9400080936B0790936C07C0926D07D0926E07FF
:10F95000E0926F07F092700720E030E040E251E45F
:10F96000C301B2010E94C9EC18160CF431C220E0A8
:10F9700030E040E251ECC301B2010E9457E687FD3E
:10F980002FC2012B09F42CC28091680781112CC26F
:10F990002091640730916507409166075091670791
:10F9A00029873A874B875C8720913C0730913D0738
:10F9B00040913E0750913F07C301B2010E94BCE64F
:10F9C0006B017C01A301920169857A858B859C85F9
:10F9D0000E94A3EA69877A878B879C876093640774
:10F9E00070936507809366079093670720913807A7
:10F9F0003091390740913A0750913B070E94BCE68D
:10FA0000A70196010E94A3EA2D813E814F8158856E
:10FA10000E94A2EA6B017C0120E030E04FE753E452
:10FA20000E94C9EC20E030E0A90118160CF4E3C1F3
:10FA3000C701B6010E9457E687FD07C0C701B6019E
:10FA40000E94E7EB759567951AC020E030E0A901A8
:10FA5000C301B2010E9457E687FF10C0A3019201C3
:10FA600069857A858B859C850E94A2EA60936407EC
:10FA700070936507809366079093670760E06093D3
:10FA80004C0780917B0790917C07A0917D07B091F6
:10FA90007E070097A105B10521F1A5019401281B5E
:10FAA000390B4A0B5B0B57FD1CC060917F077091AF
:10FAB000800780E090E00E945BE69B01AC016091D2
:10FAC0004C0470914D0480914E0490914F040E941B
:10FAD00057E687FF82C145E85BE167E97BE180E0AB
:10FAE000B1DB8091440790914507A0914607B09102
:10FAF0004707A5019401281B390B4A0B5B0B57FDE7
:10FB00000FC073DAD501C4018C53964FAF4FBF4F6E
:10FB10008093440790934507A0934607B093470707
:10FB20008091810790918207A0918307B09184070B
:10FB30000097A105B10511F1881A990AAA0ABB0A12
:10FB4000B7FC1CC0609185077091860780E090E04B
:10FB50000E945BE69B01AC016091460470914704F2
:10FB600080914804909149040E9457E687FF20C184
:10FB700043E65BE166E77BE18FEF64DB6091440481
:10FB800070914504072E000C880B990B0E945DE6CE
:10FB900069837A838B839C8395E0C92ED12C24E1E1
:10FBA000E22EF12C0FEF9E012F5F3F4F46E454E011
:10FBB00061E777E085E797E0F4DCC0904604D090F9
:10FBC0004704E0904804F090490420E030E040EA27
:10FBD00050E4C701B6010E94C9EC87FDE5C020E0F2
:10FBE00030E04CED52E4C701B6010E9457E618160A
:10FBF0000CF4DAC06091440470914504072E000CA7
:10FC0000880B990B0E945DE6A70196010E94A2EA6B
:10FC10004B015C0120913407309135074091360744
:10FC2000509137070E94BCE669877A878B879C874B
:10FC300020916007309161074091620750916307FE
:10FC4000C501B4010E94A3EA6D837E838F839887E8
:10FC500060936007709361078093620790936307D6
:10FC6000209130073091310740913207509133078E
:10FC70000E94BCE66D877E878F87988B20ED3CECD9
:10FC80004CE45DE360912C0770912D0780912E0765
:10FC900090912F070E94BCE62B013C0120915C074C
:10FCA00030915D0740915E0750915F07C701B60133
:10FCB0000E94A2EA9B01AC01C301B2010E94BCE612
:10FCC0002B013C0123E333E343E75FE360915807F3
:10FCD0007091590780915A0790915B070E94BCE68A
:10FCE0009B01AC01C301B2010E94A3EA2B013C01BC
:10FCF000609358077093590780935A0790935B0756
:10FD0000C0925C07D0925D07E0925E07F0925F07B9
:10FD10002D853E854F85588969857A858B859C859B
:10FD20000E94A3EAA30192010E94A2EA6B017C0156
:10FD300020E030E04FE753E40E94C9EC20E030E0DF
:10FD4000A9011816C4F5C501B4010E94C9EC181622
:10FD500084F4A50194016D817E818F8198850E9434
:10FD6000A2EA6093600770936107809362079093A3
:10FD700063076FE71AC020E030E0A901C501B401B4
:10FD80000E9457E687FF10C0A50194016D817E8116
:10FD90008F8198850E94A2EA609360077093610743
:10FDA000809362079093630760E060934D0707CDEF
:10FDB0000E94AA76E3CEC701B6010E9457E687FDEE
:10FDC000DACFC701B6010E94E7EB75956795EDCFD5
:10FDD00081E0809368076FE752CE80E007D881CE3C
:10FDE00081E0809368074ACE1092680719861A86C8
:10FDF0001B861C86D9CDC301B2010E94C9EC18161E
:10FE000054F7A301920169857A858B859C850E94B0
:10FE1000A2EA6093640770936507809366079093E6
:10FE200067076FE72CCE90916F00292F227091FF0A
:10FE300005C090916F009D7F90936F0034E0839F89
:10FE4000C0011124FC01EE57FF4E408151816281B7
:10FE50007381FC01E55EF84F4083518362837383B5
:10FE600081E080931A07222329F080916F0082603D
:10FE700080936F000895BC012091180730911907F5
:10FE800040911807509119072417350711F09A016E
:10FE9000F7CF81E02617370709F080E008958F92A9
:10FEA0009F92AF92BF92CF92DF92EF92FF921F93F9
:10FEB000CF93DF93C82F83ED9BE09093AF0980939E
:10FEC000AE091092EF0B82E090E0A0E0B0E08093EA
:10FED000D80B9093D90BA093DA0BB093DB0B109255
:10FEE000AD091092A9091092AA091092AB091092BB
:10FEF000AC098FEF9FEFDC018093A5099093A609D1
:10FF0000A093A709B093A809CC2379F1C53008F0D4
:10FF1000F8C040E060E070E0CB010E94BBD18823D4
:10FF200009F4EFC020E1C29FC00111248B56984F05
:10FF3000FC01E254FE4F20812F7709F0E2C03C968D
:10FF4000408151816281738144365105610571059B
:10FF500008F4D7C03497C080D180E280F380C11408
:10FF6000D104E104F10421F4CCC0C12CD12C7601E0
:10FF700040E0C701B6010E94BBD1182F882309F4C5
:10FF8000C0C08091B0079091B1078115924009F0EF
:10FF9000B8C0A091B507AA2309F4B3C06091B30714
:10FFA0007091B4076115710509F4ABC02091B207D7
:10FFB000222309F4A6C0A093EA0B2093DC0B80E077
:10FFC00030E041E050E0C82FFA01082E02C0EE0FE9
:10FFD000FF1F0A94E2F72E173F0739F08F5FC830F2
:10FFE00091F789E08093E50B8CC08093E50B20911D
:10FFF000BB073091BC072115310519F040E050E0F6
:020000021000EC
:1000000008C02091C9073091CA074091CB07509191
:10001000CC072093DD0B3093DE0B4093DF0B509326
:10002000E00B46015701860E971EA11CB11C809261
:10003000EB0B9092EC0BA092ED0BB092EE0BE091DB
:10004000B607F091B707F093F10BE093F00BB0E037
:100050000E9483EA860E971EA81EB91E8092F20B9C
:100060009092F30BA092F40BB092F50B85E0EE0F9B
:10007000FF1F8A95E1F7E150FE4FEF2FFF27E6952E
:100080008E0E9F1EA11CB11C8092E60B9092E70B76
:10009000A092E80BB092E90B2091B8073091B90714
:1000A0002115310521F0A90160E070E008C0409100
:1000B000C5075091C6076091C7077091C807D7015F
:1000C000C60188199909AA09BB09840F951FA61FA3
:1000D000B71F04C0B695A79597958795CA95D2F78F
:1000E0008093E10B9093E20BA093E30BB093E40BAE
:1000F000853F2FE09207A105B10528F48CE080939D
:10010000EF0B10E01AC0853F9F4FA105B10510F419
:1001100080E111C08091D1079091D207A091D307BF
:10012000B091D4078093F20B9093F30BA093F40B50
:10013000B093F50B80E28093EF0B812FDF91CF918D
:100140001F91FF90EF90DF90CF90BF90AF909F9066
:100150008F900895682F8AE99FE00C94D44ACF923B
:10016000DF92EF92FF921F93CF93DF931092320AA8
:100170008091650A882321F082E69AE00E94FC982B
:100180001092D70B1092D40B85E38093D30B0E946F
:10019000F258EB01A89561E08091D30B0E942AB63A
:1001A00083ED9BE00E945D9A2398229A219A209ADF
:1001B000289A85E08093D50B82E58CBD1DBC1AE0A2
:1001C0008FEF0E94629A1150D9F720E030E0A90128
:1001D00060E083ED9BE00E94679A182F8093D60B16
:1001E000813049F00E94F2586C1B7D0B613D7740D5
:1001F00060F381E054C02AEA31E040E050E068E07A
:1002000083ED9BE00E94679A82FF03C01093D70B97
:100210000EC014E00E94759F8093D60B1150D1F749
:100220008A3A11F082E03BC082E08093D70B809144
:10023000D70B823021F0C12CD12C760105C0C12C06
:10024000D12CE12C80E4F82E20E030E0A90167E316
:1002500083ED9BE00E94679AA701960169E283ED16
:100260009BE00E94679A8093D60B882349F00E94F6
:10027000F2586C1B7D0B613D774030F38AE00FC074
:100280008091D70B823011F520E030E0A9016AE3BC
:1002900083ED9BE00E94679A882351F088E0809369
:1002A000D40B83ED9BE00E945D9AE6EEFDE119C060
:1002B0000E94759F807C803C19F483E08093D70B6B
:1002C0000E94759F0E94759F0E94759F83ED9BE021
:1002D0000E945D9A1092D50B81E0E1DD811131C061
:1002E00015C08491EF012196882321F00E94E193AB
:1002F000FE01F7CFE8EDFDE18491EF01219688231F
:1003000009F456C00E94E193FE01F6CF80E0C7DDFC
:10031000811117C0E1EDFDE18491EF012196882361
:1003200021F00E94E193FE01F7CFEDEBFDE1849116
:10033000EF012196882309F43BC00E94E193FE015E
:10034000F6CF68ED7BE082E69AE00E94A9988111E1
:1003500016C0E1EDFDE18491EF012196882321F0A3
:100360000E94E193FE01F7CFECEAFDE18491EF01F9
:1003700021968823E9F00E94E193FE01F7CF81E006
:100380008093320AE6EEFDE18491EF012196882305
:1003900021F00E94E193FE01F7CFE0EAFDE18491B4
:1003A000EF012196882321F00E94E193FE01F7CF0F
:1003B0008BE1E2E6FAE0A1E8BAE001900D928A95BD
:1003C000E1F78091600A9091610A9093800A80938E
:1003D0007F0ADF91CF911F91FF90EF90DF90CF9038
:1003E000089580913F0E823041F48BE89DE1909317
:1003F000A4078093A3070E940D940E94F258609373
:10040000430E7093440E8093450E9093460E809158
:10041000320A882319F081E08093310A81E08093C9
:100420003F0E0895CF93DF931092310A83E08093BB
:100430003F0E80918C0E8823B1F0E3E8FDE18491BA
:10044000EF01882341F0082E000C990B83DE2196E2
:10045000FE018491F6CF8DE090E07CDE8AE090E0B2
:10046000DF91CF9177CEE7E8FDE18491EF0188231A
:1004700091F3082E000C990B6DDE2196FE018491FC
:10048000F6CF8F929F92AF92BF92CF92DF92EF9270
:10049000FF920F931F93CF93DF9300D01F92CDB79E
:1004A000DEB7FC018381813079F5818181FF2CC029
:1004B00081899289A389B489892B8A2B8B2B09F492
:1004C00048C07F0140E050E0BA01CF010E9412987D
:1004D0008823D1F0F70185889688A788B08CC18CD5
:1004E000D28C82E090E0A0E0B0E0F60180839183BE
:1004F000A283B3839E012F5F3F4FB501A401C601C4
:100500000E9484D2811102C080E03CC000E010E073
:100510009801B501A401C6010E94F3D18823A1F37B
:1005200089809A80AB80BC80F6018789803141F454
:10053000F8EF8F16FFEF9F06A104B10460F4DACF45
:1005400088EF88168FEF9806A8068FE0B80618F493
:10055000D1CF81E017C0F701158A168A178A108E4D
:10056000118A128A138A148A818180688183C70163
:100570000E94D2D3882341F240E050E0BA01C70183
:100580000E9412980F900F900F900F90DF91CF91D3
:100590001F910F91FF90EF90DF90CF90BF90AF90A1
:1005A0009F908F9008951092340A1092310A809192
:1005B000FD0B882321F08AEF9BE00C94FC980895B2
:1005C0002F923F924F925F926F927F928F929F9263
:1005D000AF92BF92CF92DF92EF92FF920F931F9351
:1005E000CF93DF93CDB7DEB7C257D1090FB6F894DA
:1005F000DEBF0FBECDBF8C013B014A014DB75EB7D8
:10060000E1965FAF4EAFE197AD961FAEAD971B0180
:1006100054E0250E311C7E018FE5E80EF11C9DEEA5
:10062000492E92E0592EE0E4F0E0EC0FFD1F3496E5
:10063000E396FFAFEEAFE397F3018781823008F4D2
:1006400062C184859585A685B7858F719927AA276C
:10065000BB27892B8A2B8B2B09F055C11092420A9C
:1006600042E45AE0BE016F5F7F4FC1010E946AD32E
:1006700018160CF048C18C85982F9871903129F488
:100680002091AF0C2150223078F42981222309F4E3
:100690003AC1253E89F22E3279F22091420A2E3259
:1006A00059F28A7049F6B8C04DB75EB7AF965FAFE2
:1006B0004EAFAF97BE016F5F7F4FC7010E9465D1FC
:1006C0000115110521F0F801808181119BC021E005
:1006D00081E090E0F70101900020E9F73197EE19F1
:1006E000FF098E0F9F1F02964DB75EB7481B590B2F
:1006F0000FB6F8945EBF0FBE4DBF8DB79EB7019683
:100700005C01211102C0B80102C062E273E0C501C0
:100710000E9407EEB701C5010E94E8ED62E273E0B6
:10072000C5010E94E8ED25961FAE259728961FAEBD
:10073000289724961FAE1EAE249722965FAE4EAE2B
:10074000229721E0A701B101E3968EAD9FADE3971B
:100750000E94889E81112AC08091AF0C811126C011
:10076000E6EEFDE184916F019FEFC91AD90A882353
:1007700021F00E94E193F601F5CFEFE6FDE18491CF
:100780006F012FEFC21AD20A882321F00E94E19351
:10079000F601F5CF6701F60181916F01882319F009
:1007A0000E94E193F8CF8AE00E94E1938BE1FE0181
:1007B000EC5BFF4FDE01959601900D928A95E1F773
:1007C00024968EAD9FAD24979CA38BA35AA249A2D9
:1007D00040E050E0BE016F5D7F4FC501F1DECE010C
:1007E00081960E94B5A0CE01805C9F4F0E94B5A06B
:1007F000AF964EAD5FADAF970FB6F8945EBF0FBE2C
:100800004DBF1ACFF80101900020E9F73197CF01D1
:10081000801B910B20E05ECF81E0903109F080E0F9
:100820008093330A903141F08985873409F004CFF1
:100830008A858E3709F400CF8091AF0C813029F082
:100840008230D9F18111F8CE0AC08091B00C90911C
:10085000B10C01969093B10C8093B00CEDCEBE011B
:100860006F5F7F4F85E39AE00E9465D10115110506
:1008700029F485E3C82E8AE0D82E09C06801F60164
:1008800081916F018823A9F30E94E193F8CFF601CB
:1008900081916F01882319F00E94E193F8CF80E2E3
:1008A0000E94E1936D8D7E8D8F8D98A14AE00E940C
:1008B00002978AE00E94E193BFCEBE016F5F7F4F37
:1008C00085E39AE00E9465D18114910441F065E3CB
:1008D0007AE0C4010E94D5ED892B69F414C0AD966D
:1008E000FFADAD978F2F90E02091BC0F3091BD0FE1
:1008F0008217930741F0AD962FADAD972F5FAD9660
:100900002FAFAD9799CEE1968EAD9FADE1970FB623
:10091000F8949EBF0FBE8DBFCE58DF4F0FB6F89430
:10092000DEBF0FBECDBFDF91CF911F910F91FF9022
:10093000EF90DF90CF90BF90AF909F908F907F907F
:100940006F905F904F903F902F9008950F931F935B
:10095000CF93DF93CDB7DEB76F970FB6F894DEBFB6
:100960000FBECDBF8B0122E02093AF0C9093BD0F43
:100970008093BC0F81E89AE00E94599A8BE1E1E8EC
:10098000FAE0DE01159601900D928A95E1F78091CB
:100990007F0A9091800A9C838B838DEE92E09A83EC
:1009A0008983A801BE016F5F7F4F80E090E008DE81
:1009B000CE0101960E94B5A06F960FB6F894DEBFE7
:1009C0000FBECDBFDF91CF911F910F9108952F9250
:1009D0003F924F925F926F927F928F929F92AF92CF
:1009E000BF92CF92DF92EF92FF920F931F93CF931C
:1009F000DF93CDB7DEB76F970FB6F894DEBF0FBEAB
:100A0000CDBF6C012DB63EB61D8218861C821B829E
:100A10008DEE92E09A838983FB0180819E012F5F96
:100A20003F4F39018F3241F08DE79AE0F601918313
:100A30008083F62E172F64C08EE59AE0F60191832D
:100A400080838B010F5F1F4F0115110509F456C0FC
:100A50004DB65EB66FE270E0C8010E94F3ED4C0146
:100A60000817190708F048C07C01E01AF10AFF24B2
:100A7000C70101962DB73EB7281B390B0FB6F89466
:100A80003EBF0FBE2DBF8DB79EB701965C01A7017B
:100A9000B8010E941CEEF501EE0DFF1D1082F6015B
:100AA000608171816115710511F06C5F7F4F21E0EC
:100AB000A501CE0105960E94889E811111C0B50145
:100AC0008BE59DE10E9487C58EE20E94E1938AE05A
:100AD0000E94E1930FB6F8945EBE0FBE4DBE0EC0ED
:100AE000F6017182608284010F5F1F4F0FB6F89488
:100AF0005EBE0FBE4DBEA8CFF02E02C0F12C10E09E
:100B0000C3010E94B5A08F2D912F0FB6F8943EBE61
:100B10000FBE2DBE6F960FB6F894DEBF0FBECDBFD1
:100B2000DF91CF911F910F91FF90EF90DF90CF90C9
:100B3000BF90AF909F908F907F906F905F904F90FD
:100B40003F902F900895CF92DF92EF92FF920F93F4
:100B50001F93CF93DF9388E50E94424CD82E89E4FF
:100B60000E94424CC82E882319F00E94DB4B1CC007
:100B7000DD20C1F00E940B4C20E030E040E251E467
:100B80000E94A2EA20E030E048EC51E40E94A3EA8F
:100B90002AE037ED43EA5CE30E94BCE60E94E7EB03
:100BA000653010F01FEF01C0162F89E50E94424CFE
:100BB000082F8AE40E94424CC82F882319F00E9413
:100BC000DB4B1CC00023C1F00E940B4C20E030E046
:100BD00040E251E40E94A2EA20E030E048EC51E417
:100BE0000E94A3EA2AE037ED43EA5CE30E94BCE6F8
:100BF0000E94E7EB653010F0DFEF01C0D62F8AE5E9
:100C00000E94424CE82E811105C081E50E94424CB1
:100C1000F82E01C0F12CC11001C0C0E02C2F30E033
:100C2000D11001C000E0200F311D2130310521F429
:100C3000E1101AC0F11018C0E1EDFDE18491EF015F
:100C40002196811103C0E7E9F0E204C00E94E1931C
:100C5000FE01F4CF8491EF012196882309F455C059
:100C60000E94E193FE01F6CF17FD02C0D7FF17C027
:100C7000E1EDFDE18491EF012196811103C0E8E7E8
:100C8000F0E204C00E94E193FE01F4CF8491EF01F1
:100C900021968823D1F10E94E193FE01F7CF0E94B3
:100CA0000B4C9B01AC01012F110F110BAD2FDD0F70
:100CB000BB0BFF2099F085E0809FF001819FF00D34
:100CC0001124EA0FFB1FEE0FFF1FEE0FFF1FEA5369
:100CD000FF4E608171818281938103C060E070E08A
:100CE000CB01E5E0E09FE001E19FD00D1124CA0FA8
:100CF000DB1FCC0FDD1FCC0FDD1FCA53DF4E0E9460
:100D0000A3EA688379838A839B83DF91CF911F91C4
:100D10000F91FF90EF90DF90CF90089580916F003A
:100D2000982F927081FF05C080916F008D7F809316
:100D30006F008091B4098093B3098093B2098093C6
:100D4000B10984E68093B00928EE33E030934B0775
:100D500020934A07992329F080916F008260809345
:100D60006F0081E080931A070E94126A0E94C3C933
:100D700080917C10882321F084EA98E10E947FC64C
:100D80008CE0E4EAF8E1A2E3B4E001900D928A95E8
:100D9000E1F70C9495932F923F924F925F926F924E
:100DA0007F928F929F92AF92BF92CF92DF92EF92FB
:100DB000FF920F931F93CF93DF93CDB7DEB7CD5440
:100DC000D1090FB6F894DEBF0FBECDBF85E40E94F7
:100DD0008B4C882321F00E94DB4B7B0102C0E12C6D
:100DE000F12C83E40E948B4C882321F00E94DB4B82
:100DF0006AA302C005E00AA385E50E948B4C882304
:100E000019F00E94FC4B03C085E50E94424C8CA760
:100E1000F7FC07C0812C912C16E1A12E13E4B12E12
:100E200006C0812C912CBCE8AB2EB2E4BB2E83E52E
:100E30000E948B4C882321F00E940B4C4B015C01DB
:100E4000E114F10411F410924E0710923F10ED825C
:100E50000E94F2582B013C011D8117FF05C00CE3D5
:100E600010E022E0298304C003E210E035E039837A
:100E7000D301C2018C53964FAF4FBF4F80934407AD
:100E800090934507A0934607B093470761E06E0D26
:100E9000623080F0E5EEFFE184918F010F5F1F4F1C
:100EA0001A830983882309F45FC30E94E193E981CF
:100EB000FA81F2CFEFE0F0E284917F012FEFE21AA6
:100EC000F20A882321F00E94E193F701F5CF0E94F6
:100ED00003793D8137FF04C08FE780934D0708C039
:100EE0004D81E42F440FFF0BE45BF84F8FE78083C5
:100EF000C501B4010E94E7EB072E000C880B990B8B
:100F00000E945DE66A877B878C879D878981482F51
:100F100050E09801A8EEB3E00E9493EA6DA77EA787
:100F20008FA798AB8B019C01040D151D261D371D45
:100F30000AAF1BAF2CAF3DAF81E0809320021D8133
:100F40001F3F39F40FE41FE11FAF0EAF09E11FE1AE
:100F500006C00DE31FE11FAF0EAF06E01FE12296B2
:100F60001FAF0EAF22974CA25DA26EA27FA249AA2C
:100F70005AAA6BAA7CAA1DAA1EAA1FAA18AE19AE4D
:100F8000188E10E4198F0CE10A8F16E41B8F1C8E4B
:100F90001D8E1E8E1F8E1C8A1D8A1E8A1F8A188A0D
:100FA000198A1A8A1B8A19821A821B821C828FE76D
:100FB00090E0A0E0B0E08E839F83A887B987FFE729
:100FC000CF2ED12CE12CF12C18A619A61AA61BA6FF
:100FD00011E01F861E862D961FAE2D97212C312CD9
:100FE0002E961FAE2E970D81802F000F990B9C011E
:100FF000245B384F24963FAF2EAF2497880F991F5C
:10100000880F991FDC01A45BBB4FB9A3A8A3CA0139
:10101000052E000CAA0BBB0B28968CAF9DAFAEAF74
:10102000BFAF28974C5F5F4FCA01550FAA0BBB0B90
:101030002C968CAF9DAFAEAFBFAF2C97AAA10A2E56
:10104000000CBB0BBBA3AAA380912002882309F448
:1010500089C20E94F2584B015C01809149078823A4
:1010600009F4D4C00E94D6770D8107FD0CC0A8A159
:10107000B9A1BC912D96BFAF2D97E8A1F9A1218010
:10108000328003810BC0009146042D960FAF2D973F
:101090002090470430904804009149042E960FAFE9
:1010A0002E972D962FAD2D97322D432D2E965FAD79
:1010B0002E976C8D7D8D8E8D9F8D0E9457E687FFBC
:1010C0000AC02D960FAD2D970C8F2D8E3E8E2E962D
:1010D0000FAD2E970F8F288D398D4A8D5B8D2D96F4
:1010E0006FAD2D97722D832D2E969FAD2E970E945A
:1010F00057E687FF0AC02D960FAD2D97088F298ED2
:101100003A8E2E960FAD2E970B8F809144079091BB
:101110004507A0914607B0914707A5019401281BF8
:10112000390B4A0B5B0B57FD10C00E94F577D501B8
:10113000C4018C53964FAF4FBF4F80934407909399
:101140004507A0934607B09347072D962FAD2D97DF
:10115000322D432D2E965FAD2E976A857B858C852B
:101160009D851123E9F10E9457E687FF4FC0B50125
:10117000A4014419550966097709DB01CA01885899
:101180009341A109B109B7FD41C0D701C6010E8144
:101190001F8128853985801B910BA20BB30B1D8104
:1011A000B595A7959795879517FF03C080934D0731
:1011B00005C02496EEADFFAD2497808348A759A7BC
:1011C0006AA77BA70A850C8F1B851D8F0C850E8F48
:1011D0001D851F8F8CA29DA2AEA2BFA210E016C0DB
:1011E0000E94C9EC181694F4D501C4012CA13DA1AC
:1011F0004EA15FA1821B930BA40BB50BAC01BD01EB
:10120000485853416109710977FFCBC120E030E0B4
:1012100040EA51E46A857B858C859D850E94A3EA1E
:101220002D962FAD2D97322D432D2E965FAD2E97F7
:101230000E9457E687FF10C0E1E7FFE184918F012C
:101240000F5F1F4F1A830983882309F48BC10E9403
:10125000E193E981FA81F2CFD501C40129A93AA924
:101260004BA95CA9821B930BA40BB50BB7FD96C0D1
:101270000E94F0758AE00E94E193D501C401805379
:10128000984FAF4FBF4F89AB9AABABABBCAB0DA97F
:10129000011163C02EA93FA948AD59AD2D966FAD80
:1012A0002D97722D832D2E969FAD2E970E94C9ECFF
:1012B00018160CF041C028966CAD7DAD8EAD9FAD7B
:1012C00028970E945DE62D962FAD2D97322D432D48
:1012D0002E965FAD2E970E94A3EA6EAB7FAB88AFD0
:1012E00099AF2DA53EA54FA558A9280D391D4A1D1A
:1012F0005B1D2AAF3BAF4CAF5DAF2C966CAD7DADA7
:101300008EAD9FAD2C970E945DE69B01AC016A8576
:101310007B858C859D850E94A2EA2D962FAD2D9709
:10132000322D432D2E965FAD2E970E9457E6881FD3
:101330008827881F8DAB32C0D501C4012AAD3BADD3
:101340004CAD5DAD821B930BA40BB50BB7FD26C056
:101350004EAD5FAD62E67FE11EC020E030E040EAC6
:1013600051E46A857B858C859D850E94A2EA9B015C
:10137000AC012D966FAD2D97722D832D2E969FADBE
:101380002E970E9457E687FF09C022964EAD5FADAB
:1013900022976DE27FE18D810E942279D501C401FF
:1013A000880F991FAA1FBB1F2CA13DA14EA15FA1B1
:1013B000821B930BA40BB50B84199509A609B709D9
:1013C00081389F44A241B10580F0E8EEFEE18491AE
:1013D0008F010F5F1F4F1A830983882309F4C2C04E
:1013E0000E94E193E981FA81F2CF2AA13BA14E85C7
:1013F0005F85241735070CF027CEEBE8FEE18491DA
:101400008F010F5F1F4F1F830E83882329F00E94D7
:10141000E193EE81FF81F3CF1D8117FD03C006E14B
:1014200013E002C000EF13E01F830E836E817F8103
:101430008AE79EE10E9487C549815A816B817C8140
:1014400086E79EE10E9451C58AE00E94E1936E8189
:101450007F8185E69EE10E9487C5488959896A890E
:101460007B8981E69EE10E9451C58AE00E94E1935A
:101470006E817F8180E59EE10E9487C54C895D89F0
:101480006E897F898CE49EE10E9451C58AE00E94AA
:10149000E1931CA5112309F467C00D8107FF31C03A
:1014A00029813A814B815C81209334073093350741
:1014B00040933607509337072CEA35EC47E25EE35A
:1014C000688979898A899B890E94BCE66093300784
:1014D0007093310780933207909333072CEA35ECF1
:1014E00047E25EE36C897D898E899F890E947FEB4C
:1014F00060932C0770932D0780932E0790932F07EE
:1015000033C089819A81AB81BC8180933C079093E1
:101510003D07A0933E07B0933F072CEA35EC47E226
:101520005EE3688979898A899B890E94BCE6609319
:1015300038077093390780933A0790933B072CEA5A
:1015400035EC47E25EE36C897D898E899F890E9434
:101550007FEB60934007709341078093420790931D
:10156000430702C00E94037981E080933F10C35B70
:10157000DF4F0FB6F894DEBF0FBECDBFDF91CF9126
:101580001F910F91FF90EF90DF90CF90BF90AF90A1
:101590009F908F907F906F905F904F903F902F9093
:1015A00008950E851F85012B09F42BC148A459A469
:1015B0006AA47BA4480E591E6A1E7B1E28A539A565
:1015C0004AA55BA5281B390B4A0B5B0B6E817F81FB
:1015D000888599850E9436EAA30192010E9467EAF4
:1015E000DA01C9018C0D9D1DAE1DBF1D8431910511
:1015F000A105B105FCF06C017D018C3E9105A105B2
:10160000B1052CF05BEEC52ED12CE12CF12C20E89D
:10161000C216D104E104F104DCF08EEF90E0A0E00A
:10162000B0E08C199D09AE09BF098E839F83A887FE
:10163000B98712C044E1C42ED12CE12CF12C04E175
:1016400010E020E030E00E831F832887398704C034
:10165000CE82DF82E886F986EDEDFFE184918F018D
:101660000F5F1F4F882321F00E94E193F801F6CF0E
:10167000C701B6010E946D97E8EDFFE184918F01EB
:101680000F5F1F4F882321F00E94E193F801F6CFEE
:101690006E817F81888599850E946D97488D598DCF
:1016A0006A8D7B8D81ED9FE10E9451C54C8D5D8DD2
:1016B0006E8D7F8D8AEC9FE10E9451C50E851F853E
:1016C000033011050CF49DC06E817F81888599855A
:1016D0000E945DE620E030E040E850E40E94BCE675
:1016E00069837A838B839C83288D398D4A8D5B8DAA
:1016F0006C8D7D8D8E8D9F8D0E94A2EA2BED3FE03B
:1017000049E450E40E94BCE620E030E040E05FE3C2
:101710000E94BCE69B01AC0169817A818B819C812E
:101720000E947FEB69837A838B839C83C301B20120
:101730000E945DE62FE632E143E85AE30E94BCE6F0
:101740002B013C0149815A816B817C8184EC9FE1B2
:101750000E9451C5B301A2018EEB9FE10E9451C5C9
:101760002AE939E949E15FE369817A818B819C81CA
:101770000E94BCE669837A838B839C839B01AC01C6
:101780000E94A3EAA30192010E947FEB688B798BF0
:101790008A8B9B8B29813A814B815C81C301B20189
:1017A0000E94BCE620E030E040E05EE30E94BCE640
:1017B0006C8B7D8B8E8B9F8BEEEAFFE184918F018A
:1017C0000F5F1F4F882319F0FCD7F801F7CF49812D
:1017D0005A816B817C8188EA9FE10E9451C54889CA
:1017E00059896A897B8982EA9FE10E9451C54C89A7
:1017F0005D896E897F898CE99FE10E9451C58AE0ED
:10180000E0D78E819F81A885B9858C0D9D1DAE1D69
:10181000BF1D1D81B595A7959795879517FF03C0A7
:1018200080934D0705C02496EEADFFAD24978083CD
:101830000E851F850F5F1F4F1F870E871A85188F14
:101840000B85098F1C851A8F0D850B8F240135019F
:1018500011E0DCCCCF93DF93E6EEFDE18491EF0164
:101860002196882319F0ADD7FE01F8CF83E50E94B9
:10187000424C882321F00E94FC4B80935202ECE3FF
:10188000FEE18491EF012196882319F09AD7FE0199
:10189000F8CF80915202811103C0E8E3FEE102C05B
:1018A000E4E3FEE18491EF012196882319F089D7C2
:1018B000FE01F8CFECE2FEE18491EF01219688234E
:1018C00019F07FD7FE01F8CF209114043091150450
:1018D00040911604509117046091981870919918CE
:1018E00080919A1890919B180E94A3EAAB01BC01C9
:1018F0008AE29EE10E9451C520911804309119049A
:1019000040911A0450911B0460919C1870919D188D
:1019100080919E1890919F180E94A3EAAB01BC0190
:1019200087E29EE10E9451C520911C0430911D0464
:1019300040911E0450911F046091A0187091A1184D
:101940008091A2189091A3180E94A3EAAB01BC0158
:1019500084E29EE10E9451C5ECE1FEE18491EF0139
:101960002196882319F02DD7FE01F8CF2091140479
:10197000309115044091160450911704609146026D
:101980007091470280914802909149020E94A3EA17
:10199000AB01BC018AE19EE10E9451C5209118046F
:1019A0003091190440911A0450911B0460914A022D
:1019B00070914B0280914C0290914D020E94A3EADB
:1019C000AB01BC0187E19EE10E9451C520911C043E
:1019D00030911D0440911E0450911F0460914E02ED
:1019E00070914F0280915002909151020E94A3EA9F
:1019F000AB01BC0184E19EE10E9451C58AE0DF9108
:101A0000CF91DFC6FF920F931F93CF93DF93F82EF2
:101A1000092F162FEFE0FEE18491EF012196882334
:101A200019F0CFD6FE01F8CFEF2DF02F8491EF0102
:101A30002196882319F0C5D6FE01F8CFEDE0FEE12E
:101A40008491EF012196882319F0BBD6FE01F8CFCF
:101A5000612F70E080E090E00E946D978AE0DF9156
:101A6000CF911F910F91FF90ACC64F925F926F92F2
:101A70007F928F929F92AF92BF92CF92DF92EF921E
:101A8000FF92CF93DF93209114043091150440917D
:101A900016045091170460913204709133048091C0
:101AA0003404909135040E94A3EAAB01BC018AE0A2
:101AB0009EE10E9451C52091180430911904409173
:101AC0001A0450911B046091360470913704809180
:101AD0003804909139040E94A3EAAB01BC0186E06E
:101AE0009EE10E9451C520911C0430911D0440913B
:101AF0001E0450911F0460913A0470913B04809140
:101B00003C0490913D040E94A3EAAB01BC0182E039
:101B10009EE10E9451C540913E0450913F04609166
:101B20004004709141048EEF9DE10E9451C5809167
:101B30006F00982F927081FF05C080916F008D7F9C
:101B400080936F00409082105090831060908410BA
:101B5000709085108090861090908710A0908810CB
:101B6000B0908910C0908A10D0908B10E0908C10AB
:101B7000F0908D10992329F080916F0082608093FE
:101B80006F00E4EFFDE18491EF012196882319F0C5
:101B900018D6FE01F8CFC301B2010E946D97E0EFA5
:101BA000FDE18491EF012196882319F00AD6FE0108
:101BB000F8CFC501B4010E946D97ECEEFDE1849170
:101BC000EF012196882319F0FCD5FE01F8CFC7015B
:101BD000B6010E946D978AE0DF91CF91FF90EF9060
:101BE000DF90CF90BF90AF909F908F907F906F903D
:101BF0005F904F90E6C52F923F924F925F926F9207
:101C00007F928F929F92AF92BF92CF92DF92EF928C
